:020000040800F2
:1040000000500020C9E7000801BD000803BD0008FA
:1040100005BD000807BD000809BD0008000000003C
:104020000000000000000000000000000DBD0008BE
:104030000BBD0008000000000FBD0008CD8D00087A
:1040400011BD000813BD000815BD000817BD00080C
:1040500019BD00081BBD00081DBD00081FBD0008DC
:1040600021BD000823BD000825BD00080000000098
:104070000000000000000000000000000000000040
:10408000000000000000000035BD000837BD00083A
:1040900045BD000855BD000865BD000875BD000898
:1040A00077BD000879BD00087BBD00087DBD000814
:1040B0007FBD000881BD000883BD000885BD0008E4
:1040C00087BD000889BD00088BBD00088DBD0008B4
:1040D0008FBD000891BD00085186000895BD0008FD
:1040E0002946000899BD00089BBD0008000000009B
:1040F00000000000000000000000000000000000C0
:0C41000000000000000000005FF800005C
:1041100030BF704720BF704740BF7047BFF36F8FFD
:104120007047BFF34F8F7047BFF35F8F704701DF5A
:104130007047EFF31480704780F31488BFF36F8FDC
:104140007047EFF30980704780F309887047EFF3F9
:104150000880704780F30888704772B6704762B66F
:10416000704771B6704761B6704780F31188704729
:10417000EFF31280704740BA704700BA70470000F2
:1041800010B500F03DFA0A4C0A490B4A0B4B38B106
:10419000012020700A4808600A491860116010BDAB
:1041A00020700948086009491160094A1A6010BD69
:1041B000580E0020780E0020540F0020E80E00203A
:1041C000B98D0008039400082D890008CD870008E8
:1041D0007D8800082DE9F04175488AB0754E0121AF
:1041E00008F0FAFE0420012109F0DEF9032410256D
:1041F00042F2060330466946ADF800308DF80240C1
:104200008DF8035008F059FE062373616A4F4CF293
:1042100008634FF0040830466946ADF800308DF869
:1042200002408DF8038008F048FE0820012109F0C3
:10423000BBF941F6164338466946ADF800308DF8B3
:1042400002408DF8035008F038FE41F216433B61FE
:104250004FF400637B613846E8236946ADF80030CF
:104260008DF802408DF8038008F027FE28460121D2
:1042700009F09AF98DF80240504C4FF460472046FF
:104280006946ADF800708DF8035008F016FE012164
:1042900027614B4808F0A0FE00230A211A464FF47C
:1042A00000507061B4683061B068640458BF013276
:1042B000400448BF01330139F1D10A2A414A03D1F0
:1042C0000A2B01D1012300E000233948012113709A
:1042D00008F082FE042001213B4D09F065F94FF4FE
:1042E0008050002108F078FE0121042009F068F9CF
:1042F000284609F0DBFB04A8002409F05EFD4FF618
:10430000FF73284604A9ADF81430ADF81040ADF89D
:104310001640ADF8124009F02DFC224623462846EF
:10432000032109F002FE07A809F05AFD08262846D5
:1043300007A9ADF824600AF016F80423284607A957
:10434000ADF81C300AF00FF8284641F65F610AF01C
:1043500085F8AC842846012109F053FD0F21204641
:1043600008F064FE01254FF400430DEB06000293B4
:104370008DF80C408DF80D608DF80E5008F098FA0D
:10438000124B01A89A6822F480629A60DA6822F4DB
:104390008062DA6028238DF804308DF805408DF8AE
:1043A00006408DF8075008F093FE0AB0BDE8F08192
:1043B0000002300000080140000C014000100140E4
:1043C000000430008C0E0020000800400004014072
:1043D000104B82B01B78D3B10F4B04225A610222DA
:1043E0001A610022019201990C4A914202D8019A65
:1043F0000132F7E704221A6102225A610023019375
:10440000019A064B9A42E7D8019B0133F7E702B0C5
:10441000704700BF8C0E0020000C01403F0D0300D0
:1044200010B1012805D07047044B4FF400625A6167
:104430007047024B4FF480621A617047000C0140D4
:1044400010B1012805D07047044B4FF400621A6187
:104450007047024B4FF480625A617047000C014074
:1044600038B50546002445FA04F3DB07E0B202D56F
:10447000FFF7E6FF01E0FFF7D3FF0134082CF2D18C
:1044800038BD08B503281BD8DFE800F0020B101573
:10449000002004F0D9FDB0F5006F94BF002001208A
:1044A00008BD084B9868C0F3C01008BD054B98685C
:1044B000C0F3801008BD044B9868C0F3C03008BD3D
:1044C000002008BD000C01400008014040B1012857
:1044D0000BD1074BD86880F48060C0F38020704710
:1044E000034BD868C0F3C02070470020704700BF5E
:1044F000000C014038B500242546E0B2FFF7C1FFAB
:1045000018B10123A3401D43EDB20134082CF4D1AE
:10451000284638BD20B9034B9868C0F3C0007047E7
:1045200000207047000C014010B9C90805F07ABCA2
:10453000704708B108F076BE08F07CBE62B67047DE
:1045400072B6704718B9024B4FF400425A61704777
:104550000010014018B9024B4FF400421A61704735
:104560000010014013B503230446009340B100201E
:104570000246542106F03BFE00204A21074A07E08C
:104580000246542106F033FE20464A2140F2FF72D3
:1045900002B0BDE8104006F03CBE00BF01F8FFFFCE
:1045A000074B9A88C2F30722042A06D19A88D2B20E
:1045B000742A02D1188980B270470020704700BF6A
:1045C000006C004013B503230446009340B1002063
:1045D0000246342106F00BFE00202A21074A07E09C
:1045E0000246342106F003FE20462A2140F2FF72E3
:1045F00002B0BDE8104006F00CBE00BF01F8FFFF9E
:1046000008B5084B587E10F0010005D0002006F0D8
:10461000A2FE80F0080001E006F09DFEC0F3C0009D
:1046200008BD00BF08000020684620F007018D4645
:1046300001B54FF4004008F0A1F90F4B00211960BB
:104640000E4B0F48196000220023C0E900230D4BD8
:1046500099840D4B1B785BB903F1804303F58233DA
:104660009A6822F400429A60DA6822F40042DA6022
:10467000BDE80140854670478C0F0020700E002079
:10468000900E0020000800406805002030B9044B5F
:10469000D3E90023100A40EA036070470020704706
:1046A000900E002070B50C460646C0B9FFF748FFD3
:1046B0000B492246E317C1E90023D1E900452B024B
:1046C00043EA14632202C1E90023064B1E60064B35
:1046D0001E60064B9E84BDE87040FFF72FBF70BD83
:1046E000900E00208C0F0020700E0020000800406B
:1046F00010B9024B09011960704700BF980E0020E5
:10470000F8B9104B11F0040F9A680BD0C80602D507
:1047100042F4004208E022F400429A60DA6842F46F
:10472000004205E022F400429A60DA6822F4004276
:1047300001F00801DA6001F0FF02034B01B1012230
:104740001A7070470004014068050020064B4FF4C2
:1047500000721A60054B00201860054B4FF4807200
:1047600001461A60FFF7CCBF800E00207C0E0020AF
:10477000980E002038B5184B184C9A6812F0200596
:1047800001D0606838BD04F0C3FB2A46A060FF2159
:10479000032000F065FA01220546FF21032000F006
:1047A0005FFA40EA052010F002034FEA900018BFBC
:1047B0000123C204237303D5237B43F00203237335
:1047C000830403D5237B43F004032373236923EA83
:1047D0000000606038BD00BF000C0140680500208B
:1047E0005F4B70B59B68990600F1B980FFF7C2FF77
:1047F0005C498C694861A04234DDCB69051B9D4250
:10480000594B0CDA1C68D1E908236C43121943EBAD
:10481000E473C1E908238B6A1D448D6259E091F865
:104820002C6072070CD50C691A68041B624326F0D1
:104830000406D317C1E908238C6281F82C6033E0A9
:104840000E691B68241A344404FB0334D1E908239D
:10485000121B63EBE473C1E90823F6438B6A35440A
:104860002B4411E035DACB69221A9A423E4B0DDA1D
:104870001D68041B5543D1E90823521B63EBE57304
:10488000C1E908238B6A23448B6222E091F82C5003
:104890006A070ED51A6825F004054243D317C1E90B
:1048A0000823886281F82C5000220023C1E90C23E0
:1048B0000FE00A691D680132041B14446543D1E905
:1048C0000823521943EBE573C1E908238B6A1C44A2
:1048D0008C628C6A8D6BCA6B651B85EAE576A6EBEC
:1048E000E57696421F4B2ED99E681A6CB21A642A3E
:1048F00029D91E6442F2107675435A6495FBF2F290
:104900003C256A431E699C63013692FBF6F29A6469
:1049100040F6B834002AB8BF5242A24201DDC82294
:1049200003E0B2F57A7F02DD6422DA6316E0322A10
:1049300001DD0A22F9E70A2A01DD0522F5E7012A4D
:104940000CDD0122F1E78C680A6C064BA21AB2F565
:10495000FA6F03D90122DA6300229A64886170BD7C
:10496000000C0140680500200400002008B568B96B
:10497000FFF736FF0649D1E90823D1E90C01121AE5
:1049800063EB0103100A40EA036008BD002008BD84
:104990006805002038B50D46F8B9104CFFF720FF28
:1049A000D4E908012269002871F100034FEA0222CC
:1049B00002DA404261EB4101D3170BF0DDFFC4E99D
:1049C0000C23E9170B022A02D4E90C0143EA156310
:1049D000121843EB0103C4E9082338BD6805002021
:1049E00010B9024B09011960704700BF0400002094
:1049F00010B9024B83F82C10704700BF68050020E7
:104A0000014B986C704700BF6805002010B9024B3D
:104A1000187B7047002070476805002038B5214B8F
:104A2000214A1B69214C5909090103F01F03116038
:104A30000320FE21002284F82C3000F011F94021DF
:104A40000122032000F00CF900210A46032000F0A7
:104A500007F9002105460122032000F001F9082D85
:104A600005D140F6FF7323614FF4006304E040F288
:104A7000FF3323614FF40073E72100220320E36139
:104A800000F0EEF800210122032000F0E9F8FFF722
:104A900071FEA0610002C117C4E90C01C4E908015C
:104AA00038BD00BFEC0E0020040000206805002087
:104AB00008B5082004F0C8FA5E2805D9074B93F81A
:104AC0004C2052B9012206E0082004F0BDFA542817
:104AD00003D8024B002283F84C2008BD6805002053
:104AE000044B93F84C00013801288CBF00200120B2
:104AF000704700BF68050020044B93F84C00012864
:104B000006BF022283F84C20002070476805002071
:104B100008B5FFF72FFE052808D9FFF72BFE40F256
:104B2000F933984294BF0020012008BD012008BD40
:104B30002DE9F04F4FF4804089B0012108F040FD8D
:104B4000434C0120014608F02FFD03264FF420437B
:104B50004FF0180A204602A9ADF808308DF80BA0D6
:104B60004FF0040B8DF80A6008F0A7F94FF480436A
:104B7000204602A9ADF808308DF80A608DF80BB018
:104B800008F09BF90823ADF81830324B00240125BA
:104B90004FF482794FF002084FF40077184603A9CA
:104BA000ADF80C40ADF81040ADF81A40ADF81C401F
:104BB0000193ADF80E90ADF81280ADF81450ADF839
:104BC000167008F0A9FD019B2946184608F02AFE38
:104BD00029464FF4805008F0E7FC2846214608F0AB
:104BE000FBF98DF80BA0DFF874A0A023504602A9B2
:104BF000ADF808308DF80A6008F05FF940235046A0
:104C000002A9ADF808308DF80A608DF80BB008F0F5
:104C100054F9ADF80C40ADF81040ADF81A40ADF8BD
:104C20001C400D4C2823204603A9ADF81830ADF8E0
:104C30000E90ADF81280ADF81450ADF8167008F073
:104C40006BFD2046294608F0EDFD09B0BDE8F08F68
:104C5000000C0140003800400030014000080140D5
:104C600070B504460D461646032866D8DFE800F006
:104C70000205080D4FF480520FE04FF4804201E02E
:104C80004FF400522E4B5A611BE02E4910220B8824
:104C900023F002031B041B0C0B802B4B5A61294889
:104CA000022108F043FE0028F9D02648294608F0E2
:104CB000E9FD2448012108F039FE0028F9D08EB919
:104CC0002EE02248022108F031FE0028F9D01F48CA
:104CD000294608F0D7FD1D48012108F027FE0028CD
:104CE000F9D0ECE7032C28D8DFE804F002070A0F1C
:104CF000154B4FF480521A611AE04FF4804201E0E4
:104D00004FF400520E4B1A6110E00F4B10221A6143
:104D1000A3F554431A8892B242F002021A8007E0C7
:104D2000032C0AD8DFE804F004020204074800E07C
:104D3000044808F0A9FDC0B270BD002070BD00BFDE
:104D40000010014000380040000C014000300140DC
:104D500037B5C44DA8786B782C4608B1042205E31A
:104D6000A52B00F05A8269D8852B00F02B8127D81B
:104D7000072B00F05B810FD8032B00F0238105D8AF
:104D8000012B00F0F08040F2E480FBE0052B00F006
:104D9000348140F222813CE1812B00F0E48009D88B
:104DA0000D2B00F06F81802B00F0D3800C2B40F096
:104DB000DC8247E1832B00F0108140F27581E1E055
:104DC000952B00F08F811FD88C2B00F0828110D89A
:104DD000872B00F07081C0F010818A2B40F0C582D3
:104DE0000020142101AA06F0BBFAEB788DF80630FA
:104DF00064E1932B00F0468100F224818D2B40F07A
:104E0000B48200201A2151E1A02B00F0DB8109D8E7
:104E1000992B00F07E819A2B00F0A081962B40F018
:104E2000A4826EE1A22B00F0DA81C0F0D181A32B25
:104E300000F0DC81A42B00F0E08196E2B72B00F0BB
:104E40005E8238D8AD2B00F0318215D8A92B00F046
:104E5000128205D8A72B00F0008240F2EE8103E217
:104E6000AB2B00F00E8200F21382D5F80310002065
:104E7000C9B204F07BFF7BE2B12B00F02B820BD890
:104E8000AF2B00F0198200F21E82D5F8031000202B
:104E900049B204F0BDFF6BE2B52B00F0218200F2B5
:104EA0002482B22B40F06182D5F803100020C9B2F1
:104EB00004F0FCFF5CE2CC2B00F0758120D8C22B03
:104EC00000F05D810ED8C02B00F0B08000F253815D
:104ED000B82B40F04A82D5F803100020C9B204F084
:104EE00091FE45E2C72B00F09480C82B00F04B8167
:104EF000C32B40F03A82D5F803205B4B5A6037E26F
:104F0000D52B00F05A810ED8D22B00F00482D42B7E
:104F100000F04E81D12B40F028820020D5F80310FC
:104F2000FFF738FD24E2D82B00F0068207D8D62BF5
:104F300040F01B82D5F803204B4B9A8318E2D92B03
:104F400000F00082DA2B40F01082D5F80320474BA6
:104F500009E205F0F7F820B9A178490101F0E00174
:104F60000BE0062202E205F0EDF80028F9D1A17865
:104F7000490141F0020101F0E201D4F8032006F0FA
:104F80005AF9F5E105F0DEF805460028E9D1A178E7
:104F9000D4F80320490141F0080101F0E80106F0CE
:104FA00038F9A178D4F80320490141F0060101F055
:104FB000E6012846002AB8BF524206F02AF9A37833
:104FC000012117E005F0BEF80028CAD1A1784901F7
:104FD00041F00A0101F0EA0168E00621D4F803205B
:104FE000002006F016F9D4F80310A378204A42F8FE
:104FF000231000211F4AD154BAE1D4F80310002035
:1050000006F021FAA378D4F803101B4A42F82310C3
:105010009FE01A4B01221A70E178134B5972184B1A
:105020001B78022B40F0A481002071E1134B012278
:105030001A70E1780C4B9972114B1878002840F0E7
:10504000978165E101AA0020142106F089F9D4F8BE
:1050500003209DF8053012B143F0020321E023F054
:1050600002031EE0CC090020EC0E00207C0E002084
:10507000500E0020B80500204C0A0020500F0020E0
:10508000530F002001AA0020142106F069F9D4F87A
:1050900003209DF8053012B143F0010301E023F035
:1050A00001038DF8053009E000200421D4F8032025
:1050B00006F0AFF85CE100200E21F7E7A1780020B0
:1050C000490141F0140101F0F40101AA06F07CF855
:1050D0004EE1E978A74BD972C1F10801C9B204F0D9
:1050E00043FD45E101AA142106F03AF9D5F8032061
:1050F0009DF8053012B143F00403D2E723F0040316
:10510000CFE7D5F803209C4B002A00F03081012224
:105110002DE101AA0020182106F022F9EA789DF875
:10512000053002F00F0223F00F031343A178002093
:10513000490141F0180101F0F80101AA8DF805308C
:1051400006F042F88D4BA07853F8201006F07BF95A
:10515000A3788B4A134400225A7009E101AA002067
:10516000182106F0FDF89DF80530EA7803F00F03EA
:1051700043EA0213DAE7EA787E4B1A72F8E0D5F8D0
:1051800003207C4BEFE07F4B01221A70794BD5F85E
:105190000320DA777C4B1B78032B40F0E9807B4BB4
:1051A0000020D978B4E0D5F80320724BDA81DFE033
:1051B000D5F803206F4B5A61DAE0D5F803206D4B28
:1051C0009A77D5E0D5F80310C9B204F0DBFCCFE044
:1051D000D5F803100020C9B204F0E0FCC8E0D5F80F
:1051E00003100020C9B204F0F9FCC1E0D5F80310A7
:1051F0000020C9B204F0FCFCBAE0002004F05AFD23
:10520000D5F8031020B9A878C9B204F005FDAFE0C5
:10521000A878C9B204F028FDAAE004F04BFDAB78F1
:10522000D5F8031020B91846C9B204F0FFFC9FE07E
:105230001846C9B204F02CFD9AE0002004F03AFDB3
:10524000D5F8031020B9A878C9B204F0F9FC8FE0B2
:10525000A878C9B204F012FD8AE0D5F80310002046
:10526000C9B204F0F7FC83E0D5F803100020C9B2FE
:1052700004F068FD7CE0D5F80310C9B204F06CFDC1
:1052800076E0D5F803100020C9B204F079FD6FE094
:10529000D5F803100020C9B204F07CFDAA783C4B7D
:1052A00003EBC203D5F803205A7161E0D5F803106F
:1052B000C9B204F0A3FD5BE0D5F803100020C9B229
:1052C00004F0D6FD54E0D5F803100020C9B204F074
:1052D000D9FD4DE0D5F80310C9B204F0DDFD47E07B
:1052E000D5F80320234B9A6142E0D5F80300284B00
:1052F000186000283CD1597904F04CFD38E0244B6B
:10530000D5F803201A71204B1B78012B30D1E97896
:10531000FFF70AF92CE0D5F80320164BE9781A615B
:10532000002001F01F01FFF763FBD5F80310A878F8
:105330004911FFF755FB1BE00020D5F80310FFF7DC
:10534000B1F915E0E978D5F80320124BA87801F0FF
:105350001F011A60FFF7D4F9D5F80310A878491196
:10536000FFF7C6F904E01A6002E003220A4B1A7044
:1053700003B030BDEC0E00205A0F00204C0A002074
:10538000B8050020500F0020530F0020CC0900204A
:10539000640E0020800E0020400A002037B5824DA8
:1053A000824CAA786B7812B1042323704EE2DB2B77
:1053B00000F23A82DFE813F0DC00DF00E500E800ED
:1053C000ED00EF00F100F40002011D0133012201A4
:1053D0000B0115013802380238023802380238024F
:1053E00038023802380238023802380238023802ED
:1053F00038023802380238023802380238023802DD
:1054000038023802380238023802380238023802CC
:1054100038023802380238023802380238023802BC
:1054200038023802380238023802380238023802AC
:10543000380238023802380238023802380238029C
:10544000380238023802380238023802380238028C
:10545000380238023802380238023802380238027C
:10546000380238023802380238023802380238026C
:10547000380238023802380238023802380238025C
:10548000380238023802380238023802380238024C
:10549000380238023802380238023802380238023C
:1054A000380238023802380238023802380238022C
:1054B0003802380238023802DC00DF004101ED001A
:1054C000E500E800EF0044013802380247013802E5
:1054D0004F015501380238023802380238021501EE
:1054E0000B01580162013802380264016E01220189
:1054F0003301020138023802AA01AE01B201B6013D
:10550000BA01C601D201DE01E201E601EA01EE01C3
:10551000F201F501F901FD010102050209020D0286
:1055200011021402170219021C0238023802380252
:105530003802380238023802F40077017A017C011F
:105540007F0181013802F1008301380238023802FC
:105550008601380289018B019F0120022402380252
:10556000A101A401A70127022E02320234022A025D
:105570000020014601E00020022106F0EFF8606003
:1055800054E10020082101E000200A2105F0FFFE7F
:10559000F5E7074B45E1074B43E1074B5B7A41E1F8
:1055A000054B9B7A3EE100BFCC090020400A002059
:1055B000500E00204C0A0020EC0E0020002005F0C8
:1055C000CAFEAB785B00184100F001032AE100201D
:1055D000142101AA05F0C4FE9DF80530C3F3400371
:1055E00020E10020142101AA05F0BAFE9DF8053043
:1055F00020E0974B9B68C3F3C03313E101AA00205E
:105600007C2105F0ADFEAA780223520003FA02F2D3
:105610009DF806301A420CBF0023012302E101AAC3
:1056200000207C2105F09CFEAB789DF806205B00F5
:1056300042FA03F303F00103F4E000200421A5E79C
:1056400000200E21A2E70020142101AA05F088FE07
:105650009DF80630E6E0002004F0A8FAC0F108004A
:105660008DE700201A2191E70020142101AA05F0FE
:1056700077FE9DF80530C3F38003D3E0754BADE0B2
:105680000020182101AA05F06BFE9DF8053003F0FB
:105690000F03C7E00020182101AA05F061FE9DF864
:1056A00005301B09BEE06C4B1B7ABBE06A4BB8E0CF
:1056B000694B5B68B6E0694BB3E0694BB1E0664BA0
:1056C000DB7FAFE0644BDB89ACE0664BA9E0AB78F5
:1056D000654A0021D05C616010B1644801254560D5
:1056E000D154634AD15C19B1616841F00201616033
:1056F0000021D1549AE05F4B70E0574B5B6991E019
:10570000554B9B7F8EE0544B9B8B8BE0002004F02D
:1057100055FA34E7002004F059FA30E7002004F08D
:10572000C1FA2CE7002004F0C5FA28E7002004F0B5
:10573000C1FA18B9A87804F0CDFA20E7A87804F0E7
:10574000E9FA1CE7002004F0B5FA18B9A87804F0CB
:10575000C9FA14E7A87804F0EDFA10E7002004F085
:10576000A9FA18B9A87804F0C5FA08E7A87804F0EF
:10577000D9FA04E7002004F0C5FA00E7002004F09D
:1057800013FBFCE6002004F019FBF8E6002004F00F
:105790001DFBF4E6002004F021FBF0E6364B5B79BC
:1057A00040E0002004F048FBE9E6002004F04EFB56
:1057B000E5E6002004F0B2FBE1E6002004F0B6FBD1
:1057C000DDE6002004F0BAFBD9E6002004F0BEFBC1
:1057D000D5E6002004F0CAFBD1E6284B1B7821E077
:1057E0001D4B9B691EE0244B1BE0234B1B7919E0EA
:1057F000002004F067FAC2E60020FFF7B7F8BEE623
:10580000154B1B690EE0FEF7B5FFB8E60020FFF769
:10581000FDF8B4E60020FEF739FFB0E6184B00E0D3
:10582000184B1B68636001E003232370164B1B7841
:1058300063B1164B62681A60154B1AB91A6842F0C8
:10584000080202E01A6822F008021A6003B030BDB4
:10585000000801405A0F0020EC0E00205C0E0020D2
:10586000100F0020880E0020E40E0020400A0020C7
:105870006D0E0020E50E0020640E0020620E002058
:10588000800E00207C0E00203B0A00202C0A002005
:10589000D409002038B5B14A95781446022D00F09D
:1058A0004281032D00F04681002D40F0C5815378E0
:1058B0004F2B00F0BE803BD8462B00F0918014D8CF
:1058C000422B7BD009D8402B74D0412B40F0B281C1
:1058D000D178A34B0020197074E0442BA04A75D0F6
:1058E0007AD8E178042011716CE0492B00F08B80AC
:1058F0000AD8472B7FD0482B40F09C81D378984919
:10590000262001F8263FE3E04C2B00F088804D2B49
:1059100000F08A804B2B40F08D81914CD178032090
:10592000E17002F054FCE078BDE8384002F024BF9A
:10593000572B00F0DB8013D8522B00F0A18006D843
:10594000502B00F08980512B00F08B8072E1542B9A
:1059500000F0B380C0F09B80552B00F0BB8069E164
:10596000832B00F0D1801AD8592B00F0C5805A2B18
:1059700040F060817A4DD378294601F8283F2820ED
:10598000012202F083FC95F82800BDE8384010F0B1
:1059900001001ABF00200121014605F02DBF852B13
:1059A00000F0BC80C0F0B580FF2B40F04381D2787E
:1059B0006C4B43E140F2FF70D17803E0D178684B43
:1059C00001205970BDE8384002F001BCD4F8033022
:1059D0001C20D361644909E0E17805205171F1E7A9
:1059E000D2F803305E490C2041F80C3F0422BDE898
:1059F000384002F04BBC5A4DD2F80330294641F8EA
:105A0000083F08204AE0D278554B0AB9DA7503E01E
:105A100056490122DA754A601720D97DD2E7D1783C
:105A20004F4B02209970CDE7D1784D4B1520597519
:105A3000C8E7D2F803104A4CC9B21920617602F0C7
:105A4000C6FB607E10F001001ABF28460121014606
:105A5000BDE8384005F0BEBED178414B162099759F
:105A6000B0E73F4B1A7D1D4612F0010F04D0E378DA
:105A7000DB0701D402F00FFBE17814202975A1E7C0
:105A8000D2F803303649202041F8203FAEE7344DAC
:105A9000D2F80330294641F8103F1020042202F0CA
:105AA000F5FB334B1B78002B40F0C9806879A9685F
:105AB0002A69BDE8384002F099BFD2F80330012BC3
:105AC00000F2BA80254B2649DB781A2001F81A3FEC
:105AD00001228CE7D2F80330012B00F2AD801F4B7E
:105AE0001F49DB781B2001F81B3FF1E7D3781C49E5
:105AF000272001F8273FEBE7D2F80330184924208C
:105B000021F8243F022272E7D2F80320194B5A6091
:105B100038BDD2F80320184B1A6038BDD2F80320E4
:105B2000144B9A6038BD5178144BD2F8032043F8D7
:105B3000212038BD5378272B64D02ED8022B4AD091
:105B400020D8002B3ED0012B74D10D4BD2F803206E
:105B50005A6003F0DDF9074B186138BDCC0900200D
:105B6000080000203A0A002024000020400A0020FB
:105B7000580E0020B80500203C0A0020500A0020E2
:105B8000140F00201B2B2FD01C2B34D0092B51D1EC
:105B9000D2F803202A4BDA6038BD2B2B3BD007D834
:105BA000292BD2F80320264B31D032D85A6138BD88
:105BB0002D2B3AD034D32E2B3CD1D2F80320204BBE
:105BC000DA6238BD1E4BD2F803201A6003F0A0F948
:105BD0001C4BD86038BD1A4BD2F803209A6003F0F2
:105BE00097F9184B586138BD0020D2F80310BDE872
:105BF000384005F014BD0020D2F80310BDE838404D
:105C000005F037BDD2F803200D4B1A6138BD9A61FB
:105C100038BDDA6138BDD2F80320094B1A6238BDAD
:105C2000D2F80320064B5A6238BDD2F80320044B49
:105C30009A6238BD032200E00422034B1A7038BD7B
:105C4000140F0020B8050020400A00202DE9F84379
:105C5000054614460E4600294DD000284BD08142FF
:105C600049D04FEA42185FFA88F848F006073946EB
:105C7000002005F073FD48F00C018146002005F07E
:105C80006DFD804628460AF039FC054630460AF08C
:105C900035FC014628460AF03DFD064648460AF016
:105CA0002DFC31460AF036FD0AF046FE0546404618
:105CB0000AF024FC31460AF02DFD0AF03DFE002DCD
:105CC00008BF01250D49002814BF80464FF0010888
:105CD00030460AF009FE0A4E30B12046414605F032
:105CE000B2FB331901225A70002039462A4605F0CA
:105CF000A2FA01233355BDE8F88300BF0000A0419C
:105D0000B805002038B50E4D04462B5C63B10D4B31
:105D1000410141F0060153F82420002001F0E60182
:105D200005F077FA00232B5525446B783BB1064BE1
:105D3000E0B253F8241005F086FB00236B7038BDE9
:105D4000B8050020500E00204C0A00202DE9F34138
:105D5000B94EBA4F3378D6F803006422222B7B70F9
:105D60003A70786035463C4601F038815BD80F2B9D
:105D700000F0B08526D8072B00F0D28111D8032B74
:105D800000F0D88007D8012B00F0BD80022B00F076
:105D9000C58001F083BB052B00F0BA8140F2DF80A3
:105DA000BAE10B2B00F0F08405D8092B00F0A58395
:105DB00040F27982A5E30D2B00F0198540F20185B0
:105DC00000F060BD192B00F0D68614D8152B00F01A
:105DD000358607D8132B00F0C085142B00F00C86F5
:105DE00001F05CBB172B964B00F0AB8600F2B68639
:105DF000D86101F0FFBB1E2B00F0D7840CD81B2B01
:105E000000F0DB86C0F0C8861C2B41F047838C4B2A
:105E100000221A7601F0EEBB202B01F0378040F211
:105E2000FC8701F075B8812B01F0618135D8412BD9
:105E300001F04B8117D8252B01F00B8107D8232BBC
:105E400001F0D380242B01F0D78001F027BB272B52
:105E500001F02D81C1F00681402B41F01F8303F03A
:105E600032FC01F0C7BB452B01F0388108D8432B29
:105E700001F02E8101F22F8103F027FC01F0BABB63
:105E8000472B01F03181C1F02C81802B41F006833A
:105E90006B4B00221A7601F0ADBB882B01F0B68166
:105EA0001BD8842B01F054810DD8822B01F0338153
:105EB000832B41F0F382624B002183F8441083F876
:105EC0002C1101F02CB9862B01F0538101F2D38102
:105ED0005B4B00221A7601F08DBB8C2B01F02682E1
:105EE00006D88A2B01F0068241F2EC8101F019BA42
:105EF000F22B01F08382FF2B01F0C6828D2B41F043
:105F0000CD8201F037BAB37853B904F01BF90028F9
:105F100001F0F0820623237001F06CBBB3781BB153
:105F20000423237001F066BB04F00CF9002801F093
:105F30000683EFE7B578002DF2D1424B28461D705D
:105F4000414B1D7005F094F828462946022205F0C1
:105F500036FA2846082105F0E7F901F04BBB04F0BA
:105F6000F1F80028D6D1B378002B40F09980324B5D
:105F70005B78032B00F2C880DFE803F002296C96FF
:105F80000020FFF7BFFEB1782F4B00245C542D4B4F
:105F90002E4E5C5401238B403278490122EA0303E0
:105FA000204601F0E001D5F80320337005F043F9F5
:105FB000A9782246204605F002FAAB78244901EB85
:105FC0004312927F002A41F0E18201F013BB0020CE
:105FD000FFF798FEB3781C4A0026D654194A30467B
:105FE000D6545B0143F0020101F0E20105F0B6FB7B
:105FF000A97801238B40154FD5F803803A78804467
:10600000490122EA0303304601F0E00142463B70B9
:1060100005F011F930463246A97805F0D0F9A87894
:106020000B4AC4F8048002EB40139B7F002B41F025
:10603000C68201F0DFBA00BFCC090020400A002070
:10604000B8050020E40E00206D0E0020610E002037
:10605000EC0E0020D5F80330CC4E142B20DCCC4ABB
:10606000002052F82350FFF74DFEB17801228A40FC
:10607000C84B00245C54C84B5C54C84B4901187889
:1060800001F0E00120EA02021A7020462A4605F0DB
:10609000D2F82046B178224605F091F901F0AABA6B
:1060A0000423237001F0A6BAD6F80330B74C142BA2
:1060B00001F3A0820221002005F050FBA378D4F860
:1060C0000310B34A194452F82160002506441846CB
:1060D000FFF718FEA17801228A40AE4B5D54AE4B0B
:1060E0005D54AE4B4901187801F0E00120EA02024C
:1060F0001A702846324605F09EF82846A1782A46AE
:1061000005F05DF901F076BA03233B7001F072BA35
:10611000FEF71EFE01F06EBAFFF740F901F06ABA11
:10612000B078737800287FF4FBAE9A2B2AD8992B8D
:106130007FD2822B6BD00BD8062B5AD003D8042BDE
:1061400051D0052B0AE0072B5AD00C3B012B11E054
:106150008C2B61D00AD8832B45D0862B40F09F80B2
:1061600000200C2105F023FA01F044BA8D2B5AD0FF
:10617000933B022B00F293800020142105F017FAC4
:1061800001F038BAC72B34D012D8C12B5DD004D857
:10619000B52B53D0C02B33D081E0C22B5CD0C32BA6
:1061A0007DD144207E49042202F070F801F022BA29
:1061B000D22B5FD00AD8C82B55D0CC2B6FD14E2014
:1061C0007849022202F062F801F014BAD52B58D0B7
:1061D000D62B5DD0D42B62D154207349042202F017
:1061E00055F801F007BA0020062105F0E0F901F0AA
:1061F00001BA6E4B4920597A01F0E9FF01F0FAB972
:106200006A4B4A20997A01F0E2FF01F0F3B90421C8
:1062100005F0CDF901F0EEB94B206549012202F0FD
:1062200035F801F0E7B900201A2105F0C0F901F0B6
:10623000E1B9182105F0BBF901F0DCB958205D493E
:10624000042202F023F801F0D5B9584B4820197AFE
:1062500001F0BDFF01F0CEB940205749042202F001
:1062600015F801F0C7B95F205449012202F00EF879
:1062700001F0C0B950205249042202F007F801F0A1
:10628000B9B95E204F49012202F000F801F0B2B91D
:106290005C204D49022201F0F9FF01F0ABB9032364
:1062A000237001F0A7B97378B678384F002E7FF4C9
:1062B00037AE952B3ED8932B80F0CC800D2B0DD88C
:1062C0000C2B80F0C780052B00F0A28001D8042B96
:1062D0000CE0062B00F0B780072B4DE0862B00F07A
:1062E00097801BD8822B00F0BB80832B40F001816C
:1062F0000020062105F038F9AC780020610141F05A
:10630000060101F0E60105F042F8304B304A43F84F
:106310002400AB780021D15401F06CB98C2B00F033
:10632000A5808D2B40F0E58030461A2105F01CF940
:1063300001F060B9C32B00F0C0804DD8B52B00F040
:10634000A78013D8993B012B00F2D3803046182147
:1063500005F00AF91F4BB87853F8201005F073F8D0
:10636000BB781B4A13445E7001F044B9C12B00F0A6
:10637000968000F29B80C02B40F0BB804A2001F049
:10638000FFFF0A4B987201F035B900BFCC0900201D
:10639000D80900206D0E0020E40E0020610E0020C0
:1063A000F00E0020FA0E0020000F0020EC0E00205E
:1063B000F70E0020040F0020EC0E00200B0F002031
:1063C000FC0E00200A0F0020080F0020500E0020B5
:1063D000B80500204C0A0020CC2B75D00BD8C72B59
:1063E00031D0C82B40F085805F20AA49012201F0FE
:1063F000E0FF01F0FFB8D52B6DD0D62B72D0D42B97
:1064000077D15420A449042201F0D3FF01F0F2B85F
:1064100000200C2105F0A8F8AC780020610141F0C3
:106420000C0101F0EC0104F0B2FF9C4B9C4A43F8D4
:106430002400A87800210244517053F8201005F080
:1064400002F801F0D7B8492001F09AFF954B587235
:1064500001F0D0B80020142105F086F801F0CAB888
:106460003046042105F080F801F0C4B88D4C4B2073
:1064700004F10B01012201F09CFFB87804EB4014F9
:10648000E17AC1F10801C9B203F06EFB01F0B2B8C4
:1064900058208549042201F08CFF01F0ABB8482058
:1064A00001F06EFF7F4B187201F0A4B840207F49C5
:1064B000042201F07EFF01F09DB844207C490422B3
:1064C00001F077FF01F096B84E207A49022201F0E0
:1064D00070FF01F08FB85E207749012201F069FF5B
:1064E00001F088B85C207549022201F062FF01F0DA
:1064F00081B80323237001F07DB8FFF7CBF901F0D9
:1065000079B8B2786E4B022A00F0B180032A00F00D
:10651000B380002A40F020815B78512B00F0868008
:106520002CD8472B70D014D8432B68D00AD8412BD5
:1065300060D061D8402B40F00D8140F2FF7001F037
:106540001FFFF0E0452B5F4A5CD040F28380D368A8
:10655000FEE04C2B61D008D8492B5BD056D34B2B97
:1065600040F0F880574BDB78F2E04F2B58D05AD8E8
:106570004D2B40F0EF80534B5B7DE9E0802B66D0E4
:1065800013D8552B59D005D8532B4E4A51D052D839
:10659000136ADDE0592B53D05A2B54D0572B40F0BF
:1065A000D980484B93F82730D2E0842B56D008D8B6
:1065B000822B3B4A4ED04FD8137E1E1F734273412D
:1065C000C6E0F02B4CD00DD8852B40F0C380344A68
:1065D0003D4993684B4303F540533933936023F0AF
:1065E0000043B5E0FE2B3BD0FF2B40F0B380374B90
:1065F0001B7838E0334B34E0324B5B78A8E0314B0A
:106600001B79A5E05379A3E02E4B87E02D4B93F83F
:1066100026309DE02B4BDB7D25E02A4B9B7897E0D5
:10662000284B5B7E94E0274B9B7D91E0254B1B7DA7
:106630008EE013698CE0937E8AE0224BDB7E87E05C
:10664000204B9B8C84E01F4B93F8283080E0144B48
:106650001B7E7DE0D3697BE0536879E01C4B5AE0F8
:106660001C4B1B7874E0003318BF012370E05A788C
:10667000194B53F822306BE05B78272B59D038D870
:10668000022B4AD02CD8002B44D0012B62D1134BC3
:106690005B685DE00B0F0020000F00204C0A00201B
:1066A000B8050020EC0E0020040F0020EC0E0020A6
:1066B000F00E0020FA0E00200A0F0020080F002024
:1066C000CC090020080000206D4EC6413A0A002087
:1066D0003C0A0020480F0020500A0020140F002020
:1066E0001B2B1DD01C2B20D0092B33D1A04BDB68DA
:1066F0002EE02B2B24D005D8292B9D4B1CD01DD848
:106700005B6925E02D2B21D01DD32E2B22D1984B58
:10671000DB6A1DE0964B1B681AE0954B9B6817E0FF
:10672000002004F0D0FF606018E0002004F0E0FFDB
:10673000F9E78F4B1B690BE09B6909E0DB6907E018
:106740008B4B1B6A04E08A4B5B6A01E0884B9B6AB7
:10675000636003E0032300E004232370854B1B7870
:10676000002B00F04787844B62681A60834B2AB97C
:106770001A6842F008021A6000F03CBF1A6822F062
:1067800008021A6000F036BFB378022B15D1737877
:10679000372B0ED87A4903F5A770800001EB8301EF
:1067A000042201F073FD00F025BF7378142B40F232
:1067B00002830323237000F01DBF04233B7000F00D
:1067C00019BFB378022B0ED16E4B5B78372BF0D804
:1067D0006B4903F5A770800001EB8301042201F0EF
:1067E000E8FD00F007BF04233B7000F003BFB3785F
:1067F000002B7FF495AB6B78624E012B21D002D336
:10680000022B23D03AE003F09DFC00287FF482ABFA
:10681000B07804F025FCB17839B95B4B01221A70CD
:106820005A4B00221A7000F0E5BE594A937F002BA4
:1068300000F0E08602EB4112927F9A4240F0DA8645
:10684000EBE7002004F014FC00F0D4BE002004F0BC
:1068500017FC484B78601B78002B00F0CB86464B2A
:106860001860464B1A6820B942F008021A6000F01E
:10687000C1BE22F008021A6000F0BCBE03233B70C8
:1068800000F0B8BEB37813B1022B04D01EE0FDF7C0
:1068900069FE00F0AFBE3B4B5B78072B0AD820B9EE
:1068A0001846FDF7BDFD00F0A5BE1846FDF7C8FD72
:1068B00000F0A0BEFF2B7FF47CAF451C0ABF2E4B1F
:1068C000C0B21878FDF7CCFD00F094BE04233B70F5
:1068D00000F090BEB378012B23D005D3022B24D136
:1068E0007078FDF7F3FD0DE07078082802D8FDF709
:1068F000C8FD07E00A2801D100230BE00B2803D1D3
:10690000FEF706F9606012E00C2805D1214B9B6868
:10691000C3F3C03363600AE0FF2808D1FDF7EAFD46
:10692000F0E7707802F090FBECE704233B70114B2A
:106930001B78002B00F05E860F4B62681A600F4BCD
:106940002AB91A6842F008021A6000F053BE1A68A9
:1069500022F008021A6000F04DBE7278064B092A38
:106960003BD8DFE802F0191C1F22262C2F323539C4
:10697000140F00203B0A00202C0A0020D40900201C
:10698000500A0020CC090020B80500206D0E002020
:10699000EC0E0020000801401A6810441CE01A6840
:1069A000101A19E01A68504316E01A6892FBF0F0CA
:1069B00012E01A6892FBF0F100FB11200CE01A685B
:1069C000104009E01A68104306E01A68504003E0DE
:1069D0001A68D2431A6000E018601A68A34B2AB9FB
:1069E0001A6842F008021A6000F004BE1A6822F029
:1069F00008021A6000F0FEBD9D4B1A689B4B824254
:106A0000196804DD21F0030141F0040108E00BBF27
:106A100021F0060121F0050141F0010141F00201E0
:106A200019602AB91A6842F008021A6000F0E2BD43
:106A30001A6822F008021A6000F0DCBD73780C2B93
:106A400000F2D885DFE803F0071019222B343E4707
:106A50005059626B7400854B1B681C0740F1CA8556
:106A6000844BD86100F0C6BD804B1B68190700F14C
:106A7000C185804BD86100F0BDBD7C4B1B68DA0737
:106A800040F1B8857B4BD86100F0B4BD774B1B68F3
:106A9000DB0700F1AF85774BD86100F0ABBD734BDE
:106AA0001B685F0740F1A685724BD86100F0A2BD5C
:106AB0006E4B1B6813F0050F00F09C856D4BD86181
:106AC00000F098BD694B1B689E0740F19385694BA8
:106AD000D86100F08FBD654B1B689D0700F08A856B
:106AE000644BD86100F086BD604B1B68DC0640F14A
:106AF0008185604BD86100F07DBD5C4B1B689906B9
:106B000040F178855B4BD86100F074BD574B1B6832
:106B10005A0640F16F85574BD86100F06BBD534B5F
:106B20001B681B0640F16685524BD86100F062BDC0
:106B30004E4B1B68DF0540F15D854E4BD86100F080
:106B400059BD1A6A072A00F25585511C1962D96984
:106B500003EB82025162D86100F04CBD1B6A454ACA
:106B6000002B00F04785013B136202EB83035B6A55
:106B7000D36100F03FBD73782E2B04D83E4A01212B
:106B8000D15400F037BDFF2B7FF413AE394B0122F7
:106B900083F8442000F02EBD73782E2B04D8364A9B
:106BA0000021D15400F026BDFF2B7FF402AE314B03
:106BB000002283F8442000F01DBD2E4C94F845308F
:106BC00083B9461C4FF00A0304D1294A1068434395
:106BD000A36401E05843A06402F09AF90123E06441
:106BE00084F845306B78042B00F20485DFE803F06D
:106BF000034B7AAF190002F08BF9E26CA16C801A9A
:106C000080EAE072A2EBE0728A421A4B04D90022B9
:106C100083F8452000F0EEBCDA69013ADA6100F051
:106C2000E9BCA87804F02CFA40B9104B84F8450070
:106C30001A6822F010021A6000F0DCBCA36C0D4D43
:106C4000E3B102F065F9EB6CAA6CC01A80EAE0735C
:106C5000A3EBE073934211D9002385F84530034B31
:106C60001A6842F010021A6000F0C4BCD409002077
:106C70002C0A0020B80500205B0F0020E369013BCF
:106C8000E36100F0B7BC002004F065FBAB785B006B
:106C9000184110F0010609D0002384F84530AA4BB2
:106CA0001A6822F010021A6000F0A4BCA36CA74D71
:106CB0009BB102F02DF9EB6CAA6CC01A80EAE0736C
:106CC000A3EBE073934208D99F4B85F845601A689F
:106CD00042F010021A6000F08DBCE369013BE361F1
:106CE00000F088BC6A4600207C2104F039FBAA78B9
:106CF0000223520003FA02F29DF8023012EA03075F
:106D000009D0002384F845308F4B1A6822F0100216
:106D10001A6000F06FBCA16C8C4D99B102F0F8F8CC
:106D2000E96CAE6C401A80EAE071A1EBE071B1420F
:106D300008D9854B85F845701A6842F010021A6030
:106D400000F058BCE369013BE36100F053BC6A46C4
:106D500000207C2104F004FBAB789DF802205B004E
:106D600042FA03F313F0010609D0002384F84530FA
:106D7000754B1A6822F010021A6000F03BBCA26C3E
:106D8000724D9AB102F0C4F8EA6CA96C801A80EADC
:106D9000E072A2EBE0728A4208D96B4B85F845603D
:106DA0001A6842F010021A6000F024BCE369013B4B
:106DB000E36100F01FBCB278A2B9654A6549927ED2
:106DC00041F82300002A00F01584002B00F0128403
:106DD00003F28510800001EB8301042201F056FAD2
:106DE00000F008BCFF2A7FF49BA863B94FF4C3648A
:106DF0005949204621440422043401F047FAB4F5ED
:106E0000CD6FF5D1F6E3534903F28510800001EB15
:106E10008301042201F03AFAECE37378142B3FF675
:106E2000C8AC4E4A9278B2B94A4A52F823204C4B29
:106E30007A601B78002B00F0DD834A4B1A60424BCE
:106E400022B91A6842F008021A60D3E31A6822F0E5
:106E500008021A60CEE3FF2A7FF462A863B94FF4F8
:106E6000C3643D49204621440422043401F0A1FAC0
:106E7000B4F5CD6FF5D1BDE3364903F2851080003E
:106E800001EB8301042201F094FAB3E37678142E27
:106E90003FF68FACA878314F01061BD5C20706D547
:106EA0000020022104F05AFC2A4B43F82600284B0C
:106EB0009B7E002B00F09E836B78002B00F09A8362
:106EC000244903F28510800001EB8301042201F0C4
:106ED000DDF98FE300287FF423A8022104F03EFCB3
:106EE0001B4B1C4A9B7E42F82600002B00F082833D
:106EF0007B78002B00F07E83B97803F2851008447C
:106F0000194402EB81018000042201F0BFF971E312
:106F10007278144B0A2A54D8DFE802F0060B1128C5
:106F20002E363B40454A4E000F491A6809680A440C
:106F300003E00D491A680968521A1A6041E00A49CB
:106F40001A6809684A43F8E7D4090020B805002008
:106F500008000020D8090020C4030020CC0900202C
:106F60003B0A00202C0A0020480A00209E491A688B
:106F7000096892FBF1F2E0E79B4A1968126891FBFD
:106F8000F2F002FB1012D8E7974A11681A680A401B
:106F9000D3E7954A11681A680A43CEE7924A116806
:106FA0001A684A40C9E7904A1168C943116008E06D
:106FB0001A688D490A6004E08B4A186811681060ED
:106FC00019601A68894B22B91A6842F008021A60DF
:106FD00010E31A6822F008021A600BE3844B1B6866
:106FE000C6F80330FDF7B4FE04E3814B1B68C6F816
:106FF0000330FEF74FFCFDE27378052B00F2FA82B6
:10700000DFE803F003090F151B21784B1A6802F023
:107010000F021A60EEE2754B1A6822F010021A6035
:10702000E8E2724B1A6822F020021A60E2E26F4B2B
:107030001A6822F040021A60DCE26C4B1A6822F0F7
:1070400080021A60D6E2694B1A6822F480721A60D4
:10705000D0E273782E2B3FF6ACAB664A02EB83038B
:107060001865C7E2634B6249D3F80C210A60D3F874
:1070700010215D490A60D3F814215C49DA61D3F824
:1070800018210A60D3F81C215B4983F84520D3F806
:107090002021DA64D3F824219A6493F82821885CAB
:1070A00008B101208854002283F82C21A2E2B37891
:1070B000002B7EF435AF7378142B3FF67AAB4C4A35
:1070C00011684E4A42F8231094E202F0FDFA91E270
:1070D00002F0FCFA8EE202F00BFB8BE202F009FBFD
:1070E00088E202F007FB85E202F005FB82E273789A
:1070F00013B1012B04D00BE03E4B01221A7679E24A
:10710000B0F5006FBEF40CAF3A4A1376D06171E26D
:1071100003233B706EE2374B02221A766AE2354A4D
:107120004FF0FF3002F1500343F8210032480023B2
:10713000435401312F29F2D11376D361136282F8BF
:1071400045302B4A1360284A1360284A136051E2E5
:107150002B4B1B7D9B0709D4B0F5006FBEF4E0AE4E
:10716000244B04221A76C3F8300143E208233B7013
:1071700040E2244B01221A70214B234C9A78B0F53F
:10718000006F227025D21B7D13F0010521D16946C5
:1071900000F040FF9DF80030257263709DF80130CB
:1071A000A3709DF80230E3709DF8063023719DF8BE
:1071B000053063719DF80430A3719DF80330E371CD
:1071C0000123E15C227A01330A44082B2272F8D1B0
:1071D00010E201230021E1540133082B0A4AF9D1BE
:1071E0001378137206E200BF480A0020D409002079
:1071F0002C0A0020B80500205B0F0020D8090020D1
:1072000008000020300A0020310A00207378012B8A
:107210001DD00AD3022B2BD1A24B01221A70A24BF4
:10722000A24A9B781370002319E09E4B01221A702A
:107230009D4B9E4A9B7813709D4B18680023013329
:10724000C11811F8011C082BD154F8D1D2E1042245
:10725000FA717B7174222A23BA713B71CAE1954994
:107260000133194411F8091C082BD154F7D1C1E19D
:1072700003233B70BEE17378032B00F2BB81DFE890
:1072800003F0020E191D8C4B1A7EFA7193F84520FB
:10729000D3F83031BA711A0A7A713B71AAE1864B80
:1072A0001A7EFA7193F84520DB69BA711A0A7A716D
:1072B0003B719FE1814B1B687B609BE1804B1B68AE
:1072C0007B6097E17378002B40F094817D4B997837
:1072D000002940F08F8140F2D243984240F08A81E9
:1072E00040F2FF7000F073FF00F0D5FE0120FDF7C3
:1072F00020F97FE17278744B02B101221A70EA78AA
:10730000724B1A706C4B93F83411714B19707149B0
:1073100000230B7070490B70704B19780A431A7078
:1073200068E1654B012283F8352163E1757815B179
:10733000012D0FD01BE0042240F2FB70694601F0E2
:1073400038F8009BD6F803209A4206BF01237B60E1
:107350007D604FE1B3782A2B06D140F2FB70604983
:10736000042200F093FF45E103233B7042E1032335
:107370003B703FE17378032B3DD8DFE803F0080250
:107380002E394D4A0023D2F83811154610E04A4BE9
:10739000D3F83821092A07D8511CC3F8381103EB58
:1073A0008203C3F83C0125E109233B7022E101334C
:1073B0008B4200F01F814B4A9E0052F823408442CA
:1073C000F5D13244481E834204D25068013342F85A
:1073D000040BF7E7C5F838010CE1374A0023C2F87F
:1073E0003831404A002199500433282BF9D101E16A
:1073F0000A237B60FEE003233B70FBE07378812B64
:1074000040F0F880B2782F4B922A40F0F3809A79BE
:10741000A32A40F0EF805A79B42A40F0EB801A7921
:10742000C52A40F0E780DB78D62B40F0E3802E4B76
:107430004FF400421A6102F0E6F801F069FD0446DB
:1074400001F066FD001B0028B8BF4042B0F57A7F0E
:10745000F6DBFDF775F805F0FFFD002006F0D0FA29
:107460000021224805F0D1F9204805F033F92048E1
:1074700004F0A6FC05F00EFA4FF0804006F016FB73
:107480000020FDF756F8B5E040F2D243984240F0B4
:10749000B180094B012283F86421ABE00223237001
:1074A000A8E000BF300A002008000020310A0020B8
:1074B0000000002000400008B80500202C0A002031
:1074C000480A0020CC090020600E0020840E002015
:1074D000520F0020740E0020900F0020610E00203B
:1074E000CF090020F40600200010014008000240EF
:1074F00000240140B37843B1404A02EB43139B7F21
:10750000002B77D0927F9A4274D13D4B01221A70A2
:107510003C4B00241C703C4B2046214602221C7030
:1075200003F04DFF2046062140F2FF7203F071FE8A
:1075300020460821D5F8032003F06BFE5AE0334BB8
:107540009B7843B12D4A02EB43139B7F002B51D014
:10755000927F9A424ED12A4B01221A70294B002465
:107560001C70294B2046214602221C7003F027FF85
:107570002046062140F2FF7203F04BFED5F80320AF
:1075800020460821524203F044FE33E0002B31D064
:107590008B7F93422ED12046FEF7B4FB33782046F2
:1075A00023F001033370194B2146D3F8032003F075
:1075B00042FE20462146224603F001FF1AE0C8B1F0
:1075C000927F9A4216D1FEF79DFB0221304604F0CD
:1075D000C5F80E4B3146D3F803203B78024423F024
:1075E000010330463B7003F026FE304631463246FA
:1075F00003F0E5FE02B0BDE8F08100BFEC0E002014
:10760000B8050020E40E00206D0E0020CC090020FB
:107610003649002370B50B603549364A0B60364950
:10762000D36113620B6082F8453082F8443082F8EF
:107630002C311546314A4FF0FF3142F82310304AC1
:107640000024D45401332F2BF4D10621204604F01A
:1076500085F82C4B0C211860204604F07FF82A4B4B
:1076600018602A4B2046D97AC1F10801C9B202F04C
:107670007BFA274B0022E2500434B4F5806FF8D136
:10768000244EB37E13B9F37E6BB118E04FF4C3649C
:107690002149204621440422043400F08AFEB4F536
:1076A000CD6FF5D1EFE74FF4A7641C492046214484
:1076B0000422043400F07DFEB4F5C36FF5D13379B4
:1076C00003F0EF02012A01D0212B01D1012300E0B8
:1076D000002385F86531737D23B1FDF701FA08B108
:1076E000012300E000232B7670BD00BF2C0A002090
:1076F000480A0020B8050020D40900200806002010
:107700005B0F0020500E00204C0A0020EC0E0020E1
:10771000500A002008000020C403002018050020A3
:10772000F7B50F4E0F4CC6F803300F4B86460F4689
:10773000B270002294E803001A708DE8030086F806
:1077400000E07770FEF702FB21786368074A82F851
:1077500066119DE8030084E80300184603B0F0BDFD
:10776000CC090020400A00203B0A0020B805002078
:10777000014B93F866017047B8050020F7B51F4E1E
:10778000024653780C4696E803008DE803001C4936
:1077900000270B7093786D464B70D3788B701379FC
:1077A0008B7153794B7193790B71D379CB70154BE6
:1077B0001F70FEF7CBFA144B1978334671B921705C
:1077C00032786170A2707278E270F2792271B279C7
:1077D00062717279A2713279E27109E0012907D1EF
:1077E0003A460A4911444978A1540132082AF8D18D
:1077F00095E8030083E8030003B0F0BD400A0020D1
:10780000CC0900203B0A0020300A0020310A002069
:107810002DE9F047A34B8EB01B78A34C13B994F815
:10782000673163B1A14B1B78062B08D00A2B06D019
:1078300003F0EF030F2B1CBF002384F8343194F8BE
:107840003431994A591E0129994E41D89949012B41
:10785000CA6814BF082307238DF8183094F86831DC
:10786000079232788DF8193000238DF81A30C2B99A
:107870008B688DF827208DF820308F4B19788DF884
:10788000211059788DF82210D9798DF82310997923
:107890008DF8241059791B798DF825108DF8263034
:1078A0000AE0012A08D1854901330EAA595C1A441D
:1078B000082B02F8191CF6D1814B1B78002B40F0E5
:1078C000B88006A801F00CFA002800F08F83B0E021
:1078D000032B2AD192F865511DBB33788BB9754FB4
:1078E000754DB87897F801802A78804490446A787A
:1078F0009044EA799044AA7990446A7990442A792C
:1079000020E0012B40F095806C4B585D013500F074
:1079100001FF092DF8D18CE0072B6AD192F865316F
:1079200073B3654804F0CEF983E0042BF4D1614FC2
:10793000614DB87897F80180002301226B702A709E
:107940006B608044904400F0E5FE787800F0E2FE41
:10795000287800F0DFFE687800F0DCFEE87900F0BF
:10796000D9FEA87900F0D6FE687900F0D3FE5FFA60
:1079700088F8287900F0CEFE404600F0CBFE58E0B3
:1079800032782ABB4B4B93F802C093F801804A4BE4
:107990008DF800C01F785D78C444D8798DF80270E6
:1079A000674499798DF803503D445A798DF8040065
:1079B00028441B798DF8051001448DF806200A44EF
:1079C0008DF8073013448DF801808DF8083008E0F9
:1079D000012A06D1394A9A5C0DF803200133092B9C
:1079E000F8D1374B1B7823B36846092101F03EFEDE
:1079F0001FE0082B1DD1304A002301205370107066
:107A000053602C4A8DF80200917852788DF800105E
:107A10008DF801200A4402448DF803308DF80430BB
:107A20008DF805308DF806308DF807308DF8082078
:107A3000D7E7244B224F1A789946002A00F0978006
:107A4000214B224D1B78013B062B00F28C80DFE896
:107A500003F004043F8A8A8A6800164A29789368EA
:107A60008DF836108DF8303080238DF831308A2330
:107A70008DF8323000238DF833308DF834308DF8A6
:107A800035308DF829308DF82A30D36807210B93D3
:107A90003B788DF82810002B65D10AA801F020F959
:107AA00061E000BF3A0A0020B8050020CC090020A0
:107AB000300A002008000020400A0020310A00207F
:107AC000580E0020900F0020520F0020740E00204E
:107AD000DFF834832A7898F8020098F801A08244ED
:107AE0000AF10A0A924400F015FE98F8010000F02D
:107AF00011FE802000F00EFE8A2000F00BFE002018
:107B000000F008FE002000F005FE002000F002FE5C
:107B10005FFA8AFA287800F0FDFD504600F0FAFD81
:107B200021E0B94B2A789878597880238DF80E3067
:107B30008A238DF80D108DF80F30014400238DF845
:107B400010308DF811308DF812300A313B788DF8F5
:107B500013200A448DF80C008DF814201BB103A8E3
:107B6000092101F083FD00232B7089F800300023E8
:107B700084F83431337084F8673194F8643113B188
:107B80000120FCF7D6FC94F83521A04B52B193F8B4
:107B90006521D2F1010238BF002283F8652100225D
:107BA00083F835213B78002B44D106A801F0E2F898
:107BB00000283FD09DF81830062B3BD9944B9DF8F8
:107BC00020201A709DF821205A709DF822209A706A
:107BD0009DF823209A719DF824205A719DF8252044
:107BE0001A719DF82620DA709DF8193084F86831F2
:107BF000854B1A69079B934203D1844B012283F87A
:107C0000672101F085F9834B00221860824B1A70BE
:107C10009DF81830227E072B0CBF0123022384F825
:107C20003431531E012B7D4B02D9052A40F0CC8004
:107C30000022E7E094F86551002D70D103A800F010
:107C400083FD00286BD000F09DFD10B16F4B83F8D1
:107C5000695194F869119DF80C004A1CD2B2214474
:107C6000092A6A4B84F8692181F86A0140F0DE80B4
:107C7000002283F86921644A93F86A315178994265
:107C800007D092F82710002900F0D0808B4240F0F6
:107C9000CD8092F827209A4204BF012384F86731EF
:107CA00000231A46594D05F5B571595C01330A4454
:107CB000082BD2B2F6D195F8723193422BD1544BA6
:107CC00095F86B211A7095F86C215A7095F86D2112
:107CD0009A7095F86E219A7195F86F215A7195F8FE
:107CE00070211A7195F87121DA7001F011F94C4B7D
:107CF0004C4A1860297E00231370032285F8342132
:107D00004A1E012A85F86931444A02D9052918BF5B
:107D1000012313708AE0042385F8343186E094F857
:107D200065313A4D7BB13A4803F07FFE58B101F01E
:107D3000EFF83B4B3B4A186000231370032285F891
:107D400034212A7E39E094F86561002E43D13B78D6
:107D5000002B40D00AAD284601F072FC00283AD032
:107D600033463246E95C01330A44082BD2B2F9D1DA
:107D70009DF8301091422BD1254B9DF829201A7087
:107D80009DF82A205A709DF82B209A709DF82C207F
:107D90009A719DF82D205A719DF82E201A719DF828
:107DA0002F20DA7001F0B4F81D4B1E4A1860002332
:107DB0001370072284F83421227E511E01291946AE
:107DC000164B03D9052A01D001221BE019702DE0C2
:107DD00084F834312AE0237E0C4D013B012B25D859
:107DE000EB69B3F5006F1FD2FCF77AFEE0B1E869EA
:107DF0000749431CEB6100F00DF9092385F8343184
:107E0000064B01221A7011E008000020B80500207E
:107E1000CC090020440F0020590E00203B0A00200E
:107E20004C0F0020510F002000232376237E714D3C
:107E3000042B04D1704E3278170640F1AD8094F8CF
:107E4000343113F0FB0F05D0082B03D0062B01D0E3
:107E5000FDF77CFF94F83431092B79D101F058F803
:107E6000644A664DD2682B68801A80EAE072A2EB01
:107E7000E0729A4208D9624B1A78012A04BF0222A2
:107E80001A7001F045F8E06001F042F823696A6871
:107E9000C01A80EAE073A3EBE073934208D9584B11
:107EA0005A78012A04BF02225A7001F031F8206189
:107EB00001F02EF86369AA68C01A80EAE073A3EBA8
:107EC000E073934208D94E4B9A78012A04BF0222EC
:107ED0009A7001F01DF8606194F84430002B37D09F
:107EE000444B93F82C21002A32D145498B5C022B5C
:107EF0002BD1404B03F1500050F82200451C22D0FA
:107F0000404983F8282109680022C3F80C113E4932
:107F10000968C3F81011D969D861C3F814113B4935
:107F20000968C3F8181193F8451083F84520C3F881
:107F30001C11D96C0122C3F82011996C83F82C21F3
:107F4000C3F8241104E000238B5401322F2ACCD132
:107F500094F83411274B092904D11A7E022A04BF50
:107F600005221A76D4F83821224B002A3ED009295E
:107F70003CD1197E012939D1D86900231D4901F569
:107F80009E7454F82340A04202D105230B762DE0C5
:107F900001339342F2D129E095F8343113F0FB0F0D
:107FA00024D0082B22D0062B20D0D5F83001184C35
:107FB000D6F80330B0F5006F6270636012D23146BC
:107FC00000F03BF9D5F83001314600F0A8F830B1A7
:107FD000D5F830310133C5F83031652300E007238F
:107FE000237003E00723237000232B760EB0BDE837
:107FF000F08700BFB8050020CC090020140F002036
:108000005B0F00202C0A0020480A0020D409002021
:10801000400A0020C0EBC00038B500F50065002024
:108020000C4602460321FCF71BFE0020C5F3072186
:108030000246FCF715FE0020E9B20246FCF710FEEE
:10804000002001460246FCF70BFE2070002001468E
:108050000246FCF705FE6070002001460246FCF770
:10806000FFFDA070002001460246FCF7F9FDE0701C
:10807000002001460246FCF7F3FD20710020014676
:108080000246FCF7EDFD6071002001460122FCF77D
:10809000E7FDA07138BD38B54FF40064002006211B
:1080A0000122FCF7DDFD002005210246FCF7D8FD8A
:1080B000002001460122FCF7D3FD8307F3D5002001
:1080C00002210246FCF7CCFD0020C4F30721024642
:1080D000FCF7C6FD0020E1B20246FCF7C1FD002519
:1080E000B5F13F0EDEF100024FF0000052EB0E0240
:1080F00001460135FCF7B4FD402DF1D100200521EA
:108100000246FCF7ADFD002001460122FCF7A8FD68
:10811000C307F3D44034B4F5804FBFD138BDF7B5B1
:10812000C0EBC00000F5006500200C4602460321AC
:10813000FCF796FD0020C5F307210246FCF790FDF1
:108140000020E9B20246FCF78BFD00200146024602
:10815000FCF786FD0746002001460246FCF780FD3D
:108160000646002001460246FCF77AFD054600203F
:1081700001460246FCF774FD8DF80300002001461D
:108180000246FCF76DFD8DF8040000200146024612
:10819000FCF766FD8DF80500002001460122FCF782
:1081A0005FFD23788DF80600BB420DD16378B342A2
:1081B0000AD1A378AB4207D1DDF80300D4F803302D
:1081C000C31A5842584100E0002003B0F0BD38B552
:1081D000012204460D4600200621FCF741FD002047
:1081E00005210246FCF73CFD002001220146FCF778
:1081F00037FD8207F3D5002002210246FCF730FD4F
:108200000020C4F307210246FCF72AFD0020E1B25A
:108210000246FCF725FD002029460122FCF720FD3F
:10822000002005210246FCF71BFD0020014601222B
:10823000FCF716FDC307F3D438BD38B5C0EBC00555
:108240000C4605F500600978FFF7C1FF05F601004F
:108250006178FFF7BCFF05F60200A178FFF7B7FFD2
:1082600005F60300E178FFF7B2FF05F60400217977
:10827000FFF7ADFF05F605006179FFF7A8FF05F6EA
:108280000600A179BDE83840FFF7A1BF2DE9F04114
:1082900004460F461646002006210122FCF7E0FCAA
:1082A000002005210246FCF7DBFC002001460122EC
:1082B000FCF7D6FC8507F3D5002002210246FCF727
:1082C000CFFC0020C4F307210246FCF7C9FC0020C4
:1082D000E1B20246FCF7C4FC0025B54242D00134AD
:1082E00014F03F08795D04D0721EA81A4242424140
:1082F00000E001220020FCF7B3FCB8F1000F2FD101
:10830000731E9D422CD2002005210246FCF7A8FCDA
:10831000002001460122FCF7A3FC10F00100F2D17D
:1083200006210122FCF79CFC002005210246FCF7F7
:1083300097FC002001220146FCF792FC8207F3D54E
:10834000002002210246FCF78BFC0020C4F3072129
:108350000246FCF785FC0020E1B20246FCF780FCF7
:108360000135BAE7002005210246FCF779FC002020
:1083700001460122FCF774FCC307F3D4BDE8F08189
:1083800010B50446002003210246FCF769FC0020DA
:10839000C4F307210246FCF763FC0020E1B2024669
:1083A000FCF75EFCBDE81040002001460122FCF70E
:1083B00057BC70B5044600200E4615460321024600
:1083C000FCF74EFC0020C4F307210246FCF748FCF2
:1083D0000020E1B20246FCF743FC0024AC420AD084
:1083E0006A1EA31A00205A4201465A41FCF738FC83
:1083F00030550134F2E770BD37B500200521024643
:10840000FCF72EFC002001460122FCF729FC10F0AD
:108410007104F2D100F07CFD054600F079FD401BAF
:108420000028B8BF4042B0F5FA6F09DA4CB940F203
:10843000FF70FFF7A5FFB0F142035C425C41ECE73F
:1084400014B1224B1B78ABB340F2FF700021FFF751
:10845000BEFEFFF720FE00201D494022FFF716FF59
:108460004FF480701B49B422FFF710FF40201A49D7
:108470002022FFF70BFF002301934FF4C364204633
:1084800001A904220434FFF701FFB4F5FF6FF6D110
:10849000002301934FF4A764204601A90422043469
:1084A000FFF7F4FEB4F5C36FF6D140F2FF7042213E
:1084B000FFF78DFE002006494022FFF77AFF40209B
:1084C00006492022FFF775FF03B030BD8C0E002057
:1084D0000800002004180108E4170108EC0E002031
:1084E00030B5054687B0554805F0CCFF4FF4003055
:1084F000012105F065F80420012105F055F804205C
:10850000002105F069F80820002104F065FD03232F
:108510008DF8063018230DEB03048DF80730042383
:1085200024F8143D4648214604F0C7FC48238DF842
:108530000730434808232146ADF8043004F0BDFC61
:1085400002A806F02DF80B2D25D8DFE805F024064B
:10855000090C0F1215181B1E20224FF461531CE04A
:108560004FF4964319E04FF4E14316E04FF41643FD
:1085700013E04FF4614310E04FF496330DE04FF4F5
:10858000E1330AE04FF4613307E02E4B05E02E4B58
:1085900003E02E4B01E04FF416530293029B02A915
:1085A0005B082648029305F0B7FF26230024012527
:1085B0008DF80030684607238DF801308DF80240B1
:1085C0008DF8035004F084FD1C4840F2FF3106F0A2
:1085D000CFF822461948282106F00FF82A461748F6
:1085E00040F2277106F009F82A46144840F2266145
:1085F00006F003F82A46114840F2255105F0FDFF28
:1086000022460E4840F2244105F0F7FF22460B486F
:1086100040F6460105F0F1FF2246084840F66A118F
:1086200005F0EBFF22460548602105F0E6FF034810
:10863000294605F0D6FF07B030BD00BF004400401A
:108640000008014090D0030020A1070040420F0025
:10865000684620F007018D46294919B50B889C060C
:108660001AD5284BDB68980701D58B8814E0264B78
:108670001A6858680132202A08BF0022824205D0B9
:108680001C6888881919C0B208721A601F4A0A212A
:1086900011609A6A1E4B1A60194803881A061BD586
:1086A0001B4B1A68C2B9184BDC6A196B8C420FD08D
:1086B000144902240C61196B4C1C1C63194491F879
:1086C0003410C9B28180196B202905D11A6303E0E7
:1086D00040F2277105F091FF094803885B060BD52E
:1086E00040F2266106F068F8074B1A6BDB6A9A4283
:1086F00002D1044B02225A61BDE8194085467047F9
:1087000000440040000801402C070020980F002082
:10871000940F00200A4BDA6A196B0132202A08BF35
:1087200000228A420AD0D96A194481F83400DA62F8
:10873000044840F22771012205F05FBF704700BF77
:108740002C070020004400400A4B59681A689142E7
:108750000BD05A68511C59601A44127A02705A6838
:10876000202A04D100225A6001E000207047012035
:10877000704700BF2C070020014B9862704700BF74
:108780002C070020044B1A7802F0FF0012B10022DF
:108790001A700120704700BF9C0F002008B5FBF73E
:1087A000CFFE044B00225A601A60BDE80840FBF778
:1087B000C5BE00BF2C07002010B5441E14F8010FE1
:1087C00010B1FFF7A7FFF9E710BD00BF684620F022
:1087D00007018D4631B5264C264B25681B680135AF
:1087E000082D08BF00259D4286B04FF0000037D00D
:1087F00001A903F051FE9DF80C302268042B1E4B9A
:1088000003EB021206D1012151702168029A03EB99
:10881000011105E0002151702168019A03EB01115B
:108820004A609DF80D20022A226808BF012103EB4F
:10883000021218BF0021917022689DF80E101201DB
:1088400099540022216801A8104403EB011111443E
:10885000C07A0132082A0872F4D1054B1D6001E08C
:1088600003F000FE06B0BDE831408546704700BF0A
:108870002C100020A00F0020AC0F0020684620F034
:1088800007018D4631B5264C264B25681B680135FE
:10889000082D08BF00259D4286B04FF0010037D05B
:1088A00001A903F0F9FD9DF80C302268042B1E4B42
:1088B00003EB021206D1012151702168029A03EBE9
:1088C000011105E0002151702168019A03EB0111AB
:1088D0004A609DF80D20022A226808BF012103EB9F
:1088E000021218BF0021917022689DF80E1012012B
:1088F00099540022216801A8104403EB011111448E
:10890000C07A0132082A0872F4D1054B1D6001E0DB
:1089100003F0A8FD06B0BDE831408546704700BFB2
:108920002C100020A00F0020AC0F0020684620F083
:1089300007018D4631B52A4B2A4A1968126886B05C
:10894000914204D10120002103F0C6FC43E01A68E3
:10895000254901EB0212507800F0FF0248B10422D1
:108960008DF80C20002201921A6801EB0212526865
:1089700006E018688DF80C2001EB001040680190AB
:1089800002921A6801EB0212927802F0FF001AB10B
:1089900002228DF80D2001E08DF80D001A681201F9
:1089A0008A5C8DF80E2000221C680D4801EB04142F
:1089B0001444257A01AC14440132082AE572F3D13B
:1089C0000368013303600368082B04BF00230360BE
:1089D00001A803F08DFC06B0BDE831408546704724
:1089E000A80F0020A40F002030100020F0B501389F
:1089F0008BB00F4615460C23072813D8DFE800F08C
:108A0000100E0C0A0812060402220CE004220AE0EE
:108A1000102208E0142206E0282204E0642202E08A
:108A2000C82200E008228DF8143003238DF8153099
:108A30000023ADF816208DF8133003F05FFB4FF0E4
:108A40000070012104F0BCFD0120014604F0ACFDE2
:108A50000820012104F0A8FD0820002104F0BCFD3D
:108A60004FF4EA10012104F0B7FA03238DF8063021
:108A700018230AAC8DF807304FF4007324F8243D16
:108A80002146784804F019FA042321468DF807306E
:108A900074484FF4807300240126ADF8043004F0CC
:108AA0000CFA03A88DF812408DF80C408DF80D607B
:108AB0008DF80E408DF80F408DF810608DF8116024
:108AC00003F029FBB7F5006F8DF818408DF81940B9
:108AD0008DF81A600FDA7B01ADF81C304FF6FF738A
:108AE000ADF81E40ADF82030ADF82230ADF824408E
:108AF0008DF826600DE04FF6FF73ADF81C40ADF821
:108B00001E40ADF82030ADF82230ADF824408DF88D
:108B1000264006A803F05EFB012300228DF81830E2
:108B20008DF819208DF81A3095B1B5F5006F0FDA70
:108B30006901ADF81E204FF6FF72ADF81C10ADF8BC
:108B40002020ADF82220ADF824308DF826300DE03D
:108B50004FF6FF71ADF81C20ADF81E20ADF82010C7
:108B6000ADF82210ADF824308DF8262006A803F0C9
:108B700031FB02238DF818307B13FF0047F0040708
:108B800000260124ADF81E7006A84FF6FF77ADF859
:108B90001C308DF819608DF81A40ADF82070ADF8D2
:108BA0002270ADF824608DF8264003F013FB0323F8
:108BB000B5428DF818308DF819608DF81A4010DD27
:108BC0006B13ED0045F00405ADF81C30ADF81E50F8
:108BD000ADF82070ADF82270ADF824408DF8264035
:108BE0000CE00423ADF81C60ADF81E30ADF8207029
:108BF000ADF82270ADF824408DF8266006A803F089
:108C0000E9FA012407260025142302A88DF808306C
:108C10008DF809608DF80A508DF80B4004F058FA71
:108C2000152302A88DF808308DF809608DF80A50D8
:108C30008DF80B4004F04CFA132302A88DF808308D
:108C40008DF809608DF80A508DF80B4004F040FA59
:108C50002146022003F040FB1020214603F03CFB9C
:108C60000BB0F0BD000C014037B50220002103F02D
:108C700033FB1020002103F02FFB0021012003F023
:108C80002BFB00240725142301A88DF804308DF850
:108C900005508DF806408DF8074004F019FA1523A9
:108CA00001A88DF804308DF805508DF806408DF838
:108CB000074004F00DFA132301A88DF804308DF855
:108CC00005508DF806408DF8074004F001FA03F0D6
:108CD00015FA4FF00070214604F072FC03B030BD6D
:108CE000F0B5437887B00446426833B104238DF869
:108CF0000C3000230292019303E08DF80C300192B6
:108D00000293A37803B102238DF80D3023788DF8F8
:108D10000E300023E11801AA1A44097A0133082B06
:108D2000D172F7D101A803F0E3FA042816D10E4F4F
:108D30000E4B3D681B680135082D08BF00259D427C
:108D40000ED03E680A4B03EB061694E80F0086E847
:108D50000F00012001463D6003F0BEFA012000E053
:108D6000002007B0F0BD00BFA40F0020A80F002016
:108D70003010002030B50D4B0D4C054622681B68A5
:108D80009A420ED023685A1C22600A4A02EB03134F
:108D90000FCB85E80F002368082B04D10023236044
:108DA00001E0002030BD012030BD00BF2C100020AC
:108DB000A00F0020AC0F0020684620F007018D4670
:108DC00001B5BDE801408546704700BF684620F008
:108DD00007018D46F1B5384B19781A4679B15B68B1
:108DE00001335360354B196801311960344B1968F0
:108DF00011B11968013919600023137001E00122D3
:108E00001A70304B1A683AB11A68013A1A601B6836
:108E100013B92D4B01221A702C4B2D489B8C2D49D8
:108E20009BB2036002680B689A4202680B6817DD08
:108E3000D31A294CB3F5004F284DD4E9002306DAA4
:108E4000D0F800C00F682E68C7EB0C0527E0D1F8FA
:108E500000C007682E68C7EB0C0505F5803511E0EA
:108E60009A4222DA0A6803681B4CD31AB3F5004F02
:108E70001A4DD4E900230ADAD1F800C007682E6839
:108E8000C7EB0C057543521B63EBE5730BE0D0F8A1
:108E900000C00F682E68C7EB0C0505F580357543DB
:108EA000521943EBE573C4E900230368BDE8F140C0
:108EB0000B608546704700BF800700203C0A0020F9
:108EC000940F0020980F00209C0F00200008004005
:108ED0008C0F0020700E0020900E0020980E0020B5
:108EE00008B5042004F066FD48F6A04004F06EFDCD
:108EF000012004F071FD05480321002204F0BEF9B1
:108F0000BDE80840012004F07BBD00BF9AC3020009
:108F1000014B5868704700BF800700200000000028
:108F200070B592B0012400250326414801A9ADF88F
:108F300004408DF806608DF8075003F0BEFF112342
:108F40003C4801A9ADF804308DF806608DF8075053
:108F500003F0B3FF2046214604F01AFB21464FF4EC
:108F6000007004F021FB344803F0B4FB334B32486B
:108F70000793334B07A9089380230C934FF4807316
:108F80000D934FF480630E9320230F934FF40053FF
:108F9000109309950A960B95119503F00BFC264842
:108FA000214603F032FC4FF46023264802A90493C3
:108FB00002958DF80C408DF80D4005958DF81860E0
:108FC00002F02AFF1F4808212246334602F09CFF88
:108FD0001C4804210222334602F096FF334619480A
:108FE0002946324602F090FF2A4616484FF4FC61AB
:108FF00002F051FF1348214602F044FF1148214678
:1090000002F037FF0F4802F04FFF0E4802F051FF09
:109010000028FAD10B4802F050FF0A4802F052FF34
:109020000028FAD10748012102F050FF12B070BDAC
:10903000000C014000080140080002404C2401409F
:1090400088070020002401400828F8B507D0092827
:109050000DD0002858D13A4B188880B2F8BD384B53
:10906000588840F2132380B258430013F8BD344BA4
:10907000988880B207F042FA06F024FE0022314BB5
:1090800006F074FE22A3D3E9002306F06FFE044627
:109090000D4622462B461EA1D1E9000106F0B2FC86
:1090A0001DA3D3E9002306460F462046294606F0B5
:1090B00087FF02460B463046394606F081FF07F02F
:1090C00017F906F0FFFD00221F4B06F079FF08F0AC
:1090D000E7F813A3D3E9002306F048FE12A3D3E96F
:1090E000002306F091FC02460B4611A1D1E90001D4
:1090F00006F066FF10A3D3E9002306F083FC07F017
:10910000F7F807F019FCF8BD0020F8BDAFF30080B8
:109110006666666666660A409A99999999990140C9
:10912000C3F5285C8FA272400000000000FEAA4038
:109130009A999999FD6F2F41C3F5285C8F12714060
:10914000880700200000303F00002440AFF300807B
:10915000014B00221A60704790070020034B9B7A56
:1091600013B1034B05225A60704700BFBC100020AA
:1091700090070020014B04225A607047900700209E
:10918000034B1A7A202A04BF00221A72704700BFCC
:10919000900700207047212810B508D1104B1B689C
:1091A0001B7803F07F03212B10D0022010BD202854
:1091B000FBD10B4B0B4A1B681B78107203F07F032B
:1091C000212B094B18BF00230BB9EEE7074B044ACC
:1091D000002412682046936154829847204610BDAF
:1091E0001C110020900700203D92000825920008E5
:1091F000074B1B681B7803F07F03212B06D100F07F
:10920000DF0002280CBF00200220704702207047B8
:109210001C11002021B9022834BF00200220704711
:109220000220704720B9034B08221B681A8270473E
:10923000014870471C1100204800002020B9034B52
:1092400008221B681A827047014870471C110020D1
:109250004800002008B5032006F050FA064B0246ED
:10926000D8604FF48871054805F0FAFFBDE8084062
:10927000032006F0C2B800BF900700202211002092
:1092800038B5334B00241B68C0259C725D72DC72BC
:10929000204606F021F820464FF4007106F039F818
:1092A0002046102106F04CF82046402106F0A8F98F
:1092B0008021204606F093F9204606F0CAF8254B97
:1092C000204693F8341006F0E8F9204606F095F8A9
:1092D0000120214606F01DF80120294606F07FF9FD
:1092E0000120202106F02CF80120214606F03DF84F
:1092F00002204FF4C06106F00CF802204FF4807198
:1093000006F06DF90220214606F02FF802202021F8
:1093100006F016F80320214605F0FBFF03204FF46A
:10932000887106F06DF90320402106F0B6F903209C
:109330004FF4405106F019F80320214606F000F8DA
:10934000204605F02BFE044B01225A6038BD00BFB9
:109350001C1100204800002090070020014905F062
:1093600017BC00BF80000020014905F011BC00BF00
:1093700088000020054B1B68DB78042B04D80449C7
:1093800001EBC30105F004BC002070471C11002054
:109390009000002008B5002004F084F8BDE80840E3
:1093A0004FF40000012104F00BB9024B03225A6074
:1093B000704700BF90070020044B9A7A044B0AB113
:1093C000052200E001225A60704700BFBC10002057
:1093D0009007002007B514238DF8043000238DF882
:1093E00005308DF8063001A801238DF8073003F011
:1093F0006FFE03B05DF804FB00B10120FBF7E2B89B
:109400007047684620F007018D4679B5154D164B1B
:109410002A681C4692B21A80144A18881188164687
:10942000014011F4806F05D04FF6FF332B60104BD5
:10943000DB689847238832881340990507D54FF693
:10944000FF532B600B4B197C0131C9B2197423886F
:109450001A40130401D505F009FEBDE879408546A0
:10946000704700BF445C0040B21000206211002031
:10947000480000209007002008B50120FBF7A2F863
:10948000064B01221A60064A002006491860106047
:109490004FF4E0520A801A6008BD00BF405C0040F3
:1094A000445C004062110020084B10B51B6800248A
:1094B0009C72FFF7E1FF064B064A1C604FF406431F
:1094C0001380054A1360054B5C6010BD1C11002021
:1094D000445C004062110020405C00409007002086
:1094E00038B5064D01232B60054B00241C60204637
:1094F000FBF768F803232B60204638BD405C004032
:10950000445C0040074B1A6892B242F008021A60AD
:109510001A6892B242F004021A60034B03225A60A6
:10952000704700BF405C00409007002010B5064C1B
:109530004FF6FB73226813402360FFF73DFF4FF4A3
:109540000643236010BD00BF405C004010B51E4CB8
:10955000072818BF20702378052B32D8DFE803F0E6
:1095600003060A0E1621FFF7E1FF2AE0FFF7DEFFF0
:10957000042327E002236370032323E06378013B85
:10958000DBB263706378F3B9042217E00F4B1A68FB
:1095900092B242F010021A60052323700A2363700E
:1095A00010BD6378013BDBB2637063785BB9074A37
:1095B0004FF6EF7311680B4013600622024B1A70CE
:1095C00010BD0623237010BD20110020405C004018
:1095D00008B5FFF7DFFEFFF7FDFEBDE8084005F028
:1095E00029BD07B514238DF8043000238DF805300C
:1095F0008DF8063001A801238DF8073003F068FDCF
:1096000003B05DF804FBFFF76BBF0B4910B5CA68E8
:1096100082B14B68052B0CD10023CC68A34204D245
:10962000064C1C5DC4540133F7E7034B0021D9609D
:1096300000E00022104610BD9007002022110020FB
:10964000084BDA68082A1A460AD900230649595CE9
:10965000C1540133092BF9D10023D3600120704795
:1096600000207047900700202211002010B5084C00
:109670000A46216092B2C02105F0DAFD012021885E
:1096800005F0EAFFBDE81040012005F0A7BE00BFCD
:1096900090070020704710B5FFF73AFC074C23688D
:1096A000C01AB0F5FA7F07D9054BDA6882F00402D8
:1096B000DA60FFF72DFC206010BD00BF64110020B0
:1096C000000C01407047704770477047054B064AD1
:1096D000D3F80310054B09B9928800E0128992B2C1
:1096E0005A607047CC090020006C0040400A0020FE
:1096F00070477047704710B5FBF73CF805280E4CD3
:1097000001D8012306E0FBF735F840F2F93398421F
:10971000F7D800236360094B1B7863B1084B62687C
:109720001A60084B1AB91A6842F0080202E01A6877
:1097300022F008021A6010BD400A00203B0A0020F7
:109740002C0A0020D409002070B50546C5F3074156
:1097500000220120FBF784FA0A4C0602C5F3072118
:10976000002201202660FBF77BFA3043060201202D
:10977000E9B202462660FBF773FA30430609266019
:1097800070BD00BFA407002038B5484C0B2303FB75
:10979000004203FB004311790433032984BF0321F2
:1097A00011719A78032A84BF03229A700B2303FB5A
:1097B000004203FB0043117A04320F2984BF0F21BA
:1097C00011715A7A0433072A84BF07225A710B2376
:1097D00003FB004203FB0043917A04320F2984BF4C
:1097E0000F2191715A7B0C330F2A84BF0F225A70BC
:1097F0000B2202FB004302FB0042997B0C330F2932
:1098000084BF0F21997013795279DB0343F400214F
:1098100021611AB1254943F404230B610B2101FB9B
:109820000041C979214B19B1196941F400511961FD
:109830000B2372B903FB0043197A9A79C90141EAF3
:10984000C221043322695B790A4342EA031222618E
:109850001AE003FB00431B7B144A1BB1136943F45A
:10986000805313610B2202FB0042917B557B2269DE
:109870000E4B42EAC51201F0070542EA051209073C
:1098800048BF42F400621A610B2202FB0040C27A18
:10989000064B04301AB91A6981790A431A612069A2
:1098A000FFF752FF2369636138BD00BFA4070020A2
:1098B00010B5114C0023C000236123185B7F13B146
:1098C0004FF4007323612218927F0B4B1AB11A696F
:1098D00042F480721A612318DA7F20440F2A84BF71
:1098E0000F22DA77C07F236918432061FFF72CFF2E
:1098F0002369236210BD00BFA407002010B5224CCD
:109900004FF46023C0002361231893F82B3013B168
:109910004FF470232361231893F8252093F8241023
:10992000120342EA813293F826302169012B42EA80
:109930000102226103D1144B42F480621A612218A1
:1099400092F82710236992F8282043EA0123012A7C
:10995000236103D10C4A43F080031361221892F86B
:109960002920094B012A03D11A6942F040021A61E9
:109970002044236990F82A0043EA00102061FFF791
:10998000E3FE2369E36210BDA407002038B52A4C2A
:1099900043001A18224492F9311030323F29C4BFD3
:1099A0003F2151701A18224492F9311030323F3160
:1099B000BCBFC12151701A18224492F832103032C3
:1099C0001F2984BF1F2191704FF4402222611A1871
:1099D000224492F83020012A03D1174A4FF4502133
:1099E000116104EBC00191F82B10134A51B91918F9
:1099F000114491F83150116905F07F0541EA0521C4
:109A000011610CE01D18154495F8315001F0030167
:109A100005F07C052943156945EA012515610344D4
:109A2000234493F83200236918432061FFF78CFE2A
:109A30002369636338BD00BFA407002010B583000D
:109A4000244C1A18224492F83810012984BF0121AD
:109A500082F838101A18224492F839103832032943
:109A600084BF032151701A18224492F83A103832F8
:109A70000F2984BF0F2191701A18224492F83B10CD
:109A80003832032984BF0321D1701A18224492F876
:109A90003C1003440F2902F1380284BF0F211171D9
:109AA000234493F83C0003F1380293F8383040F433
:109AB000202040EAC330537840EA4330937840EAAC
:109AC0000320D37840EA43102061FFF73DFE23696D
:109AD000236410BDA4070020224B012010B50322EF
:109AE0000024052183F8300083F82900022083F840
:109AF000264083F8274083F8284083F82A0083F81B
:109B00002B4083F8384083F8394083F83A4083F893
:109B10003B4083F83C405C779C77DC7718715C7144
:109B2000DC719C711872DC721C735C7383F83110E9
:109B300083F8321083F8242083F825205A72997212
:109B40009A732046FFF77AFF2046FFF71FFF204653
:109B5000FFF7D4FE2046FFF7ABFE2046BDE81040DD
:109B6000FFF712BEA4070020054B042903EBC00336
:109B700018BF0022D97718BF5A77FFF799BE00BFE8
:109B8000A4070020044B03EBC003597709B104225A
:109B9000DA77FFF78DBE00BFA4070020024B03EB6E
:109BA000C0039977FFF784BEA4070020024B03EBA4
:109BB000C000C07F704700BFA4070020024B03EB2A
:109BC000C000407F704700BFA4070020024B03EB9A
:109BD000C000807F704700BFA4070020034B0B220A
:109BE00002FB00331971FFF7CFBD00BFA4070020AF
:109BF000034B0B2202FB00335971FFF7C5BD00BFB9
:109C0000A4070020034B0B2202FB0033D971FFF79E
:109C1000BBBD00BFA4070020034B0B2202FB003397
:109C20009971FFF7B1BD00BFA4070020034B0B22C1
:109C300002FB00331972FFF7A7BD00BFA407002085
:109C4000034B0B2202FB00335972FFF79DBD00BF8F
:109C5000A4070020034B0B2202FB00339972FFF78D
:109C600093BD00BFA4070020034B0B2202FB00336F
:109C70001973FFF789BD00BFA4070020034B0B2217
:109C800002FB00335973FFF77FBD00BFA40700201C
:109C9000034B0B2202FB00339973FFF775BD00BF26
:109CA000A4070020024B0B2202FB00300079704712
:109CB000A4070020024B0B2202FB003040797047C2
:109CC000A4070020024B0B2202FB0030C079704732
:109CD000A4070020024B0B2202FB00308079704762
:109CE000A4070020024B0B2202FB0030007A7047D1
:109CF000A4070020024B0B2202FB0030407A704781
:109D0000A4070020024B0B2202FB0030807A704730
:109D1000A4070020024B0B2202FB0030007B70479F
:109D2000A4070020024B0B2202FB0030407B70474F
:109D3000A4070020024B0B2202FB0030807B7047FF
:109D4000A4070020034A00EB8003134483F8381073
:109D5000FFF774BEA4070020034B00EB80021344FE
:109D60005970FFF76BBE00BFDC070020034B00EB10
:109D7000800213449970FFF761BE00BFDC0700202A
:109D8000034B00EB80021344D970FFF757BE00BFAE
:109D9000DC070020034B00EB800213441971FFF72E
:109DA0004DBE00BFDC070020034B00EB80001844D1
:109DB00090F83800704700BFA4070020024B00EB6A
:109DC0008000184440787047DC070020024B00EB0D
:109DD0008000184480787047DC070020024B00EBBD
:109DE00080001844C0787047DC070020024B00EB6D
:109DF0008000184400797047DC070020034A00EB1C
:109E00004003134483F83010FFF7C0BDA4070020BF
:109E1000034B00EB400213445970FFF7B7BD00BF7E
:109E2000D4070020034B00EB400213449970FFF766
:109E3000ADBD00BFD4070020034B00EB4000184429
:109E400090F83000704700BFA4070020034B00EBE0
:109E50004000184490F90100704700BFD40700206B
:109E6000024B00EB4000184480787047D407002074
:109E7000034B03EBC00383F82410FFF73FBD00BF83
:109E8000A4070020034B03EBC00383F82510FFF762
:109E900035BD00BFA4070020034B03EBC00383F8CC
:109EA0002610FFF72BBD00BFA4070020034B03EBD8
:109EB000C00383F82710FFF721BD00BFA4070020CF
:109EC000034B03EBC00383F82810FFF717BD00BF57
:109ED000A4070020034B03EBC00383F82910FFF70E
:109EE0000DBD00BFA4070020034B03EBC00383F8A4
:109EF0002A10FFF703BD00BFA407002010B5064BD2
:109F0000044603EBC00383F82B10FFF7F7FC204651
:109F1000BDE81040FFF73ABDA4070020024B03EB59
:109F2000C00090F824007047A4070020024B03EB08
:109F3000C00090F825007047A4070020024B03EBF7
:109F4000C00090F826007047A4070020024B03EBE6
:109F5000C00090F827007047A4070020024B03EBD5
:109F6000C00090F828007047A4070020024B03EBC4
:109F7000C00090F829007047A4070020024B03EBB3
:109F8000C00090F82A007047A4070020024B03EBA2
:109F9000C00090F82B007047A40700202DE9F0477F
:109FA0002E4D1E462B1893F8443004468A4691469F
:109FB000DDF82080099F042B1AD8DFE803F003089E
:109FC0000D121700FFF7E0FB2B19012212E0FFF73B
:109FD00095FC2B1902220DE0FFF730FD2B1903220F
:109FE00008E0FFF7D3FC2B19042203E0FFF760FC25
:109FF0002B19002205EBC40483F8442094F82A208E
:10A00000164B012A13D002D3022A15D021E0BAF14F
:10A01000000F03D01B689B0C8AF80030B9F1000FC9
:10A0200017D02B68C3F38923A9F8003011E086B15B
:10A030001B689B0A33600CE01EB11B68DB0B5B01E5
:10A040003360B8F1000F04D02B68C3F3842388F881
:10A0500000300FB12B683B70BDE8F087A4070020EB
:10A0600030B9044BDA7A1AB90122DA72FFF78CBBE5
:10A07000704700BFA407002028B9034BD97A11B15B
:10A08000D872FFF781BB7047A40700202DE9F0418B
:10A09000114AC700D31993F82A600546032E90464B
:10A0A00004D0032283F82A20FFF728FC2846FFF774
:10A0B00025FCD8F80040230344BF6FEA04346FEA5C
:10A0C0001434032E05D0474487F82A602846FFF74A
:10A0D00015FC2046BDE8F081A407002070B5084CAF
:10A0E0009DF810609DF8145004EBC0042176627650
:10A0F000A376E6762577BDE87040FFF7D9BB00BFB1
:10A10000A407002006281AD8DFE800F004070A0D8B
:10A11000101316000A4B1B6810E0094B1B6A0DE078
:10A12000074B5B690AE0064B1B6C07E0044B5B6B5B
:10A1300004E0034BDB6A01E0014BDB7A0B60704704
:10A14000A4070020014B1878704700BFEC070020DF
:10A15000034B00201870034B997AFAF7E5B900BF5A
:10A16000530F0020EC0E00202DE9F04F8D4C87B0EE
:10A17000637823B96FF00043636001236370257A2D
:10A18000894F4DB9E8B2FAF77CF978550135082DB9
:10A19000F8D1844B01221A7227250026F0B2FAF773
:10A1A00070F9BB5D83421AD07F4B321DF0547F4B58
:10A1B00053F82230022B05D0032B0AD0012B0ED1ED
:10A1C00068B106E058B97A4A515D012907D1535563
:10A1D00005E0774B5A5D012A04BF02225A55013629
:10A1E000082E05F10105D9D1724EF36993B1724D74
:10A1F0002F787FB9FEF78CFE704B1B68C01AF3698D
:10A200000028B8BF4042984204D9384601F0F2F91C
:10A2100001232B70336AA3B1694D2E788EB9FEF7F6
:10A2200077FE684B634A1B68126AC01A80EAE073C3
:10A23000A3EBE073934204D9304601F0DBF901232C
:10A240002B70607C604D574E05EB40131F7B002F39
:10A2500000F0FC805D4B5E4F03440093C3190193F3
:10A260005C4B002103EB80030A46FFF797FE707CEE
:10A270004301EA18127B013A042A00F2D580DFE894
:10A2800002F0033AAF3AAF00534A544E926812F4C8
:10A29000004F04EB0002927C10D0022A03D1325C02
:10A2A000002A00F0C1801D44697AFAF73DF9607C0C
:10A2B000FFF7E2FE637C0221E21818E0012A03D1D5
:10A2C000325C002A00F0B0802B44997AFAF72CF91E
:10A2D000607C05EB4015AB7A13B9FFF7C1FE03E0D4
:10A2E000335C0BB1FFF7C8FE637C0121E218917467
:10A2F0000022F25498E03A56384E002A19DB221810
:10A30000927C022A01D1325C62B12B44597AFAF76D
:10A310000BF9607CFFF7B0FE637C0221E2189174B8
:10A320000022F254667CFEF7F3FD04EB86067060B3
:10A3300032E02044837C1B4F012B03D1637CF35C10
:10A3400093B929E0FEF7E4FD7B7C0A2107EB830744
:10A3500005EB43139B8B7A684B43801A80EAE072CB
:10A36000A2EBE0729A42E9DD607C05EB4013997A3A
:10A37000FAF7DAF8607C05EB40139B7A13B9FFF724
:10A380006FFE03E0335C0BB1FFF776FE637C0121C7
:10A39000E21891740022F254637C05EB43152B7B89
:10A3A000042B36E0EC070020F5070020140F0020F6
:10A3B0005B0F002008000020510F00204C0F0020F0
:10A3C000590E0020440F0020EC0E0020620E0020E9
:10A3D000E50E0020880E002000080140500F0020EC
:10A3E0002218927C984E022A01D1325C62B12B4431
:10A3F000597AFAF799F8607CFFF73EFE637C0221F8
:10A40000E21891740022F254637C05EB43152B7B18
:10A41000052B09D18D4B4FF400429B6813F4004F7C
:10A420008B4B14BF5A611A61FEF772FD6369C01A43
:10A4300080EAE073A3EBE0730A2B40F34D83FAF755
:10A44000CFF9FEF765FD834B586145E3FAF7C8F98C
:10A45000FAF746FB88B9367886B97F4F00F008FED8
:10A46000304601F0C7F83B7823B13046A97AFAF7B5
:10A470005BF83E700123237000E03770207E00F00F
:10A480003DFB744B00221A76FEF742FD6369C01A49
:10A4900080EAE073A3EBE0730A2B04DC6B4B9B6850
:10A4A0005B0500F1198320786A4F002840F00E8385
:10A4B000797C490141F00A0101F0EA0100F067FFEF
:10A4C0000646787C002840F0588201F0DBF9787C61
:10A4D0000C2242436149604F8B18D3F804808A589C
:10A4E0001B7ADFF88091002B18BF90463B5C032B52
:10A4F00000F2CA80DFE803F002611440002E00F091
:10A50000C38005EB4013D97F21B1FAF70DF8637CC6
:10A5100003227CE0597AFAF707F8637C022276E09E
:10A520006EB94F4B1B5C002B4BD1400140F0080132
:10A5300001F0E801304600F02AFF002841D086EA09
:10A54000E673A3EBE673B8F1000FB8BFC8F10008DB
:10A550004345607C02D0002E40F0868059F83020C0
:10A56000934280F08B803F4B03EBC0031979F9F7DE
:10A57000DBFF384B5B7C17E086EAE673A3EBE67300
:10A58000B8F1000FB8BFC8F10008434501D0002E54
:10A5900074D159F83020934208D2324B03EBC003F8
:10A5A0001979F9F7C1FF637C012266E005EB4013DE
:10A5B000597AF9F7B9FF637C43E056BB284B1B5C23
:10A5C000D3B1FEF7A5FC637C4FF00A0E04EB8302C7
:10A5D0005268801A05EB4312918B0028B8BF4042A5
:10A5E0000EFB01F188424FDD1846917AF9F79CFF86
:10A5F000184B00225B7C0AE0400140F0080101F0AA
:10A60000E801304600F0C3FE0028DAD001E0FA5439
:10A610003AE086EAE673A3EBE673B8F1000FB8BF41
:10A62000C8F100084345607C00D0EEB959F83020ED
:10A63000934223D305EB4013597AF9F775FF054B85
:10A640005B7C022219E000BF500F0020000801408F
:10A6500000100140EC070020530F00209C0E00204A
:10A660005A0F0020640E002005EB4013D97F29B15A
:10A67000F9F75AFFAF4B03225B7CFA54677CFEF775
:10A6800047FC04EB87077860607CAB4B00210344F8
:10A690000093AA4B0A4603440193A94BDFF8948226
:10A6A00003EB8003FFF77AFC607CA64F05EB4013B9
:10A6B0009B694BB3F9F72EFF30B398F8110086EA87
:10A6C000E672A2EBE67207EB40139B699A421BD934
:10A6D00000F090FF98F811309B4A0121D15407EB0C
:10A6E00043139B7F43B1BA7F9A4205D1002000F00B
:10A6F00081FF002000F0BCFC637C944A0F33D15CE6
:10A70000012904BF0221D154627CDFF82882510163
:10A710006B185B69DFF82CA2002B69D08C4B9F5C17
:10A720009B46002F64D1002E62D041F0020101F05F
:10A73000E201384601F012F8024698F8110003923F
:10A74000FAF714F998F81110039A0AEB41135B69B0
:10A75000101A80EAE072A2EBE07283EAE37EAEEBCD
:10A76000E37E724544DD002B10DD084600F042FF19
:10A7700098F811300AEB43139B7F5BB39AF81E20C5
:10A780009A4227D1384600F035FF20E038460222B1
:10A7900000F015FE98F811103846490141F0080103
:10A7A00001F0E80100F0C0FD98F811300AEB431306
:10A7B0009B7F7BB19AF81E209A420BD138463946CE
:10A7C000022200F0FCFD3846082100F0ADFD3846BD
:10A7D00000F04EFC607C5D4A00F11503D15C01295C
:10A7E00004BF0221D15401230BF8003000F040FCDB
:10A7F000DFF86CB1DBF80030002B4AD0544A637CA0
:10A80000DFF83081D75C9246002F42D1002E41D034
:10A810005B0143F0020101F0E201384600F09EFFC7
:10A82000024698F811000392F9F730FF039ADBF81B
:10A830000030101A80EAE072A2EBE07283EAE37162
:10A84000A1EBE3718A4235DD002B98F8111003DD8E
:10A85000084600F0CFFE0DE03846022200F0AFFDC2
:10A8600098F811103846490141F0080101F0E8015B
:10A8700000F05AFD607C354A00F11503D15C0129D6
:10A8800004BF0221D15401230AF8003000F0F0FB8C
:10A8900010E07EB9617C0020490141F0080101F01F
:10A8A000E80100F074FD28B9637C05EB4312D289FE
:10A8B00062B10EE0677C274BDB5D002BF4D1FEF725
:10A8C00027FB1C4B03EB8707F8611EE0214AD35C92
:10A8D000DBB1FEF71DFB637C04EB8302D26905EB61
:10A8E0004315801AE98980EAE072A2EBE0720A203F
:10A8F00041438A4209DD184DEA5C32B91846FFF738
:10A90000AFFB0C4B01225B7CEA54607C002EB8BF8D
:10A91000764259F83030074F9E42104D22D2FFF751
:10A9200065FA7B7C05EBC3056A79824225D118461E
:10A93000002120E0EC070020620E0020E50E002040
:10A94000880E0020EC0E0020E40E00205B0F00209B
:10A950006D0E0020580F0020590F0020640E0020BB
:10A960007C0E0020FFF742FA7B7C05EBC30569797A
:10A97000884202D01846FFF70DFA002000F0EBFCE9
:10A9800094F82020C70702F0F802554B48BF42F068
:10A990000102460783F8202005D594F8203043F0C3
:10A9A000020384F82030C50605D594F8203043F022
:10A9B000040384F820304B4B1A78D10716D594F84D
:10A9C0002020D20712D5484A1178CF070ED441F083
:10A9D00001011170454A117841F001011170444A9A
:10A9E00001211170434A127802B91A7094F820308C
:10A9F000DE070AD53A4A92F82120D50705D43E4A07
:10AA0000D178012904BF0221D170990709D594F8A2
:10AA10002120920705D4384A1179012904BF022167
:10AA200011715F0709D594F82120560705D4324AE1
:10AA30005179012904BF02215171050684F82130A2
:10AA4000617C43D5490141F01601002001F0F60177
:10AA500005AA00F085FC9DF81630580609D5204A55
:10AA60002549527C52001B32885C012804BF022019
:10AA70008854190609D5617C1F4A0E3112F811005D
:10AA8000012804BF022002F81100DA0608D5627C12
:10AA9000194952001B32885C012804BF02208854E7
:10AAA0009B0609D5627C144B0E3213F81210012953
:10AAB00004BF022103F81210617C0020490141F01B
:10AAC000160101F0F60105AA00F07EFB044B0022FE
:10AAD0005A74FEF71DFA606107B0BDE8F08F00BF41
:10AAE000EC070020840E0020610E0020740E002070
:10AAF000900F0020600E00205B0F00202DE9F04F2A
:10AB0000BB4D85B02B5C0446002B00F0A2824FEABF
:10AB100040195FFA89F646F07C0103AA002000F094
:10AB20001FFCB44B600003EB0907397A022211F0D5
:10AB3000400F9C467F689DF80E3002FA00F20DD05F
:10AB40004FF0010808FA00F81A4003EA08085CF818
:10AB50000930C7F1000AC3F1000B07E002EA03085D
:10AB6000012282405CF809B01A40BA46A24B11F0AB
:10AB7000800F9B6801F03F0718BF83F40043791EE4
:10AB8000C3F3C033072900F26482DFE811F0080044
:10AB90000800080008001B011B011B011B012B5DA5
:10ABA0000F2B00F25682DFE813F05402100053011D
:10ABB0003C007B01480051005D007000A100D900FD
:10ABC000DE005402F80001013E0246F0140103AA1F
:10ABD000002000F0C5FB46F006069DF80D3005EBA1
:10ABE0008405314600206B6000F0D1FB2146A8604F
:10ABF0000222002000F0E3FB0020314640F2FF7209
:10AC000000F007FB00202146032200F0FAFB023F80
:10AC1000012FDFF8DC8194BF0223042308F80430FD
:10AC200017E2002A00F01582002046F0020100F031
:10AC300095FD724B43F8240029E1B8F1000F00F0B4
:10AC40000882204600F0D6FC062301E221460020BF
:10AC5000032200F0D6FB002046F00801524600F027
:10AC6000D8FA46E1B8F1000F40F0F38146F008064B
:10AC700040463146424600F0CCFA40463146CAF1E1
:10AC8000000200F0C6FA0823E2E1B8F1000F00F07C
:10AC9000E08146F00201002000F060FD0746002040
:10ACA000024646F0080100F0B4FA544B002053F875
:10ACB00024202146D21B43F82420032200F0A1FBCC
:10ACC000002046F006018AEAEA72A2EBEA7200F07E
:10ACD000A0FA002009F0E0013A4600F0ACFA0020AA
:10ACE0002146024600F06BFB0923B1E1002000F091
:10ACF00032FB63001841C10740F1AB8146F0020806
:10AD00004146002000F02AFD3D4B46F0080643F87E
:10AD1000240000200246314600F07BFA0020214644
:10AD2000022200F04CFB00200246414600F083FA6C
:10AD30000020024609F0E00100F07DFA033F2046C2
:10AD40000021F9F727FE012F00F27881002021462B
:10AD5000022200F034FB00203146F6E0B8F1000F8B
:10AD600040F0038175E1B8F1000F40F0728146F0C8
:10AD70000201404600F0F2FC46F008010746424658
:10AD8000404600F046FA0222404609F0E00197FBF7
:10AD9000F2F200F050FA404612E1002000F0DBFA37
:10ADA00063001841C20740F1548147E105EB840775
:10ADB000002046F00601BA6800F02BFA0020214678
:10ADC0003A7942E1295D0F2900F24381DFE811F071
:10ADD00041011A003E0059006600820041019300C3
:10ADE00041014101C300CF00A900FE0038012B0141
:10ADF00010080020EC0E0020000801405C0E00202E
:10AE0000100F002046F0140103AA002000F0A8FA59
:10AE10009DF80D2005EB84035A6000202146022294
:10AE200000F0CDFA002046F0060140F2FF7200F07B
:10AE3000F0F900202146032200F0E3FA062F51D05A
:10AE4000082F4FD0844B04221A5502E1062F09D156
:10AE500005EB84035A68002002F00402214642F008
:10AE6000010204E0082F04D100202146032200F053
:10AE7000C8FA002046F008015A4600F0CAF9032338
:10AE8000E6E0791F012904D81AB1062F2CD104233A
:10AE9000DEE0002B00F0DD800C23D9E0052F09D186
:10AEA00005EB84035A68002002F00402214642F0B8
:10AEB000020204E0072F04D100202146032200F003
:10AEC000A0FA002046F00801CBF1000200F0A1F941
:10AED0000523BDE07A1F012A08D8B8F1000F05D07C
:10AEE000052F01D10223B3E00F23B1E0002B00F0C6
:10AEF000B0800723ACE0002B40F0AB80073F012F70
:10AF00000AD905EB84025268184602F00402214671
:10AF100042F0010200F075FA002046F008015246A6
:10AF200015E0002B40F09580073F012F0AD905EB73
:10AF300084025268184602F00402214642F00202DE
:10AF400000F05FFA002046F00801CAF1000200F0AC
:10AF500060F90A237CE0002B7BD0002046F0020140
:10AF600000F0FCFB05EB8403D8600B2370E0002BA2
:10AF70006FD1184646F002018DE8081000F0EEFB94
:10AF8000DDF804C0009B0CEB09025373074646F042
:10AF9000060118468AEAEA72A2EBEA72009300F010
:10AFA0004AF905EB8402D268009B17440222184636
:10AFB00009F0E00197FBF2F200F03DF9009B184622
:10AFC0002146024600F0FBF90D2341E0002000F08D
:10AFD000C2F963001841C3073BD50E232B5546F039
:10AFE00002052946002000F0B9FB1C4B46F0080181
:10AFF00043F824000020024600F00BF9214600200F
:10B00000022200F0DCF900202946024600F013F984
:10B01000002009F0E001024600F00DF92046002171
:10B02000F9F7B8FC15E000202146022200F0C7F92C
:10B03000002046F00801024600F0EBF80E2307E07E
:10B0400005EB84031A790020214600F0DAF9002389
:10B050002B5505B0BDE8F08F10080020100F002020
:10B06000024B1A5C0AB901221A54704710080020DA
:10B07000024B1A5C0AB10F221A54704710080020C4
:10B08000014B185C704700BF100800200000000052
:10B090002DE9F041144612780746C2F341150E46D9
:10B0A0006DBB444901EB451101F10803187930BB30
:10B0B000D00724D45F2A22D83F48405DF8B912F067
:10B0C000970F1CD1DFF8F88018F8050060B9C97F28
:10B0D00019B1F9F729FA032304E008465978F9F77A
:10B0E00023FA022308F80530DFF8D88018F8053075
:10B0F0002BB10020FEF7C0FF002308F805302178AF
:10B1000000220220F9F7ACFD3070617800220220A5
:10B11000F9F7A6FD7070A17800220220F9F7A0FDD2
:10B12000B07001220220E178F9F79AFDF0702378DF
:10B13000DA073DD45F2B3BD803F01E02082A12D059
:10B14000142A2BD0062A33D1242257435B090C2220
:10B1500002FB0373A178E278184F42EA01223B44D4
:10B160005A60BDE8F081242179435B090C2000FB83
:10B170000313A678E578114A45EA0625D550A37849
:10B180001B0715D527787F0900FB0717D3596FEAEE
:10B1900003536FEA1353D351BDE8F08124214F4389
:10B1A0005B090C2101FB0373044FE2783B441A72E4
:10B1B000BDE8F081EC0E0020580F00209C0E00200E
:10B1C000530F0020590F002007B513788DF8001099
:10B1D0008DF80130537801A98DF8023093786A46D2
:10B1E0008DF80330FFF754FF03B05DF804FB07B59B
:10B1F0008DF802309DF810308DF800108DF8012088
:10B2000001A96A468DF80330FFF742FF03B05DF8ED
:10B2100004FB07B500238DF800108DF801308DF880
:10B220000320131201A96A468DF80230FFF730FFA0
:10B2300003B05DF804FB5F292DE9F34105460E4696
:10B24000144658D811F01E07C1F3411202D0022F44
:10B250001DD050E000EB40031A4430491201881819
:10B2600043688C50C3EB040EBEF1000FB8BFCEF1A3
:10B27000000EBEF5000F08DB9C42CCBF284C294CC9
:10B280000A441C440123137335E0077333E000EBD9
:10B290004007224B17443F01D91924F07F4EC1F8D3
:10B2A00008E04C6001F10800D9599846C4EB010E42
:10B2B000BEF1000FB8BFCEF1000EBEF5000F18DBD7
:10B2C000A142CCBF164B174B520123448DF80020EE
:10B2D0001A148DF801201A128DF80220284601A9AF
:10B2E0006A468DF803304744FFF7D2FE01233B73D3
:10B2F00001E00023037123148DF801302846231246
:10B3000001A96A468DF800608DF802308DF803407F
:10B31000FFF7BEFE02B0BDE8F08100BF681100205B
:10B32000FFFF7F00010080FF07B511F01C0202D172
:10B33000FFF781FF0CE000238DF800106A4601A999
:10B340008DF801308DF802308DF80330FFF7A0FE44
:10B3500003B05DF804FB012102200A46F9F780BC26
:10B3600013B541F0010114468DF8041001AA694695
:10B37000FFF78EFE9DF801309DF8000023709DF8C8
:10B38000023063709DF80330A37002B010BD07B5A2
:10B3900041F001018DF8041001AA6946FFF778FE1B
:10B3A0009DF803309DF8020043EA0020030544BFE6
:10B3B0006FEA00506FEA105003B05DF804FB73B5FC
:10B3C0004901CCB244F01503164601A96A46054668
:10B3D0008DF80030FFF75CFE9DF8053044F0140452
:10B3E0008DF801309DF80630284601A96A468DF88F
:10B3F00000408DF802308DF80360FFF749FE02B07F
:10B4000070BD73B54901CCB244F01503164601A9CD
:10B410006A4605468DF80030FFF73AFE9DF8053084
:10B4200044F014048DF801309DF80730284601A936
:10B430006A468DF800408DF802608DF80330FFF702
:10B4400027FE02B070BD2DE9F3474001C7B2C1F33A
:10B450000A06002047F0180101AAFFF781FF9DF8B6
:10B46000058030464FEA181908F00F08C8450FDB71
:10B4700004F006FCC9EB08080446012000FA08F0B5
:10B480000D4604F00DFC0022354B04F06FFC10E07B
:10B4900004F0F6FBC8EB09080446012000FA08F0A6
:10B4A0000D4604F0FDFB02460B4600202C4904F03B
:10B4B00087FD02460B462046294604F081FD04F034
:10B4C00017FF04F0FFFB24A3D3E9002304F04EFC94
:10B4D00004F00EFF04F0F6FB0022224B04F046FCC1
:10B4E0004FF0FF3904460D46CA464FF000080120D0
:10B4F00000FA08F004F0D4FB02460B462046294629
:10B5000004F034FC04F0CCFEA0F18002802A38BFA5
:10B51000C14608F1010828BF5046B8F10E0F01D00E
:10B520008246E4E700248DF8050047F0120120462A
:10B5300001AA8DF804408DF80690FFF745FE2046DD
:10B5400047F00C013246FFF764FE204602B0BDE82A
:10B55000F08700BFAFF3008004560E2DB29DEF3F81
:10B56000000060400000204073B54C0804EB440428
:10B57000B42304F5807403FB0044054620460E46C0
:10B58000FCF7FEFE8DF80400601CFCF7F9FE8DF858
:10B590000500A01CFCF7F4FE46EA45118DF80600F4
:10B5A000C9B2002001AAFFF70FFE02B070BD37B587
:10B5B0000C46640841EA401101AA0546C9B20020C0
:10B5C00004EB4404FFF7CCFE04F58074B42303FBC2
:10B5D00005449DF804102046FCF7F9FD601C9DF819
:10B5E0000510FCF7F4FDA01C9DF80610FCF7EFFD1C
:10B5F00003B030BD10B5C4B221466401E4B20020EE
:10B600000222FFF7DCFE44F008010020FFF78CFE69
:10B6100044F00A010020BDE81040FFF785BE37B5B1
:10B62000400140F01604E4B20D4601AA2146002074
:10B63000FFF796FE9DF8053015F0010F14BF43F09B
:10B64000400323F040038DF805309DF8053015F0D8
:10B65000020F14BF43F0100323F010030020214613
:10B6600001AA8DF805308DF80600FFF7ADFD03B097
:10B6700030BD37B5400140F01604E4B20D4601AAD2
:10B6800021460020FFF76CFE9DF8053015F0010FF4
:10B6900014BF63F07F0303F07F038DF805309DF83E
:10B6A000053015F0020F14BF43F0200323F02003F0
:10B6B0000020214601AA8DF805308DF80600FFF71D
:10B6C00083FD03B030BD07B5400140F0160101F025
:10B6D000F60101AA0020FFF743FE9DF80530C3F3F1
:10B6E0008010DB0648BF40F0020003B05DF804FBA9
:10B6F00007B5400140F0160101F0F60101AA002053
:10B70000FFF72EFE9DF80530D8099B0648BF40F094
:10B71000020003B05DF804FB70B50F4C0001231864
:10B720009A68914209DD8A1AC2F18075AA425E6860
:10B7300001DC324409E0751B0AE00ADA521AC2F150
:10B740008075AA425E6802DCB21A5A6001E0354494
:10B750005D602044816070BD6811002037B541F004
:10B7600001030C4601AA69468DF804300546FFF72F
:10B770008FFC9DF802309DF801201B0243EA024332
:10B780009DF8032043EA02010B0248BF41F07F41CC
:10B790005F2C19D8C4F3411214F01E040ED0022CF1
:10B7A00012D105EB45051544E8B221F07F41FFF7C2
:10B7B000B3FF074B03EB0515696805E005EB45058D
:10B7C0002A44034B12019958084603B030BD00BF0C
:10B7D0006811002038B50C4668210546FFF7BEFF0A
:10B7E00014B140F0010201E020F001022846682176
:10B7F000BDE83840FFF71FBD38B50C466821054647
:10B80000FFF7ACFF14B140F0100201E020F010028D
:10B8100028466821BDE83840FFF70DBD13B5184B29
:10B8200000245A7E93F8283012F0010F14BF212211
:10B830002022DB0748BF42F0100200206821FFF7FA
:10B84000FAFC009420467E2120222346FFF7CFFCFD
:10B85000E1B200200134FFF787FE1D2CF8D10C2146
:10B860000020FFF77BFF01460020FFF7ECFD0020E2
:10B87000162143F2FF1202B0BDE81040FFF7C9BC29
:10B8800008000020F0B5450185B0044645F00303EB
:10B8900003AA002002A98DF80C30FFF7F9FB9DF8F0
:10B8A0000A109DF80930090241EA03419DF80B3066
:10B8B00020461943FFF730FF15482301C21802F153
:10B8C00008010E790EB3134E0C2707FB0464247A8B
:10B8D000DCB9C6585268B71A002FB8BF7F42B7F517
:10B8E000000F05DB9642CCBF0B4B0C4B134401E021
:10B8F000C3580C71DAB200920020C3F3074205F07E
:10B90000E001C3F30723FFF772FC05B0F0BD00BFF1
:10B91000681100209C0E0020FFFF7F00010080FFC7
:10B92000074B10B518681C4601460A780B460131D2
:10B930001AB12C2AF9D100221A700133236010BDEC
:10B940002008002070B5124B06461B78E3B1FCF7C7
:10B95000FBFE104C054618B100232371012070BD79
:10B96000A368E268934207D25A1C23441B7C01203F
:10B9700033702071A26070BD04F11000FDF745FE28
:10B98000A560E060284670BDBDE87040FCF7DCBEF5
:10B99000580E00202008002010B50E4B1B7813B164
:10B9A0000D4C23791BB9BDE81040FCF7B3BE226DE6
:10B9B0000D2802F101032244236582F8540002D0CD
:10B9C0003F2B00D829B919460448FDF74FFE002344
:10B9D000236510BD580E00202008002074080020A8
:10B9E00070B50121044686B02020FFF7D5FF002C5A
:10B9F00004DA2D200121FFF7CFFF644200230A2142
:10BA000094FBF1F201FB124101AE30311D46995514
:10BA100014460133002AF2D1705D0121FFF7BCFF0B
:10BA200015F1FF35F8D206B070BD2DE9F34105469A
:10BA30000DF10700FFF786FF974C002800F0C88043
:10BA400094F894309DF80700944E03BB737840330C
:10BA500098420DD1D4F89830002B40F0B98031795C
:10BA6000012331F0010184F8943040F0B180ADE061
:10BA70000D2801D01B2801D1002305E0D4F898300F
:10BA80007E2B00F2A5800133C4F89830A0E0317914
:10BA900031F0010101D1FFF77FFF9DF807301F2B27
:10BAA0000CD9D4F898207C497E2A00F28280501C60
:10BAB0000A44C1F8980082F89C307AE0082B08D13B
:10BAC000D4F89830002B74D0734A013BC2F89830F8
:10BAD0006FE00D2B6DD1D4F89830002B69D03379FD
:10BAE000112B16D16D4B0121587800274030C0B280
:10BAF000FFF752FFD4F898309F4206D2684B0121DD
:10BB0000D85DFFF749FF0137F4E70D200121FFF76A
:10BB100043FF0023D4F898802768C4F81C311A46E4
:10BB20001946424537D0012911D002D3022925D028
:10BB30002FE0DFF864C10CF19C00105C202828D0B5
:10BB40000CEB030181F820010133012121E052486F
:10BB500000F19C0C12F80CC0BCF1200F0AD1012B93
:10BB600004D91844002180F8201101334D4F0221DF
:10BB70001F440EE0184480F820C109E0DFF818C126
:10BB80000CF19C00105C202803D09C448CF8200110
:10BB900001330132C5E70022C4F81C31234483F885
:10BBA00020210123276084F89F3184F89420C4F871
:10BBB00098209DF807301B2B0AD133790021012BE7
:10BBC000C4F8981084F8941002D10D20FFF7E4FE19
:10BBD00094F89F01002600285AD02F4B83F89F61CC
:10BBE000F7B2DFF8DC80C7EBC70708EB07042D4886
:10BBF000214605F09DFA28B9A6796379F1072B70E3
:10BC000036D506E018F807300136002BE8D12B7046
:10BC10003DE0FFF785FE2B780446042B14D1224922
:10BC200005F086FA08B900230CE020461F4905F00C
:10BC30007FFA08B9012305E01D49204605F078FA8E
:10BC400090B902236B7013E00D2B0ED1194905F04A
:10BC50006FFA0028E7D02046174905F069FA002856
:10BC6000E8D020461549E9E7204605F05DFA6870FE
:10BC7000B20704D5FFF754FE05F056FAA870730713
:10BC800005D5FFF74DFE05F04FFAC5F8030001207A
:10BC900002B0BDE8F08100BF2008002008000020AD
:10BCA000BC08002040090020EA190108EE1901082B
:10BCB000F2190108F8190108FE190108031A010810
:10BCC000E518010838B50D4D0446A878012140302B
:10BCD000C0B2FFF761FE687801214030C0B2FFF7C3
:10BCE0005BFE2078FFF77CFE6068FFF779FEBDE819
:10BCF00038400D200121FFF74FBE00BF0800002093
:10BD00007047FEE7FEE7FEE7FEE7704770477047C3
:10BD1000704770477047704770477047704770476B
:10BD2000704770477047704770477047704770475B
:10BD300070477047704708B5014B1B68984708BDAE
:10BD4000780E002008B5024B1B68984708BD00BF5D
:10BD5000540F002008B5024B1B68984708BD00BF70
:10BD6000E80E002008B5024B1B68984708BD00BFCD
:10BD70000C0F00207047704770477047704770473E
:10BD800070477047704770477047704770477047FB
:10BD900070477047704770477047704770477047EB
:10BDA00070477047704770477047704770477047DB
:10BDB000704770477047704770477047704700BFC3
:10BDC00008B5144B98420FD003F5A053984213D0F6
:10BDD000A3F5C05398421BD14FF40070012101F02C
:10BDE000FBFB4FF400700EE04FF48060012101F086
:10BDF000F3FB4FF4806006E04FF40040012101F0B6
:10BE0000EBFB4FF400400021BDE8084001F0E4BB2B
:10BE100008BD00BF0028014043680A6823F470236E
:10BE200023F4807313430A7910B543EA0223436075
:10BE30008A68CB6884681A43084B234013434A79C5
:10BE400043EA420383600B7CC26A013B22F4700226
:10BE5000DBB242EA0353C36210BD00BFFDF7F1FF3E
:10BE600000230360037143718360C3600123037483
:10BE70007047836811B143F0010301E023F001032F
:10BE800083607047836811B143F4807301E023F449
:10BE9000807383607047C9B243680AB1194301E0F7
:10BEA00023EA010141607047836843F0080383601F
:10BEB00070478068C0F3C0007047836843F0040394
:10BEC000836070478068C0F380007047836811B159
:10BED00043F4A00301E023F4A0038360704780686B
:10BEE000C0F3805070474368013923F4604343EA4C
:10BEF000413343607047436811B143F4006301E08C
:10BF000023F4006343607047092970B50DD9A1F18E
:10BF10000A0404EB44040725A540A340C66826EAAA
:10BF2000050545EA0304C4600BE001EB4104072565
:10BF3000A54003FA04F4066926EA050545EA040368
:10BF40000361062A0CD8013A02EB82021F239340B8
:10BF500001FA02F2446B24EA03031A43426370BD00
:10BF60000C2A0CD8073A02EB82021F23934001FAF5
:10BF700002F2046B24EA03031A43026370BD0D3A14
:10BF800002EB82021F23934001FA02F2C46A24EA00
:10BF900003031A43C26270BD836811B143F4801376
:10BFA00001E023F4801383607047C06C80B2704757
:10BFB000014B1868704700BF4C240140436811B121
:10BFC00043F4806301E023F4806343607047436877
:10BFD00011B143F4805301E023F480534360704770
:10BFE000836823F4E043194381607047836811B18B
:10BFF00043F4004301E023F4004383607047836807
:10C0000011B143F4021301E023F40213836070477B
:10C010008068C0F340507047092970B50DD9A1F16F
:10C020000A0404EB44040725A540A340C66826EA99
:10C03000050545EA0304C4600BE001EB4104072554
:10C04000A54003FA04F4066926EA050545EA040357
:10C050000361846B931CC4F301555B1BDBB203EBE0
:10C0600083031F229A40994024EA020444EA010310
:10C07000836370BD836B013923F4401343EA01539A
:10C0800083637047425070472831405880B27047F0
:10C09000436823F4400323F400731943416070475D
:10C0A000416282627047436823F01F031943416075
:10C0B0007047054B9A6810B142F4000201E022F487
:10C0C00000029A60704700BF0024014003681942D3
:10C0D0000CBF002001207047C943016070474368CE
:10C0E000006810EA112004D0C9B219420CBF002028
:10C0F000012070476FEA11210160704708B54FF0C9
:10C100000070012101F074FABDE808404FF00070A2
:10C11000002101F06DBA2E4B01221A605A6812F00C
:10C12000010252D00278012A1A680CBF42F0800244
:10C1300022F080021A604378012B254B1A680CBF4D
:10C1400042F0400222F040021A608278012A1A6806
:10C150000CBF42F0200222F020021A60C378012BAB
:10C160001B4B1A680CBF42F0100222F010021A603A
:10C170000279012A1A680CBF42F0080222F0080274
:10C180001A604379012B124B1A680CBF42F004026B
:10C1900022F004021A608279C379920742EA0362AC
:10C1A000037A42EA0342437A42EA03524389013B5B
:10C1B0001A43074BDA611A6822F001021A605868C4
:10C1C00000F0010080F0010070471046704700BF8A
:10C1D00000640040037801219940354B70B5D3F8D5
:10C1E000002289B242F00102C3F80022D3F81C22D7
:10C1F000CC432240C3F81C228278A2B9D3F80C2287
:10C2000046892240C3F80C220278C588483245EAA4
:10C21000064543F8325083880289057843EA024292
:10C22000244BED005A518378012B15D1204B868881
:10C23000D3F80C22C5880A43C3F80C22027845EAD9
:10C240000645483243F8325043890289057843EA6B
:10C250000242184BED005A514378154A1BB9D2F8E7
:10C260000432234002E0D2F804320B438589C2F83D
:10C2700004320F4B2DB9D2F814522C40C2F814429C
:10C2800006E0012D04D1D3F814220A43C3F8142286
:10C29000827B012A04D1D3F81C221143C3F81C125B
:10C2A000D3F8002222F00102C3F8002270BD00BFC3
:10C2B00000640040446600400023037043708370B4
:10C2C000C370037143718371C3710323037202232B
:10C2D0004372012343817047044B5A6909B11043EB
:10C2E00001E022EA00005861704700BF006400408E
:10C2F000334A03469168F0B5480107D491680901B3
:10C3000006D49268D20005D40420F0BD002002E0DB
:10C31000012000E00220010101F1804202F5C84243
:10C32000D2F8804104F00104C2F880411C7A5D7AA1
:10C330003CB91E6876051E60D2F8804125432E4325
:10C3400007E05E682C43F6005E60D2F880712643F9
:10C350003E43C2F880619C7A01F1804104F00F04F1
:10C360009C72D2F8844101F5C84124F00F04C2F850
:10C3700084419D7AD2F884412C43C2F884415D7B8C
:10C380009C7B2D0445EA0465DC7A25431C7B45EA49
:10C390000425C1F8885101F5C474597C9D7C0904B9
:10C3A00041EA0561DD7B1B7C294341EA032363608D
:10C3B000D2F8803143F00103C2F88031F0BD00BFF4
:10C3C0000064004001281DD00FD3022829D1174A4C
:10C3D0009368916803F48033926801F400319B0BF9
:10C3E00043EA1143C2F3007219E0104A916893685E
:10C3F000926801F0010103F0020343EA8103C2F3F2
:10C4000080620CE0094A9368916803F48073926833
:10C4100001F400719B0943EA1123C2F3C062134384
:10C4200000E00023024AD05C704700BF0064004077
:10C43000C5190108012808D002D302280AD0704784
:10C44000074B9A6842F0800208E0054B9A6842F474
:10C45000004203E0024B9A6842F400029A6070477F
:10C4600000640040034B202208B9DA6070471A616B
:10C47000704700BF0064004010B9064BD86803E065
:10C48000012804D1034B186900F003007047002015
:10C49000704700BF00640040020102F1804303F5D1
:10C4A000C84310B5D3F8B04104F00404E4B20C72F0
:10C4B00024B9D3F8B041640D0C6003E0D3F8B04167
:10C4C000E4084C60D3F8B04104F002044C72D3F895
:10C4D000B44104F00F048C72D3F8B4311B0ACB744E
:10C4E00002F1804303F5C843D3F8B84103F5DC7289
:10C4F000CC72D3F8B841240A0C73D3F8B841240C99
:10C500004C73D3F8B831BDE810401B0E8B735368E1
:10C51000CB7353681B0A0B7453681B0C4B74536822
:10C520001B0E8B74FFF79EBF044B1A6842F0020289
:10C530001A601868C0F34000704700BF00640040F4
:10C54000054B1A6822F002021A60186880F0020097
:10C55000C0F34000704700BF00640040034B9B697C
:10C5600018420CBF00200120704700BF006400404B
:10C57000024B9A6922EA000098617047006400400B
:10C58000202838D010D8062828D006D804282FD044
:10C59000052848D1254B986833E0072823D0082880
:10C5A00041D1224BD86836E0B0F5007F2CD007D8B7
:10C5B000402823D0B0F5807F35D11C4B986920E00E
:10C5C000B0F5803F2AD0B0F5003F22D0B0F5806FA3
:10C5D00029D1164B9869C0F380007047134B9868B7
:10C5E000C0F300207047114B9868C0F300407047BB
:10C5F0000E4BD86814E00D4B186911E00B4B18690D
:10C6000009E000F001007047084B9869C0F3400052
:10C610007047064B5868C0F300107047034B5868CA
:10C62000C0F3C00070470020704700BF00640040A6
:10C63000202835D00CD8062824D004D8042829D0A6
:10C6400005281DD07047072821D0082824D070471E
:10C65000B0F5007F2FD005D8402823D0B0F5807FDB
:10C6600024D07047B0F5803F2BD0B0F5003F2AD0E2
:10C67000B0F5806F2AD1164B9A6922F004021EE0B1
:10C68000012201E04FF48072114B9A6070474FF421
:10C690008032F9E7082200E010220D4BDA60704783
:10C6A000082200E010220A4B1A617047084B9A6971
:10C6B00022F0010203E0064B9A6922F002029A611D
:10C6C0007047082200E01022014B5A60704700BFFB
:10C6D00000640040036823F001030360002303604B
:10C6E00043608360C3602D4B984234D011D83C3BEB
:10C6F00098422AD006D8283B984222D01433984238
:10C7000021D07047264B984221D01433984220D034
:10C710007047244B98422DD008D8A3F567739842F0
:10C720001ED003F5627398421FD070471E4B98428B
:10C7300029D0143398422BD0283B98422DD11B4B43
:10C740001DE01B4B12E01A4B15E0194B17E0184B7C
:10C750001AE0174B1DE0164B5A6842F470021BE0BA
:10C76000134B5A6842F0706216E0104B5A6842F060
:10C770000F0211E00D4B5A6842F0F0020CE05A68CB
:10C7800042F4706208E0094B5A6842F4704203E0D8
:10C79000064B5A6842F470225A6070476C0002409F
:10C7A000440002401C0402404404024000040240D1
:10C7B000000002408A6810B50C6A036814430A69D5
:10C7C00023F4FF4314434A6923F0700314438A6936
:10C7D0001443CA6914434A6A14438A6A22431343BE
:10C7E0000360CB6843600B6883604B68C36010BD17
:10C7F0000023036043608360C3600361436183611E
:10C80000C3610362436283627047036811B143F0FE
:10C81000010301E023F001030360704703680AB1DC
:10C82000194301E023EA010101607047406880B2CA
:10C830007047C3004CBF044B044B1B6803420CBF42
:10C8400000200120704700BF0004024000000240A9
:10C85000C3004CBF014B024B5860704700040240BC
:10C8600000000240C3004CBF034B044B1B68034253
:10C870000CBF00200120704700040240000002406D
:10C88000C3004CBF014B024B58607047000402408C
:10C8900000000240044B00221A605A609A60DA607D
:10C8A000024A5A61704700BF00040140FFFF0700C1
:10C8B000837930B50168027943B3194BCC431D68C5
:10C8C00002F1804225401D605D6802F582322C40F5
:10C8D0005C6014682143116002689C68D1430C407D
:10C8E0009C60DC682140D9604179102906D19968A3
:10C8F00011439960D9680A43DA6030BD01F1804381
:10C9000003F5823319680A431A6030BD02F180438F
:10C9100003F582331A6822EA0101196030BD00BFB5
:10C920000004014000230C220360037142718371F3
:10C930007047024B1A6910431861704700040140A8
:10C94000034B5B6918420CBF00200120704700BFF9
:10C9500000040140014B5861704700BF00040140D2
:10C96000054B1A685B69034004D010420CBF0020DD
:10C97000012070471846704700040140014B586180
:10C98000704700BF00040140044B1A6802F03802EF
:10C990001A601A6810431860704700BF00200240F8
:10C9A000044B1A6822F008021A601A6810431860D3
:10C9B000704700BF00200240044B1A6822F01002AA
:10C9C0001A601A6810431860704700BF00200240C8
:10C9D000034B044A5A6002F188325A60704700BF24
:10C9E0000020024023016745024B1A6942F0800291
:10C9F0001A61704700200240014BD86980087047D7
:10CA000000200240014B186A704700BF002002401E
:10CA1000024BD869C0F34000704700BF00200240BD
:10CA2000024B1868C0F34010704700BF002002405E
:10CA3000044B1A6909B1104301E022EA00001861B1
:10CA4000704700BF002002400128064B03D1D8697F
:10CA500000F001007047DB6818420CBF0020012085
:10CA6000704700BF00200240014BD860704700BFF4
:10CA700000200240084BDA68D10709D4DA6852076F
:10CA800008D4DB6813F0100F0CBF0420032070479C
:10CA900001207047022070470020024013B5044671
:10CAA000FFF7E8FF01280FD164B100230193FF23B2
:10CAB0000193019B13B1019B013BF9E7FFF7DAFFFB
:10CAC000013CEFE7052002E0002C08BF052002B082
:10CAD00010BD38B5054640F6FF70FFF7DFFF0428AC
:10CAE00014D10B4C40F6FF70236943F0020323611D
:10CAF0006561236943F040032361FFF7CFFF0128FD
:10CB000004D0226941F6FD731340236138BD00BF94
:10CB10000020024010B540F6FF70FFF7BFFF042869
:10CB200013D10A4C40F6FF70236943F004032361DC
:10CB3000236943F040032361FFF7B0FF012804D0CD
:10CB4000226941F6FB731340236110BD00200240AF
:10CB500010B540F6FF70FFF7A1FF042829D1154C4E
:10CB6000154B40F6FF70A36003F18833A36023697F
:10CB700043F020032361236943F040032361FFF75F
:10CB80008DFF04280ED1226941F6DF731340236123
:10CB90002369A52243F010032361084B0F201A805C
:10CBA000FFF77CFF012804D0226941F6EF731340A0
:10CBB000236110BD002002402301674500F8FF1FDC
:10CBC00070B505460F200E46FFF768FF042817D101
:10CBD0000C4C0F20236943F001032361B3B22B8077
:10CBE000FFF75CFF042804D1360C6E800F20FFF79E
:10CBF00055FF012804D0226941F6FE7313402361DA
:10CC000070BD00BF0020024070B505460F200E46E3
:10CC1000FFF744FF04280FD1084C0F20236943F08D
:10CC2000010323612E80FFF739FF012804D0226918
:10CC300041F6FE731340236170BD00BF0020024027
:10CC400070B505460F200E46FFF728FF042814D1C3
:10CC50000A4C0B4B0F20A36003F18833A3602369B8
:10CC600043F0100323612E80FFF718FF012804D042
:10CC7000226941F6EF731340236170BD002002402A
:10CC80002301674510B504460F20FFF707FF04286E
:10CC90003ED1204B2049E443996001F188319960ED
:10CCA0001969E2B241F01001FF2A196104D1C4F3FD
:10CCB0000723FF2B08D10EE0184B0F201A81FFF736
:10CCC000EDFE04281CD1F2E7144A0F205381FFF730
:10CCD000E5FE042814D1C4F30743FF2B06D00F4A06
:10CCE0000F209381FFF7DAFE042809D1240EFF2CD0
:10CCF00001D1042006E0094B0F20DC81FFF7CEFEB6
:10CD0000012805D0034A41F6EF7311690B40136106
:10CD100010BD00BF002002402301674500F8FF1F3F
:10CD200038B5054640F6FF70FFF7B8FE042836D147
:10CD30001B4C1C4B40F6FF70A36003F18833A360CB
:10CD4000236943F020032361236943F040032361F7
:10CD5000FFF7A4FE04281BD1226941F6DF731340BC
:10CD60002361236943F0100323610F4B0DB10022AF
:10CD700000E0A5221A8040F6FF70FFF78FFE012821
:10CD80000DD0074A41F6EF7311690B40136138BDAE
:10CD9000012804D0226941F6DF731340236138BDB6
:10CDA000002002402301674500F8FF1FF8B5114C31
:10CDB000114B0546A36003F18833A3600F200E4694
:10CDC0001746FFF76BFE042813D1236947F0F807D5
:10CDD00043F0100323613E43084B35435D800F2031
:10CDE000FFF75CFE012804D0226941F6EF7313407F
:10CDF0002361F8BD002002402301674500F8FF1FB2
:10CE000008B5264B98422FD011D8A3F5006398425D
:10CE10001ED003F58063984220D0A3F500639842AA
:10CE20003AD10420012100F0D7FB04202FE01C4B55
:10CE300098421FD003F58063984221D0A3F5006388
:10CE4000984229D14020012100F0C6FB40201EE07D
:10CE50000820012100F0C0FB082018E0102001216B
:10CE600000F0BAFB102012E02020012100F0B4FBFA
:10CE700020200CE08020012100F0AEFB802006E0A5
:10CE80004FF48070012100F0A7FB4FF48070002167
:10CE9000BDE8084000F0A0BB08BD00BF0014014081
:10CEA000001C014008B50120014600F095FBBDE8DB
:10CEB00008400120002100F08FBBCB78F0B5DA06E6
:10CEC00048BF8A78098803F00F0548BF154311F061
:10CED000FF0F1DD0046800220127974007EA0106D2
:10CEE000BE4211D197004FF00F0C0CFA07FC05FA67
:10CEF00007F724EA0C04282B44EA070401D1466111
:10CF000002E0482B08BF06610132082AE4D1046020
:10CF1000FF291FD94468002202F108060127B74003
:10CF200007EA0106BE4211D197004FF00F0C0CFA30
:10CF300007FC05FA07F724EA0C04282B44EA070447
:10CF400001D1466102E0482B08BF06610132082A80
:10CF5000E2D14460F0BD4FF6FF730380022383707B
:10CF60000423C3707047836819420CBF002001205E
:10CF70007047806880B27047C36819420CBF0020B8
:10CF800001207047C06880B27047016170474161FD
:10CF900070470AB10161704741617047C1607047D5
:10CFA00041F4803383618161836183698369704760
:10CFB000054B1A6822F07F021204120C114341EA59
:10CFC00000101860704700BF00000140014B18605E
:10CFD000704700BF1C00204230B5134A00F44015D2
:10CFE000B5F5401F536884B206D1556823F07063CD
:10CFF00025F0706555600FE0C20205D5C0F303420D
:10D00000032505FA02F203E0420D120104FA02F2CE
:10D0100023EA020343F0706319B1400D000184401C
:10D020002343014A536030BD0000014001F0030377
:10D030009B000F229A40984001F0FC0101F18041D1
:10D0400001F5803110B58C6824EA02028A608A6892
:10D0500002438A6010BD00BF0B4B6FF070424FF06F
:10D06000FF31C3F88010C3F88420C3F88011C3F8DF
:10D070008421002202F1C001013200200F2A43F86E
:10D080002100F7D1704700BF00E100E0094B4FF0ED
:10D09000206209495A6000229A60D9601A615A6177
:10D0A0009A61DA611A625A624FF0FF329A62DA626A
:10D0B0001A63704700ED00E00000FA0540F0BF6021
:10D0C000024B40F40030D860704700BF00ED00E034
:10D0D000C27830B503785AB31B4A4478D268857851
:10D0E000D243C2F30222C2F1040104FA01F10F2477
:10D0F000D4402C400C4303F00301C9002401FF225B
:10D100008C408A4003F0FC0303F1604303F5614364
:10D11000D3F8005325EA020122400A43C3F8002352
:10D1200003780122590903F01F0302FA03F306E012
:10D130005909012203F01F0302FA03F32031034AC5
:10D1400042F8213030BD00BF00ED00E000E100E01A
:10D150000023037043708370C3707047F6F7FDBF00
:10D16000F6F7FDBFF6F7FDBFF6F7FDBF0001F6F7D6
:10D17000FCBFF6F7FDBF024B5868C0F3093070479B
:10D1800000ED00E000F01F03012202FA03F3400962
:10D19000044A403052F820001840C31A58425841FF
:10D1A000704700BF00E100E0014B1860704700BF0E
:10D1B00000EF00E04209012300F01F0003FA00F035
:10D1C000024B603243F82200704700BF00E100E0EC
:10D1D000024B5868C0F30900704700BF00ED00E043
:10D1E00000F01F03012202FA03F34009044A8030D1
:10D1F00052F820001840C31A58425841704700BFE7
:10D2000000E100E0014B1868704700BF00ED00E04E
:10D2100021F0604121F07F01014B08439860704785
:10D2200000ED00E0014A024BDA6070470400FA05A5
:10D2300000ED00E0014A024BDA6070470100FA0598
:10D2400000ED00E0044B1A6909B1104301E022EA45
:10D2500000001861704700BF00ED00E0012300F0FE
:10D260001F0003FA00F0044B5A6A09B1104301E0B1
:10D2700022EA00005862704700ED00E0114B30B523
:10D28000DB68DB43C3F30223C3F10404A140FF24A2
:10D2900024FA03F31A401143C0F30122D200944050
:10D2A000090101FA02F2C0F38110800000F1604030
:10D2B00000F56D40836923EA0404846185692A438B
:10D2C000826130BD00ED00E0C0F383200123834084
:10D2D000034A506A1840C31A58425841704700BF69
:10D2E00000ED00E000F01F00012101FA00F0024B08
:10D2F0005A6802435A60704700ED00E000F01F00DA
:10D30000411E012000FA01F1024B5A680A435A609B
:10D31000704700BF00ED00E0C0F38330012383407D
:10D32000034A506A1840C31A58425841704700BF18
:10D3300000ED00E0C0F38142094B0AB9D86A70479A
:10D34000012A0AD1C0F30152986AD300D840022AB8
:10D3500014BF00F00F00C0B27047186B704700BFD9
:10D3600000ED00E0034B10F4800F0CBF586B986B7E
:10D37000704700BF00ED00E00C4B1A6842F001025C
:10D380001A6059680A4A0A405A601A6822F0847280
:10D3900022F480321A601A6822F480221A605A68D5
:10D3A00022F4FE025A6000229A6070470010024088
:10D3B0000000FFF80C4BB0F5803F1A6822F4803271
:10D3C0001A601A6822F480221A6003D0B0F5802F08
:10D3D00004D070471A6842F4803202E01A6842F4BE
:10D3E000A0221A60704700BF00100240034B1A6869
:10D3F00022F0F80242EAC0001860704700100240B4
:10D40000014B1860704700BF00004242034B5A684E
:10D4100022F47C1211430843586070470010024008
:10D42000014B1860704700BF60004242034B5A68CE
:10D4300022F0030210435860704700BF0010024002
:10D44000024B586800F00C00704700BF001002400B
:10D45000034B5A6822F0F00210435860704700BF37
:10D4600000100240034B5A6822F4E06210435860F7
:10D47000704700BF00100240034B5A6822F460520C
:10D4800042EAC0005860704700100240044B1A780E
:10D4900009B1104301E022EA00001870704700BF94
:10D4A00009100240014B1860704700BFD80042428B
:10D4B000034B5A6822F4404210435860704700BF43
:10D4C00000100240064B002201281A701A7002D088
:10D4D000042802D070471870704705221A707047F0
:10D4E00020100240014B1860704700BF8004424288
:10D4F000024B1A6A10431862704700BF00100240C6
:10D50000014B1860704700BF3C0442421C4B10B5F1
:10D510005A6802F00C02042A01D0082A01D0194AE4
:10D520000EE05A685968C2F38342CC0302F102024A
:10D5300002D55968890301D5134900E011494A43CE
:10D5400002605968114AC1F30311545C0168E1405B
:10D5500041605C68C4F30224145D21FA04F4846021
:10D560005C68C4F3C224145DE140C1605B68C3F32E
:10D5700081331A44137CB1FBF3F1016110BD00BF8C
:10D580000010024000127A0000093D00CD19010888
:10D59000044B5A6909B1104301E022EA00005861C6
:10D5A000704700BF00100240044B9A6909B1104354
:10D5B00001E022EA00009861704700BF00100240BD
:10D5C000044BDA6909B1104301E022EA0000D86196
:10D5D000704700BF00100240044BDA6809B11043E5
:10D5E00001E022EA0000D860704700BF001002404E
:10D5F000044B1A6909B1104301E022EA00001861E6
:10D60000704700BF00100240014B1860704700BF18
:10D6100040044242014B1860704700BF4C00424238
:10D62000014B1870704700BF071002404309012BDF
:10D63000074A01D1136803E0022B0CBF136A536A37
:10D6400000F01F0023FA00F000F00100704700BF57
:10D650000010024008B53120FFF7E8FF094B1870B1
:10D660005A6801325A601A7822B95A6840F2FF1398
:10D670009A42F0D13120FFF7D9FF003018BF0120C6
:10D6800008BD00BFC0090020024B5A6A42F08072F8
:10D690005A62704700100240034B9B6818420CBF4F
:10D6A00000200120704700BF00100240014B18709D
:10D6B000704700BF0A10024008B5164B98421BD0B5
:10D6C00003F5744398420BD0A3F5784398421FD1D9
:10D6D0004FF480400121FFF78BFF4FF4804012E0B0
:10D6E0004FF480500121FFF777FFBDE808404FF469
:10D6F00080500021FFF770BF4FF400400121FFF779
:10D7000077FF4FF400400021BDE80840FFF770BFED
:10D7100008BD00BF003C00400B8810B54C88028853
:10D7200023438C8802F441522343CC8823430C8941
:10D7300023434C8923438C892343CC8923431343BC
:10D740009BB20380838B23F400631B041B0C838335
:10D750000B8A038210BD838BF0B523F47B6323F027
:10D760000F031B041B0C8383022303840B89868B0A
:10D77000022B87B005460C46B6B223D08B8801A891
:10D78000002B14BF02270127FFF7C0FEE388228980
:10D79000B3F5007F019B4FF00A011CBF7F017A4364
:10D7A00001FB03F308BF1202B3FBF2F305330A22B5
:10D7B0009BB2B3FBF2F303F001021202C3F34F0377
:10D7C00092B200E00022991E89B2FE2928BF0022F1
:10D7D000E18828BF022313430B439BB22B84238889
:10D7E0006288334343F400631343A288134362897E
:10D7F00013439BB2AB8307B0F0BD0023038043808B
:10D800008380C380038143818381C3810723038293
:10D81000704700230222038043808380C3800281FB
:10D8200043817047038819B19BB243F0400303E082
:10D8300023F040031B041B0C03807047838B19B13A
:10D840009BB243F4806303E023F480631B041B0C4E
:10D8500083837047090901238B409BB21AB18288E8
:10D8600092B2134303E0828892B222EA03038380D8
:10D87000704783889BB20AB1194301E023EA010192
:10D880008180704781817047808980B270474FF6F0
:10D89000FF639942038803D09BB243F4807303E093
:10D8A00023F480731B041B0C03807047838819B119
:10D8B0009BB243F0040303E023F004031B041B0C9E
:10D8C00083807047038823F400631B041B0C0380D0
:10D8D00003889BB219430180704703889BB243F4CD
:10D8E000805303807047038819B19BB243F40053FF
:10D8F00003E023F400531B041B0C03807047012931
:10D9000014BF008B808A80B27047008A80B2704753
:10D91000B1F5804F038803D19BB243F4804303E009
:10D9200023F480431B041B0C0380704703891942B6
:10D930000CBF002001207047202906D103890388ED
:10D940009BB243F0400303807047402901D008296F
:10D9500001D103897047C94389B20181704701F041
:10D960000F02012303FA02F210B584880089A4B2E1
:10D9700080B2104005D009098B401C420CBF00202A
:10D98000012010BD552906D1038903889BB243F0BD
:10D99000400303807047562901D0532901D10389E0
:10D9A000704701F00F01012303FA01F1C94389B265
:10D9B00001817047044B04281A680CBF42F004022E
:10D9C00022F004021A60704710E000E0014B58603A
:10D9D000704700BF10E000E00128084B03D11A682F
:10D9E00042F0010204E0023004D11A6822F0010280
:10D9F0001A60704700229A60704700BF10E000E094
:10DA0000044B1A6810B142F0020201E022F0020257
:10DA10001A60704710E000E0014B9868704700BF43
:10DA200010E000E0C308022B044B0CBF1B68DB684E
:10DA300023FA00F000F00100704700BF10E000E0A2
:10DA400030B5048C24F001042404240C0484058BD8
:10DA5000048CADB225F0F305A4B22A4324F00204ED
:10DA600042EA031344F001049DB22143058301847B
:10DA700030BD30B5048C24F010042404240C04843C
:10DA8000058B048C25F44075A4B22D052D0D24F0D2
:10DA9000200444F0100445EA022242EA033344EA37
:10DAA00001119BB28CB20383048430BD08B52E4BA8
:10DAB00098423AD010D8A3F50063984225D003F5D8
:10DAC000806398422BD0B0F1804F4CD101200146A9
:10DAD000FFF78EFD01201DE0244B984231D004D881
:10DAE000A3F58063984226D008BD214B984204D00C
:10DAF00003F5006398422AD008BD4FF4006001216D
:10DB0000FFF76AFD4FF4006028E002200121FFF7D3
:10DB10006FFD02200021BDE80840FFF769BD042029
:10DB20000121FFF765FD0420F4E708200121FFF73C
:10DB30005FFD0820EEE710200121FFF759FD1020BE
:10DB4000E8E720200121FFF753FD2020E2E74FF412
:10DB500000500121FFF740FD4FF400500021BDE8C7
:10DB60000840FFF739BD08BD000C0040001400401C
:10DB7000002C01400388CA8803F08F0303800388C8
:10DB80009BB213434A8813439BB203808B888385DF
:10DB90000B880385054B984203D003F50063984238
:10DBA00001D10B7A0386012383827047002C014048
:10DBB000038C70B523F001031B041B0C0384038C3E
:10DBC0008488028B0D8822F070021204120C4E8899
:10DBD0002A430D8923F002031B043543ADB21B0C0D
:10DBE0002B43CD88A4B285860D4DA84203D005F500
:10DBF0000065A8420FD14D8923F008032B438D887F
:10DC000023F004032B4347F6FF452540CC8989893F
:10DC10000C43A4B22C4384800283038470BD00BFF4
:10DC2000002C0140038C30B523F010031B041B0CA7
:10DC30000384038C8288048B0D8824F4E04424043C
:10DC4000240C23F0200344EA05241B040D891B0C3B
:10DC500043EA05134D8892B243EA0513CD88A4B276
:10DC60000587114D9BB2A84203D005F50065A84277
:10DC700016D14D8923F080039BB243EA05134FF67A
:10DC8000BF751D408B8845EA031347F2FF351540E9
:10DC90008A899BB245EA8205CA8945EA820292B224
:10DCA00082800483038430BD002C0140038C30B596
:10DCB00023F480731B041B0C0384038C8288848BE5
:10DCC0000D8824F070042404240C23F400732C43E6
:10DCD0001B040D891B0C43EA05234D8892B243EACD
:10DCE0000523CD889BB28587104DA84203D005F54A
:10DCF0000065A84216D14D8923F400639BB243EA24
:10DD000005234FF6FF351D408B8845EA032344F673
:10DD1000FF7515408A899BB245EA0215CA8945EA12
:10DD2000021292B282808483038430BD002C0140B1
:10DD3000038C30B523F480531B041B0C0384038C29
:10DD40008488828B0D8822F4E0421204120C23F4A2
:10DD5000005342EA05221B040D891B0C43EA0533DC
:10DD60004D88A4B243EA0533CD8892B2A0F8405062
:10DD7000084D9BB2A84203D005F50065A84205D125
:10DD80008989C4F30D0444EA8114A4B28480828397
:10DD9000038430BD002C01404A880B8813438A88D5
:10DDA0001343CA8813430A8913434A8913438A8950
:10DDB00013439BB2A0F8443070474FF6FF73838043
:10DDC00000230380C38043800372704700230380D5
:10DDD00043808380C380038143818381C3817047F3
:10DDE00000230122038043808280C3800381704727
:10DDF0000023038043808380C38003814381838128
:10DE00007047038819B19BB243F0010303E023F08C
:10DE100001039B059B0D03807047B0F8443029B186
:10DE20006FEA43436FEA53439BB201E0C3F30E032F
:10DE3000A0F84430704783899BB20AB1194301E0CE
:10DE400023EA010181817047818270470A43A0F86B
:10DE50004820704783899BB20AB1194301E023EA45
:10DE6000010181817047038923F007031B041B0C08
:10DE700003817047038923F070031B041B0C1943B3
:10DE8000018103899BB243F007030381704738B5D2
:10DE90000D46602D114604464FF0010202D1FFF7F6
:10DEA000E8FD01E0FFF7CCFD238923F070031B049C
:10DEB0001B0C2B43238123899BB243F0070323814F
:10DEC00038BD10B5048942EA0323E4B21C43A4B26E
:10DED0002143018110BD10B50446FFF7F2FF2389ED
:10DEE00023F077031B041B0C43F07703238110BD41
:10DEF00010B50446FFF7E5FF23899BB243F4804346
:10DF0000238110BD018582827047038823F070034E
:10DF10009B059B0D194301807047038923F0700313
:10DF20001B041B0C19430181704770B50589048BD4
:10DF3000068C24F44074B6B224F0030426F02206C2
:10DF400025F00705240432432D04240C2D0C44F441
:10DF5000807442EA0313294344F001049EB2018114
:10DF60000483068470BD038B23F070031B041B0C19
:10DF7000194301837047038B23F4E0431B041B0CFC
:10DF800043EA01218BB203837047838B23F0700334
:10DF90001B041B0C194381837047838B23F4E043DC
:10DFA0001B041B0C43EA01218BB283837047038857
:10DFB00019B19BB243F0800303E023F080039B057B
:10DFC0009B0D03807047838819B19BB243F0040313
:10DFD00003E023F004031B041B0C83807047838839
:10DFE00019B19BB243F0080303E023F008031B04BC
:10DFF0001B0C83807047838819B19BB243F00103E7
:10E0000003E023F001031B041B0C83807047038B88
:10E0100023F008031B041B0C194301837047038B77
:10E0200023F400631B041B0C43EA01218BB203831E
:10E030007047838B23F008031B041B0C1943818357
:10E040007047838B23F400631B041B0C43EA0121FC
:10E050008BB283837047038B23F004031B041B0CD8
:10E06000194301837047038B23F480631B041B0C4B
:10E0700043EA01218BB203837047838B23F00403AF
:10E080001B041B0C194381837047838B23F480632B
:10E090001B041B0C43EA01218BB283837047038B63
:10E0A00023F080031B041B0C194301837047038B6F
:10E0B000C3F30E0343EA01218BB203837047838BC2
:10E0C00023F080031B041B0C194381837047838B4F
:10E0D000C3F30E0343EA01218BB283837047038CA1
:10E0E00023F002031B041B0C194301847047038CAB
:10E0F00023F008031B041B0C194301847047038C95
:10E1000023F020031B041B0C43EA01118BB2038490
:10E110007047038C23F080031B041B0C43EA01119E
:10E120008BB203847047038C23F400731B041B0C15
:10E1300043EA01218BB203847047038C23F400630C
:10E140001B041B0C43EA01218BB203847047038C30
:10E1500023F400531B041B0C43EA01318BB20384EC
:10E16000704701238B408A4010B5048CA4B224EA86
:10E1700003030384038C13439BB2038410BD042365
:10E180008B408A4010B5048CA4B224EA03030384B4
:10E19000038C13439BB2038410BD01238B4010B545
:10E1A000048C1830A4B224EA0303038121F008038D
:10E1B0003BB9490844584FF68F73234043504358A6
:10E1C0000AE00439C1F34E01445848F6FF73234076
:10E1D00043501202435892B21A43425010BD038872
:10E1E00019B19BB243F0020303E023F002039B0545
:10E1F0009B0D03807047038819B19BB243F0040361
:10E2000003E023F004039B059B0D03807047838884
:10E2100019B19BB243F0800303E023F080031B0499
:10E220001B0C83807047038823F008039B059B0D1C
:10E23000038003889BB2194301807047838823F0D1
:10E2400070031B041B0C838083889BB2194381805D
:10E250007047038923F007031B041B0C0381038908
:10E260009BB2194301817047038923F080031B048B
:10E270001B0C038103899BB2194301817047818480
:10E280007047818570478186704701877047818715
:10E290007047A0F840107047038B23F00C031B0459
:10E2A0001B0C0383038B9BB2194301837047038BC1
:10E2B00023F440631B041B0C0383038B9BB243EAD0
:10E2C00001218BB203837047F8B50C464988A288B8
:10E2D0000029B4F800E014BF00270227012A0546F0
:10E2E00014BF012602262389BEF1000F11D1FFF7CA
:10E2F000A7FB2846E188FFF7CFFF2846394632467C
:10E300002389FFF7B6FB2846E188BDE8F840FFF710
:10E31000CEBFFFF7AEFB2846E188FFF7C8FF2846CF
:10E32000394632462389FFF78BFB2846E188BDE852
:10E33000F840FFF7B1BF838B23F00C031B041B0CC9
:10E340008383838B9BB2194381837047838B23F430
:10E3500040631B041B0C8383838B9BB243EA012124
:10E360008BB283837047F8B50E880D460446498802
:10E37000AA882B893EB9FFF763FB2046E988BDE8F0
:10E38000F840FFF789BF042E07D1FFF772FB204644
:10E39000E988BDE8F840FFF78ABF082EEF88068CB1
:10E3A0001CD126F480763604360C0684858B068CC8
:10E3B000ADB225F0F30545EA0313B6B29BB21A439A
:10E3C00026F4007343EA012189B241F4807182830B
:10E3D00001843946BDE8F840FFF7ADBF26F480560A
:10E3E0003604360C0684858B068C25F440752D0585
:10E3F000B6B22D0D45EA022526F4005242EA01315B
:10E4000045EA033389B29BB241F48051838301848E
:10E410003946BDE8F840FFF799BF0388DBB20380B7
:10E4200003889BB2194301807047808E80B2704789
:10E43000008F80B27047808F80B27047B0F8400084
:10E4400080B27047808C80B27047008D80B2704778
:10E45000038A19420CBF002001207047C94389B2CA
:10E4600001827047038A828911EA030092B203D0C5
:10E4700011420CBF002001207047C94389B20182BC
:10E48000704700BF08B5224B98422CD008D8A3F59E
:10E490000063984217D003F5806398421BD008BDF3
:10E4A0001C4B984227D003F5684398422FD14FF474
:10E4B00080400121FFF790F8BDE808404FF480400C
:10E4C0000021FFF789B84FF400300121FFF790F8E1
:10E4D0004FF4003016E04FF480200121FFF788F858
:10E4E0004FF480200EE04FF400200121FFF780F868
:10E4F0004FF4002006E04FF480100121FFF778F878
:10E500004FF480100021BDE80840FFF771B808BD46
:10E51000004C004000500040038ACA889BB223F49C
:10E520004053134330B503820D4682890989AB8875
:10E5300092B20B43698922F4B0520B4322F00C02D1
:10E5400013439BB28381838AAA899BB223F44073CD
:10E5500087B013430446838201A8FEF7D7FF049ACD
:10E56000039B0E498C4208BF134619214B432A686E
:10E570009200B3FBF2F16423B1FBF3F21201100934
:10E5800003FB101109013231B1FBF3F303F00F0368
:10E590001A4392B2228107B030BD00BF003801405B
:10E5A0004FF4165303600C2200238380C380038141
:10E5B0004281838170470B8810B54C88028A2343BF
:10E5C0008C88C98892B223430B4322F470621343B0
:10E5D0009BB2038210BD0023038043808380C380ED
:10E5E0007047838919B19BB243F4005303E023F4CD
:10E5F00000531B041B0C83817047C1F3421310B5F9
:10E60000012401F01F01A34204FA01F101D10C30F1
:10E6100003E0022B0CBF1030143003680AB1194319
:10E6200001E023EA0101016010BD838A9BB20AB1B7
:10E63000194301E023EA010181827047038A23F034
:10E640000F031B041B0C0382038A9BB21943018234
:10E650007047838923F400631B041B0C8381838927
:10E660009BB2194381817047838919B19BB243F0F2
:10E67000020303E023F002031B041B0C8381704799
:10E68000038A23F020031B041B0C0382038A9BB222
:10E69000194301827047038A19B19BB243F4804346
:10E6A00003E023F480431B041B0C03827047C1F377
:10E6B0000801818070478088C0F308007047838913
:10E6C0009BB243F0010383817047038BDBB203836A
:10E6D000038B9BB243EA012101837047038B03F450
:10E6E0007F430383038B9BB2194301837047838A63
:10E6F00019B19BB243F0200303E023F020031B0475
:10E700001B0C83827047838A19B19BB243F01003BC
:10E7100003E023F010031B041B0C83827047838AE1
:10E7200019B19BB243F0080303E023F008031B0474
:10E730001B0C83827047838A23F004031B041B0C89
:10E740008382838A9BB2194381827047838A19B17D
:10E750009BB243F0020303E023F002031B041B0CF3
:10E7600083827047038819420CBF00200120704744
:10E77000C94389B20180704710B5C1F3421401F05A
:10E780001F030122012C02FA03F201D1838903E065
:10E79000022C0CBF038A838A9BB21340028892B278
:10E7A00043B10123090A03FA01F111420CBF002011
:10E7B000012010BD184610BD090A01238B40DB4320
:10E7C0009BB20380704700BF684620F007018D466A
:10E7D00001B500230B4A0C499818884204D20B4912
:10E7E000595899500433F5E7094B0A4A934203D22A
:10E7F000002243F8042BF8E702F0A4FBBDE8014037
:10E80000854670470000002064050020241B010895
:10E81000680500208011002010B5064C18B9236847
:10E8200001221A8210BD044B1B681B6898472068A0
:10E830000A3010BD1C110020D810002010B5064C65
:10E8400018B9236801221A8210BD044B1B689B680B
:10E85000984720680C3010BD1C110020D8100020F3
:10E8600010B5204B18B91B6802221A8210BD1E4A2F
:10E870001968002010800C78134614F07F040DD125
:10E880004A7A910644BF0221197012F0400F1A789B
:10E8900014BF22F0010242F0010214E0012C1FD04B
:10E8A000022C1ED1497901F00F02920002F1804240
:10E8B00002F5B84211F0800F126806D002F0300263
:10E8C000102A07D101221A7004E002F44052B2F576
:10E8D000805FF6E7054B1B681B699847024810BD2F
:10E8E000104610BD1C11002078110020D810002007
:10E8F000234A2DE9F84314689046238A267A214F4B
:10E90000A3B9042E12D120490A78012A0AD11F4A3C
:10E9100010681F4A80B202445200136030223A80CD
:10E920000B7027E010233B80072623E0A58AAB422B
:10E930008CBF022604269D4228BF1D462846A36997
:10E9400098478146002000F06BFE2A460146484663
:10E9500000F06EFC2946002000F07EFE238A4FF472
:10E9600040525B1B2382638A1D4430233B80094B4A
:10E9700065821A80D8F800301E72BDE8F88300BFA7
:10E980001C1100207C110020C8090020505C0040B0
:10E99000023000207A11002010B50A4B0A491B688A
:10E9A0004978DA7891420AD3997841B99C8834B988
:10E9B0009A72064B1B685B689847204610BD022080
:10E9C00010BD00BF1C110020D8000020D81000206E
:10E9D00038B50E4A0E4C1268236892695879D97876
:10E9E000904723689A7A7AB170B91A7962B99D789A
:10E9F00055B9084B1B68DB689847236828465A7945
:10EA0000DA72DA781A7338BD022038BDB4100020EB
:10EA10001C110020D810002038B52F4B1B68187827
:10EA200010F07F0004D15A7A22F020025A7238BDC9
:10EA300002284ED15A88002A4CD11A79002A49D18D
:10EA40005A79264D22F08000840004F1804101F5BE
:10EA5000B84109682D7812F0800F14BF01F0300121
:10EA600001F44051A84234D2002932D09B7A83B3BA
:10EA700004F1804404F5B844120623680CD503F071
:10EA80003003102B1FD1C4B2204600F080FD204679
:10EA9000302100F055FC16E003F44053B3F5805FDD
:10EAA00011D128B90E4B93F82C1000F0F6FD01E0BF
:10EAB00000F05DFD236823F4804323F070039BB2D4
:10EAC00083F440532360074B1B685B699847002021
:10EAD00038BD022038BD00BF1C110020D800002026
:10EAE00050000020D810002038B51D4B1D4D19686E
:10EAF0002D784A7922F08004A30003F1804000F5CC
:10EB0000B840006812F0800F14BF00F0300000F42D
:10EB10004050AC4222D24C8804BBF8B1897AE9B1AA
:10EB200003F1804303F5B84312F0800F1A6807D051
:10EB300022F4E04222F0400292B282F0100206E09B
:10EB400022F4804222F0700292B282F480521A6063
:10EB5000054B1B689B699847002038BD022038BDD3
:10EB60001C110020D8000020D810002008B5064B4A
:10EB70001B685A7A42F020025A72044B1B68DB6908
:10EB80009847002008BD00BF1C110020D8100020AD
:10EB9000054B1A68538A18B98988CB1A13827047B3
:10EBA00008681844704700BF1C11002008B50B4BC3
:10EBB000002093F82C1000F070FD094B1B68187AA8
:10EBC000082806D1074B4FF480521A80064B1022BA
:10EBD0001A80B0F109035842584108BD5000002086
:10EBE0001C1100207A1100207C110020F7B5914FF4
:10EBF000914B3A68914D92B213442E685B001C68A9
:10EC0000337A092B15D0A4B2640004F1804404F5D2
:10EC1000C0442378337063787370A08800F0E8FEF6
:10EC2000708020892E6800F0E3FEB080A2892B68F6
:10EC3000DA802B6801221A72DA885C78002A61D1A6
:10EC40001A7812F07F023AD1092C02D1FFF7A4FE04
:10EC500044E0052C0FD193F90320002A01DA0823A0
:10EC60004DE09A78002AFAD19A88002AF7D19B7A47
:10EC7000002B37D0F3E7032C13D1DA78012A07D021
:10EC80006F4B20461B685B699847032828D135E005
:10EC90009A88002AF4D15B7A9806F1D5FFF766FFCF
:10ECA0001CE0012CECD1DA78012AE9D19A88002AFB
:10ECB000E6D15B7A9906E3D5FFF7AEFE0EE0012AB6
:10ECC00004D10B2CDCD1FFF783FE07E0022AD7D159
:10ECD000012CF1D0032CD3D1FFF706FF10B1CFE701
:10ECE0000028BCD13A68574B92B213445B00002213
:10ECF0001A60554B30221A80062300E009232A6847
:10ED00001372D0E0062C13D11A78520678D19A7873
:10ED10004B4B012A02D11B68DB6968E0022A02D151
:10ED20001B681B6A63E0032A6AD11B685B6A5EE0AA
:10ED3000002C3DD15988002962D15A6822F47F42C3
:10ED4000B2F5003F5CD11A7812F07F0204D19B88A3
:10ED5000002B00F0AC8053E0012A0DD1384A5879DD
:10ED600012689269904700284AD1344B1B689B7AFD
:10ED7000002B40F09C8043E0022A41D15B7933486C
:10ED800003F00F018A0002F1804202F5B8421268D6
:10ED9000007813F0800F14BF02F0300202F44052EA
:10EDA00081422DD213F0700F2AD1002A7FD127E0A3
:10EDB000082C03D11B785B067BD021E00A2C1FD1E5
:10EDC0001A7802F07F02012A1AD19A7AC2B15988C0
:10EDD000B1B95A6822F47F42B2F5803F10D1184A87
:10EDE0005879126892699047002864D008E03BB1D6
:10EDF0002A680024548293612046984720460AE0FE
:10EE00000F4B1A682B68126958789047032802D173
:10EE10000A4B1B6805E02B684FF6FF711A8A8A427D
:10EE200001D1092203E0022800D08AB908221A720F
:10EE300039E000BF505C0040043000201C1100206D
:10EE4000B4100020023000207C110020D8000020E7
:10EE500093F90010002920DAD988019101988242A3
:10EE6000164802D9019A1A8210E08A420ED201682D
:10EE700091F82C108A4201D2002105E092FBF1F4B6
:10EE800001FB142212B901210D4A1170026892F897
:10EE90002C209A82FFF72CFD05E003221A72094B01
:10EEA0004FF440521A80FFF781FE03B0F0BD064BCD
:10EEB0009EE7064B9CE7064B9AE700BFB410002084
:10EEC000C80900207A11002061E8000819E800084C
:10EED0003DE80008F8B52B4D2C68237A032B01D0B0
:10EEE000052B41D1A369228AABB1A2B1A68A964271
:10EEF00028BF164630469847238A07469B1B238225
:10EF0000638A00203344638200F098FB3246014656
:10EF1000384600F0A5F9238A53B11B4B00204FF46B
:10EF2000405201461A8000F097FB184B30221A809D
:10EF3000238AA28A9A4202D82B68032202E01BB1DC
:10EF40002B6805221A720CE02A6806211172104AF9
:10EF50001168104A89B20A44520013600B4B3022E8
:10EF60001A802B681B7A06E0072B03D10A4B1B681B
:10EF7000DB68984708232A681372BDE8F840FFF75A
:10EF800015BE00BF1C1100207A1100207C1100204A
:10EF9000505C004002300020B410002030B50B4B14
:10EFA0001C780023A3420CD203F1805202F5B85220
:10EFB00091000D6848F68F722A401A430A600133A7
:10EFC000F0E7034B40F08000186030BDD80000200F
:10EFD0004C5C004010B5134C23681A7A022A01D009
:10EFE000042A04D1FFF784FC23681B7A13E0062A65
:10EFF00010D15A78052A09D11A78520606D1D87844
:10F00000FFF7CCFF084B1B681B6A9847074B1B6830
:10F010009B689847082322681372BDE81040FFF7E9
:10F02000C5BD00BF1C110020D8100020B410002066
:10F03000704700BF08B5074A074B08491360022212
:10F040001A72074B074A1360074A1B6811609847FA
:10F0500008BD00BF1C110020BC100020B40000201F
:10F0600050000020B4100020D810002070B54C4A89
:10F070004C4B116888B20C04188040F1908047F620
:10F08000FF7111601A88484C02F00F022270002AAA
:10F090005FD1464C464D2268464E02F440522A80CB
:10F0A000226802F030023280226822F4804222F08C
:10F0B000700292B282F400522260226822F4E0428E
:10F0C00022F0400292B282F0200222601B88D80611
:10F0D00002D52368190607D5226848F60F73134036
:10F0E0002360FFF777FF12E01A0507D5226840F684
:10F0F0008F7313402360FFF779FD08E01804B6D53D
:10F10000226840F68F7313402360FFF7E3FE236805
:10F110002A8823F4804323F070039BB2D10448BFB4
:10F1200083F480539504214A48BF83F4005313604D
:10F130001368318823F4E04323F040039BB2CC06EC
:10F1400048BF83F01003880648BF83F02003136094
:10F1500070BD930003F1804303F5B8431D68290493
:10F1600009D5186840F68F7101401960124B013AB9
:10F1700053F8223098472B067FF579AF217848F66F
:10F180000F728B0003F1804303F5B843186801390F
:10F1900002401A60094B53F82130984767E770BD69
:10F1A000445C0040B2100020B8100020005C004019
:10F1B0007A1100207C110020DC000020F8000020E3
:10F1C00008B5164A164B116888B20904188024D570
:10F1D00047F6FF7111601A88124B02F00F021A7085
:10F1E000930003F1804303F5B8431968080407D579
:10F1F000186840F68F7101401960013A0A4B08E027
:10F200000906DED5186848F60F7101401960074BF2
:10F21000013A53F822309847D3E708BD445C0040D8
:10F22000B2100020B8100020DC000020F800002000
:10F2300030B501F10051013201F540515210490041
:10F240000023934200F1020009D010F8015C10F88D
:10F25000024C44EA052421F823400133F1E730BD94
:10F2600010B501F10051013201F540515210490031
:10F270000023934205D051F8234020F81340013376
:10F28000F7E710BD014B1860704700BF405C0040BD
:10F29000014B186880B27047405C0040014B186019
:10F2A000704700BF445C0040014B186880B2704753
:10F2B000445C0040014B186880B27047485C0040D5
:10F2C000014B1860704700BF4C5C0040014B186850
:10F2D00080B270474C5C00404FF6F873014A03401F
:10F2E00013607047505C0040014B186880B2704753
:10F2F000505C0040800000F1804000F5B8400160A3
:10F300007047800000F1804000F5B840006880B28E
:10F310007047800000F1804000F5B840036823F496
:10F32000EC4323F0700319438BB2036070478000F5
:10F3300000F1804000F5B840006800F4C0607047FC
:10F34000800000F1804000F5B8400368CA0623F44D
:10F35000E04323F040039BB248BF83F010038A06CA
:10F3600048BF83F0200303607047800000F18040B5
:10F3700000F5B8400368CA0423F4804323F0700307
:10F380009BB248BF83F480538A0448BF83F4005380
:10F3900003607047800000F1804000F5B84001290B
:10F3A000026802D14EF6FF7303E0022903D14FF643
:10F3B000EF73134003607047800000F1804000F558
:10F3C000B840006800F030007047800000F18040D5
:10F3D00000F5B840006800F440507047800000F12C
:10F3E000804000F5B840036823F4E04323F0400375
:10F3F0009BB283F0300303607047800000F18040CF
:10F4000000F5B840036823F4804323F070039BB2F7
:10F4100083F4405303607047800000F1804000F5A2
:10F42000B840036823F4E04323F0700343F480738F
:10F430009BB203607047800000F1804000F5B84047
:10F44000036823F4E24323F070031B041B0C0360E6
:10F450007047800000F1804000F5B840036823F455
:10F46000E24323F070031B041B0C03607047800011
:10F4700000F1804000F5B840036823F4E04323F036
:10F48000700343F480739BB203607047800000F107
:10F49000804000F5B840036823F4E04323F0700394
:10F4A00043F480739BB203607047800000F180409A
:10F4B00000F5B840036823F4E24323F070031B0413
:10F4C0001B0C03607047800000F1804000F5B840DD
:10F4D000006800F03000B0F1100358425841704706
:10F4E000800000F1804000F5B840006800F4405012
:10F4F000B0F58053584258417047800000F1804079
:10F5000000F5B840036823F070031B051B0D036072
:10F510007047800000F1804000F5B840036823F494
:10F52000E14323F070031B041B0C03607047800051
:10F5300000F1804000F5B840036823F4E04323F075
:10F5400070031B041B0C43F480430360704780006E
:10F5500000F1804000F5B840036823F4E04323F055
:10F5600070031B041B0C43F04003036070478000D2
:10F5700000F1804000F5B84003685B0406D50268DE
:10F5800048F68F73134043F4804303607047800054
:10F5900000F1804000F5B84003685B0606D50268BC
:10F5A00048F68F73134043F04003036070478000B8
:10F5B00000F1804000F5B840036823F4E04323F0F5
:10F5C00070031B041B0C194301607047800000F19D
:10F5D000804000F5B840006800F00F007047074B0E
:10F5E00049081B6849009BB203EBC00000F10050C2
:10F5F00000F5405040000160704700BF505C004083
:10F60000054B49081B6849009BB203EBC000034B44
:10F6100003445B0019607047505C004004300020D8
:10F62000054B1B689BB203EBC00000F1005000F5D6
:10F630004050400000887047505C0040044B1B68FD
:10F640009BB203EBC000034B03445B001888704778
:10F65000505C004004300020044B1B689BB203EB5D
:10F66000C000034B03445B0019607047505C0040CE
:10F67000023000203E2909D94B09C90604BF03F115
:10F68000FF339BB29B0243F4004304E04B08CA07DC
:10F6900048BF01339B02036070470E4B3E291B6835
:10F6A0009BB203EBC0000C4B03444FEA430209D961
:10F6B0004B09C80604BF03F1FF339BB29B0243F41E
:10F6C000004304E04B08C90748BF01339B021360A5
:10F6D000704700BF505C004006300020054B1B689F
:10F6E0009BB203EBC000044B03445B001868C0F3FB
:10F6F00009007047505C004002300020054B1B6839
:10F700009BB203EBC000044B03445B001868C0F3DA
:10F7100009007047505C00400630002010B50B4CCB
:10F72000C000236849089BB2034403F1005303F56A
:10F7300040535B0049001960236852089BB218448B
:10F74000034B520003445B001A6010BD505C004044
:10F7500004300020064B49081B6849009BB203EBAC
:10F76000C00000F1005000F54050400001607047BB
:10F77000505C0040054B49081B6849009BB203EBF5
:10F78000C000034B03445B0019607047505C0040AD
:10F7900004300020054B1B689BB203EBC00000F156
:10F7A000005000F54050400000887047505C004019
:10F7B000044B1B689BB203EBC000034B03445B008C
:10F7C00018887047505C004004300020012910B5B3
:10F7D0002FD1254CC0002168244B89B201440B4431
:10F7E0003E2A4FEA43010AD9530912F01F0F04BF02
:10F7F00003F1FF339BB29B0243F4004305E053083F
:10F8000012F0010F18BF01339B020B6023683E2AE0
:10F810009BB21844164B03444FEA43031CD95109C9
:10F82000D00604BF01F1FF3189B2890241F40041E1
:10F8300017E0022917D10C49C0000C680B4BA4B289
:10F84000044423445B001A600B689BB21844084BC5
:10F8500003445B001A6010BD5108D20748BF013154
:10F860008902196010BD10BD505C004002300020BC
:10F870000630002001291BD1134B3E2A1B689BB286
:10F8800003EBC000114B03444FEA430109D953096C
:10F89000D00604BF03F1FF339BB29B0243F4004345
:10F8A00004E05308D20748BF01339B020B60704746
:10F8B000022908D1044B1B689BB203EBC000034B29
:10F8C00003445B001A607047505C00400230002027
:10F8D00001291BD1134B3E2A1B689BB203EBC000CE
:10F8E000114B03444FEA430109D95309D00604BF21
:10F8F00003F1FF339BB29B0243F4004304E053083F
:10F90000D20748BF01339B020B607047022908D120
:10F91000044B1B689BB203EBC000034B03445B002A
:10F920001A607047505C004006300020054B1B6891
:10F930009BB203EBC000044B03445B001868C0F3A8
:10F9400009007047505C004002300020054B1B68E6
:10F950009BB203EBC000044B03445B001868C0F388
:10F9600009007047505C0040063000200D4AC0007E
:10F9700013689BB2C1180C4B0B445B001B8813F43B
:10F980007C4F0DD113689BB21844084B03445B00B5
:10F990001B88C3F30903002B0CBF00200220704713
:10F9A00001207047505C00400630002002300020EB
:10F9B00001290BD1800000F1804000F5B8400268B9
:10F9C00048F68F73134043F040030CE002290BD13B
:10F9D000800000F1804000F5B840026848F68F735F
:10F9E000134043F480430360704741EA00207047AE
:10F9F000C3B2000A40EA0320704700BF81F0004113
:10FA000002E000BF83F0004330B54FEA41044FEA03
:10FA1000430594EA050F08BF90EA020F1FBF54EA9E
:10FA2000000C55EA020C7FEA645C7FEA655C00F03A
:10FA3000E2804FEA5454D4EB5555B8BF6D420CDD0B
:10FA40002C4480EA020281EA030382EA000083EA8E
:10FA5000010180EA020281EA0303362D88BF30BD2E
:10FA600011F0004F4FEA01314FF4801C4CEA113184
:10FA700002D0404261EB410113F0004F4FEA0333E3
:10FA80004CEA133302D0524263EB430394EA050F6E
:10FA900000F0A780A4F10104D5F1200E0DDB02FADD
:10FAA0000EFC22FA05F2801841F1000103FA0EF271
:10FAB000801843FA05F359410EE0A5F120050EF137
:10FAC000200E012A03FA0EFC28BF4CF0020C43FA68
:10FAD00005F3C01851EBE37101F0004507D54FF075
:10FAE000000EDCF1000C7EEB00006EEB0101B1F5C5
:10FAF000801F1BD3B1F5001F0CD349085FEA30000B
:10FB00004FEA3C0C04F101044FEA445212F5800F15
:10FB100080F09A80BCF1004F08BF5FEA500C50F1B2
:10FB2000000041EB045141EA050130BD5FEA4C0C95
:10FB3000404141EB010111F4801FA4F10104E9D11E
:10FB400091F0000F04BF01460020B1FA81F308BF15
:10FB50002033A3F10B03B3F120020CDA0C3208DDE1
:10FB600002F1140CC2F10C0201FA0CF021FA02F1BC
:10FB70000CE002F11402D8BFC2F1200C01FA02F12C
:10FB800020FA0CFCDCBF41EA0C019040E41AA2BF51
:10FB900001EB0451294330BD6FEA04041F3C1CDA19
:10FBA0000C340EDC04F11404C4F1200220FA04F039
:10FBB00001FA02F340EA030021FA04F345EA0301E3
:10FBC00030BDC4F10C04C4F1200220FA02F001FAA5
:10FBD00004F340EA0300294630BD21FA04F0294627
:10FBE00030BD94F0000F83F4801306BF81F48011C0
:10FBF0000134013D4EE77FEA645C18BF7FEA655C33
:10FC000029D094EA050F08BF90EA020F05D054EA04
:10FC1000000C04BF1946104630BD91EA030F1EBF09
:10FC20000021002030BD5FEA545C05D1400049410D
:10FC300028BF41F0004130BD14F580043CBF01F500
:10FC4000801130BD01F0004545F0FE4141F47001E6
:10FC50004FF0000030BD7FEA645C1ABF19461046C1
:10FC60007FEA655C1CBF0B46024650EA013406BFC2
:10FC700052EA033591EA030F41F4002130BD00BF81
:10FC800090F0000F04BF0021704730B54FF480643E
:10FC900004F132044FF000054FF0000150E700BFBF
:10FCA00090F0000F04BF0021704730B54FF480641E
:10FCB00004F1320410F0004548BF40424FF000010B
:10FCC0003EE700BF42004FEAE2014FEA31014FEA4E
:10FCD00002701FBF12F07F4393F07F4F81F060519D
:10FCE000704792F0000F14BF93F07F4F704730B50C
:10FCF0004FF4607401F0004521F0004120E700BF9F
:10FD000050EA010208BF704730B54FF000050AE025
:10FD100050EA010208BF704730B511F0004502D526
:10FD2000404261EB41014FF4806404F132045FEA28
:10FD3000915C3FF4DCAE4FF003025FEADC0C18BFCD
:10FD400003325FEADC0C18BF033202EBDC02C2F1C3
:10FD5000200300FA03FC20FA02F001FA03FE40EA55
:10FD60000E0021FA02F11444C1E600BF70B54FF055
:10FD7000FF0C4CF4E06C1CEA11541DBF1CEA135537
:10FD800094EA0C0F95EA0C0F00F0DEF82C4481EA9F
:10FD9000030621EA4C5123EA4C5350EA013518BFBF
:10FDA00052EA033541F4801143F4801338D0A0FBAC
:10FDB00002CE4FF00005E1FB02E506F00042E0FB59
:10FDC00003E54FF00006E1FB03569CF0000F18BF5F
:10FDD0004EF0010EA4F1FF04B6F5007F64F5407407
:10FDE00004D25FEA4E0E6D4146EB060642EAC6219A
:10FDF00041EA55514FEAC52040EA5E504FEACE2E07
:10FE0000B4F1FD0C88BFBCF5E06F1ED8BEF1004F09
:10FE100008BF5FEA500E50F1000041EB045170BD85
:10FE200006F0004646EA010140EA020081EA0301C9
:10FE3000B4EB5C04C2BFD4EB0C0541EA045170BDC5
:10FE400041F480114FF0000E013C00F3AB8014F13F
:10FE5000360FDEBF002001F0004170BDC4F1000488
:10FE6000203C35DA0C341BDC04F11404C4F1200509
:10FE700000FA05F320FA04F001FA05F240EA020064
:10FE800001F0004221F0004110EBD37021FA04F69A
:10FE900042EB06015EEA430E08BF20EAD37070BD54
:10FEA000C4F10C04C4F1200500FA04F320FA05F0B3
:10FEB00001FA04F240EA020001F0004110EBD370B5
:10FEC00041F100015EEA430E08BF20EAD37070BD25
:10FED000C4F1200500FA05F24EEA020E20FA04F3FE
:10FEE00001FA05F243EA020321FA04F001F00041AD
:10FEF00021FA04F220EA020000EBD3705EEA430E1E
:10FF000008BF20EAD37070BD94F0000F0FD101F04C
:10FF10000046400041EB010111F4801F08BF013C85
:10FF2000F7D041EA060195F0000F18BF704703F0C3
:10FF30000046520043EB030313F4801F08BF013D4A
:10FF4000F7D043EA0603704794EA0C0F0CEA135506
:10FF500018BF95EA0C0F0CD050EA410618BF52EAC0
:10FF60004306D1D181EA030101F000414FF00000C6
:10FF700070BD50EA410606BF1046194652EA4306D4
:10FF800019D094EA0C0F02D150EA013613D195EA48
:10FF90000C0F05D152EA03361CBF104619460AD190
:10FFA00081EA030101F0004141F0FE4141F470019A
:10FFB0004FF0000070BD41F0FE4141F4780170BD8A
:10FFC00070B54FF0FF0C4CF4E06C1CEA11541DBFEF
:10FFD0001CEA135594EA0C0F95EA0C0F00F0A7F8F1
:10FFE000A4EB050481EA030E52EA03354FEA01311E
:10FFF00000F088804FEA03334FF0805545EA131331
:020000040801F1
:1000000043EA12634FEA022245EA111545EA1065F8
:100010004FEA00260EF000419D4208BF964244F18F
:10002000FD0404F5407402D25B084FEA3202B61AAE
:1000300065EB03055B084FEA32024FF480104FF482
:10004000002CB6EB020E75EB030E22BFB61A7546F6
:1000500040EA0C005B084FEA3202B6EB020E75EB89
:10006000030E22BFB61A754640EA5C005B084FEAF1
:100070003202B6EB020E75EB030E22BFB61A7546BE
:1000800040EA9C005B084FEA3202B6EB020E75EBC9
:10009000030E22BFB61A754640EADC0055EA060E8A
:1000A00018D04FEA051545EA16754FEA06164FEACD
:1000B000C30343EA52734FEAC2025FEA1C1CC0D179
:1000C00011F4801F0BD141EA00014FF000004FF006
:1000D000004CB6E711F4801F04BF01430020B4F1C7
:1000E000FD0C88BFBCF5E06F3FF6AFAEB5EB030C7F
:1000F00004BFB6EB020C5FEA500C50F1000041EB7C
:10010000045170BD0EF0004E4EEA113114EB5C0448
:10011000C2BFD4EB0C0541EA045170BD41F480111B
:100120004FF0000E013C90E645EA060E8DE60CEA23
:10013000135594EA0C0F08BF95EA0C0F3FF43BAF40
:1001400094EA0C0F0AD150EA01347FF434AF95EAF7
:100150000C0F7FF425AF104619462CE795EA0C0FDB
:1001600006D152EA03353FF4FDAE1046194622E7A8
:1001700050EA410618BF52EA43067FF4C5AE50EA82
:1001800041047FF40DAF52EA43057FF4EBAE12E772
:100190004FF0FF3C06E000BF4FF0010C02E000BF53
:1001A0004FF0010C4DF804CD4FEA410C7FEA6C5C36
:1001B0004FEA430C18BF7FEA6C5C1BD001B050EAD9
:1001C000410C0CBF52EA430C91EA030F02BF90EAC4
:1001D000020F0020704710F1000F91EA030F58BF83
:1001E000994208BF90422CBFD8176FEAE37040F0E5
:1001F000010070474FEA410C7FEA6C5C02D150EA83
:10020000013C07D14FEA430C7FEA6C5CD6D152EA3D
:10021000033CD3D05DF8040B704700BF8446104602
:1002200062468C461946634600E000BF01B5FFF701
:10023000B7FF002848BF10F1000F01BD4DF808EDD1
:10024000FFF7F4FF0CBF012000205DF808FB00BFA2
:100250004DF808EDFFF7EAFF34BF012000205DF8FC
:1002600008FB00BF4DF808EDFFF7E0FF94BF012049
:1002700000205DF808FB00BF4DF808EDFFF7CEFF4A
:1002800094BF012000205DF808FB00BF4DF808ED89
:10029000FFF7C4FF34BF012000205DF808FB00BF5A
:1002A0004FEA410212F5001215D211D56FF478739E
:1002B000B3EB625212D94FEAC12343F0004343EA41
:1002C000505311F0004F23FA02F018BF404270471C
:1002D0004FF00000704750EA013005D111F00040A6
:1002E00008BF6FF0004070474FF00000704700BF3C
:1002F0004FEA4102B2F1E04324BFB3F5001CDCF148
:10030000FE5C0DD901F0004C4FEAC0024CEA50707F
:10031000B2F1004F40EB830008BF20F001007047AE
:1003200011F0804F21D113F13872BCBF01F00040B1
:10033000704741F480114FEA5252C2F11802C2F1E3
:10034000200C10FA0CF320FA02F018BF40F0010064
:100350004FEAC1234FEAD32303FA0CFC40EA0C0016
:1003600023FA02F34FEA4303CCE77FEA625307D153
:1003700050EA01331EBF4FF0FE4040F4400070478A
:1003800001F0004040F0FE4040F40000704700BF24
:1003900080F0004002E000BF81F0004142001FBF3A
:1003A0005FEA410392EA030F7FEA226C7FEA236C43
:1003B0006AD04FEA1262D2EB1363C1BFD218414038
:1003C00048404140B8BF5B42192B88BF704710F0CE
:1003D000004F40F4000020F07F4018BF404211F071
:1003E000004F41F4000121F07F4118BF494292EAD9
:1003F000030F3FD0A2F1010241FA03FC10EB0C0005
:10040000C3F1200301FA03F100F0004302D5494291
:1004100060EB4000B0F5000F13D3B0F1807F06D33E
:1004200040084FEA310102F10102FE2A51D2B1F136
:10043000004F40EBC25008BF20F0010040EA03002B
:100440007047490040EB000010F4000FA2F10102D8
:10045000EDD1B0FA80FCACF1080CB2EB0C0200FA62
:100460000CF0AABF00EBC25052421843BCBFD040B0
:100470001843704792F0000F81F4000106BF80F42A
:1004800000000132013BB5E74FEA41037FEA226CED
:1004900018BF7FEA236C21D092EA030F04D092F0B8
:1004A000000F08BF0846704790EA010F1CBF0020EC
:1004B000704712F07F4F04D1400028BF40F0004049
:1004C000704712F100723CBF00F50000704700F069
:1004D000004343F0FE4040F4000070477FEA226290
:1004E00016BF08467FEA23630146420206BF5FEA61
:1004F000412390EA010F40F4800070474FF0000361
:1005000004E000BF10F0004348BF40425FEA000C27
:1005100008BF704743F0964301464FF000001CE0CF
:1005200050EA010208BF70474FF000030AE000BF25
:1005300050EA010208BF704711F0004302D5404263
:1005400061EB41015FEA010C02BF844601460020D5
:1005500043F0B64308BFA3F18053A3F50003BCFAF0
:100560008CF2083AA3EBC25310DB01FA02FC63449D
:1005700000FA02FCC2F12002BCF1004F20FA02F2A4
:1005800043EB020008BF20F00100704702F1200297
:1005900001FA02FCC2F1200250EA4C0021FA02F2F8
:1005A00043EB020008BF20EADC7070474FF0FF0CFD
:1005B0001CEAD0521EBF1CEAD15392EA0C0F93EAF8
:1005C0000C0F6FD01A4480EA010C400218BF5FEA9A
:1005D00041211ED04FF0006343EA501043EA51110D
:1005E000A0FB01310CF00040B1F5000F3EBF490007
:1005F00041EAD3715B0040EA010062F17F02FD2A0B
:100600001DD8B3F1004F40EBC25008BF20F00100ED
:10061000704790F0000F0CF0004C08BF49024CEA04
:10062000502040EA51207F3AC2BFD2F1FF0340EA96
:10063000C250704740F400004FF00003013A5DDC07
:1006400012F1190FDCBF00F000407047C2F1000248
:10065000410021FA02F1C2F1200200FA02FC5FEA35
:10066000310040F1000053EA4C0308BF20EADC707F
:10067000704792F0000F00F0004C02BF400010F4F1
:10068000000F013AF9D040EA0C0093F0000F01F09E
:10069000004C02BF490011F4000F013BF9D041EAC0
:1006A0000C018FE70CEAD15392EA0C0F18BF93EAC2
:1006B0000C0F0AD030F0004C18BF31F0004CD8D1EC
:1006C00080EA010000F00040704790F0000F17BF73
:1006D00090F0004F084691F0000F91F0004F14D0B9
:1006E00092EA0C0F01D142020FD193EA0C0F03D111
:1006F0004B0218BF084608D180EA010000F0004014
:1007000040F0FE4040F40000704740F0FE4040F4EE
:10071000400070474FF0FF0C1CEAD0521EBF1CEA8D
:10072000D15392EA0C0F93EA0C0F69D0A2EB0302AB
:1007300080EA010C49024FEA402037D04FF0805345
:1007400043EA111143EA10130CF000408B4238BF0A
:100750005B0042F17D024FF4000C8B4224BF5B1A18
:1007600040EA0C00B3EB510F24BFA3EB510340EA66
:100770005C00B3EB910F24BFA3EB910340EA9C0014
:10078000B3EBD10F24BFA3EBD10340EADC001B0184
:1007900018BF5FEA1C1CE0D1FD2A3FF650AF8B4228
:1007A00040EBC25008BF20F0010070470CF0004C35
:1007B0004CEA50207F32C2BFD2F1FF0340EAC25060
:1007C000704740F400004FF00003013A37E792F021
:1007D000000F00F0004C02BF400010F4000F013A7F
:1007E000F9D040EA0C0093F0000F01F0004C02BF7A
:1007F000490011F4000F013BF9D041EA0C0195E7E3
:100800000CEAD15392EA0C0F08D142027FF47DAF7B
:1008100093EA0C0F7FF470AF084676E793EA0C0F6B
:1008200004D14B023FF44CAF08466EE730F0004C69
:1008300018BF31F0004CCAD130F000427FF45CAFF9
:1008400031F000437FF43CAF5FE700BF4FF0FF3C67
:1008500006E000BF4FF0010C02E000BF4FF0010CBA
:100860004DF804CD4FEA40024FEA41037FEA226C83
:1008700018BF7FEA236C11D001B052EA530C18BFA5
:1008800090EA010F58BFB2EB030088BFC81738BF0A
:100890006FEAE17018BF40F0010070477FEA226CF8
:1008A00002D15FEA402C05D17FEA236CE4D15FEAF4
:1008B000412CE1D05DF8040B704700BF8446084628
:1008C0006146FFE70FB5FFF7C9FF002848BF10F1E9
:1008D000000F0FBD4DF808EDFFF7F4FF0CBF01202E
:1008E00000205DF808FB00BF4DF808EDFFF7EAFFB8
:1008F00034BF012000205DF808FB00BF4DF808ED73
:10090000FFF7E0FF94BF012000205DF808FB00BF67
:100910004DF808EDFFF7D2FF94BF012000205DF8ED
:1009200008FB00BF4DF808EDFFF7C8FF34BF0120FA
:1009300000205DF808FB00BF42000ED2B2F1FE4F6E
:100940000BD34FF09E03B3EB126209D44FEA00239E
:1009500043F0004323FA02F070474FF00000704765
:1009600012F1610F01D1420202D14FF0FF30704706
:100970004FF00000704700BF73B96AB9002908BF83
:100980000028BCBF00204FF00041C4BF6FF0004101
:100990004FF0FF3000F03CB882B0EC462DE900503B
:1009A00000F006F8DDF804E002B00CBC704700BFB0
:1009B0002DE9704F089E14461D468046894600F07A
:1009C00029F804FB01F3A4FB00AB00FB05329344C0
:1009D000B8EB0A0869EB0B09C6E90089BDE8708F1E
:1009E0002DE9704F089E14461D468046894600F04A
:1009F00061F900FB05F5A0FB04AB04FB0154A34423
:100A0000B8EB0A0869EB0B09C6E90089BDE8708FED
:100A1000704700BF00292DE9F00FC0F2A18000242B
:100A2000002BC0F29880154606460F46002B3FD19A
:100A30008A4258D9B2FA82F34BB1C3F1200201FACB
:100A400003F720FA02F29D4000FA03F61743290C3F
:100A5000B7FBF1F201FB1277A8B200FB02F34FEAF9
:100A6000164C4CEA0747BB4209D97F1902F1FF3CFB
:100A700080F00581BB4240F20281023A2F44FF1A06
:100A8000B7FBF1F301FB137100FB03F0B6B246EACA
:100A90000141884208D9491903F1FF3780F0F180FC
:100AA000884240F2EE80023B43EA0242002303E028
:100AB0008B420AD900231A461046194614B1404207
:100AC00061EB4101BDE8F00F7047B3FA83F8B8F16C
:100AD000000F40F088808B4202D3824200F2E28015
:100AE00000230122E8E712B90123B3FBF2F5B5FABE
:100AF00085F2002A3AD17F1B280C1FFA85FC0123BE
:100B0000B7FBF0F100FB11770CFB01F24FEA16483E
:100B100048EA0747BA4207D97F1901F1FF3802D2E4
:100B2000BA4200F2C4804146BF1AB7FBF0F200FBA4
:100B300012700CFB02FCB6B246EA0040844507D9AD
:100B4000401902F1FF3702D2844500F2AE803A46E6
:100B500042EA0142B0E7E443524263EB430362E7F7
:100B6000404261EB41014FF0FF3459E79540C2F13B
:100B7000200927FA09F126FA09F99740280CB1FB58
:100B8000F0F800FB18111FFA85FC0CFB08F349EA8A
:100B900007094FEA194747EA01418B4206FA02F674
:100BA00008D9491908F1FF327AD28B4278D9A8F1D5
:100BB00002082944C91AB1FBF0F300FB13170CFB20
:100BC00003F21FFA89F949EA0747BA4207D97F19A0
:100BD00003F1FF3160D2BA425ED9023B2F44BF1A03
:100BE00043EA08438CE7C8F1200225FA02F103FA30
:100BF00008FC27FA02F320FA02F207FA08F741EAA2
:100C00000C0C4FEA1C49B3FBF9F109FB11331FFA35
:100C10008CFA0AFB01FB17433A0C42EA03439B455B
:100C200005FA08F008D913EB0C0301F1FF3235D2B5
:100C30009B4533D902396344CBEB0303B3FBF9F291
:100C400009FB12330AFB02FABFB247EA0347BA456F
:100C500008D917EB0C0702F1FF331BD2BA4519D99B
:100C6000023A674442EA0145A5FB0001CAEB0707C7
:100C70008F424FF000030AD305D02A461CE7624694
:100C8000FDE63B4610E706FA08F68642F5D26A1EF4
:100C9000002311E71A46E5E70B46A0E71146CBE72C
:100CA000904687E74346424606E7023A50E7023954
:100CB0002F4439E72DE9F00F144605460E46002B68
:100CC00043D18A4253D9B2FA82F757B1C7F120060D
:100CD00020FA06F601FA07F302FA07F400FA07F51C
:100CE0001E43210CB6FBF1F201FB1266A0B200FB21
:100CF00002F32F0C47EA0646B34209D9361902F12E
:100D0000FF3780F0FD80B34240F2FA80023A264479
:100D1000F61AB6FBF1F301FB136100FB03F0ADB271
:100D200045EA0141884208D9091903F1FF3680F0EC
:100D3000E980884240F2E680023B43EA0242002317
:100D400010461946BDE8F00F70478B424CD8B3FAF5
:100D500083F6002E4FD18B4202D3824200F2DD8017
:100D6000BDE8F00F0023012210461946704712B962
:100D70000124B4FBF2F4B4FA84F2002A40F0828039
:100D8000091B260CA7B20123B1FBF6F006FB1011DC
:100D900007FB00F24FEA154C4CEA01418A4207D9A1
:100DA000091900F1FF3C02D28A4200F2C880604675
:100DB000891AB1FBF6F206FB121107FB02F7ADB27E
:100DC00045EA0145AF4208D92C1902F1FF3180F004
:100DD0009B80A74240F29880023A42EA00421046C5
:100DE0001946BDE8F00F704700231A461046194611
:100DF000BDE8F00F7047C6F1200522FA05F703FAA7
:100E000006F421FA05F301FA06FB20FA05F53C4346
:100E10004FEA1448B3FBF8FC08FB1C331FFA84F9B3
:100E200009FB0CFA45EA0B0B4FEA1B4545EA034365
:100E30009A4502FA06F204D91B190CF1FF356FD35B
:100E4000AC46CAEB0303B3FBF8F508FB153309FB0B
:100E500005F91FFA8BFB4BEA0347B94504D93F1943
:100E600005F1FF3362D31D4645EA0C4CACFB02236F
:100E7000C9EB07079F424FF000054AD346D06246B0
:100E80002B465DE79440C2F1200921FA09FC91400C
:100E900020FA09F9260CBCFBF6F806FB18CCA7B221
:100EA00007FB08F349EA01094FEA194141EA0C4CF2
:100EB000634500FA02F509D91CEB040C08F1FF3276
:100EC0003BD2634539D9A8F10208A444C3EB0C0C0A
:100ED000BCFBF6F306FB13C107FB03F21FFA89F90B
:100EE00049EA01418A4207D9091903F1FF3022D2A8
:100EF0008A4220D9023B2144891A43EA084343E746
:100F00003A4605E7334618E70A4666E7B04090429E
:100F1000B5D20CF1FF32002312E7334632460FE719
:100F20009A458DD9ACF1020C23448AE7B9459AD988
:100F3000023D274498E70346DEE79046C6E70238BD
:100F4000214435E7F7B5734EFCF716FA00244FF449
:100F500080303470FCF72EFAFCF77CFB0128054644
:100F600026D11020FBF728FD2046FCF771FA204619
:100F7000FCF782FA4FF48060FCF774FA4FF44030CB
:100F80004FF4E011FCF742FA2846FCF749FA392001
:100F9000FCF74CFB0028FAD00220FBF7F5FC0220FE
:100FA000FCF744FAFCF74CFA0828FBD10123337014
:100FB00004200121FCF7F8FA4FF48073ADF80430F7
:100FC000032301A98DF80630534818238DF8073004
:100FD000FBF773FF0620FCF723FB01200146FCF71B
:100FE000E3FA4FF0C0500121FCF7EAFA4B4C4FF402
:100FF00080414FF00060FCF70BF94FF44070FCF7B4
:101000005DF8474DF3F7E6F8F3F792FDF3F7B8F81C
:10101000F3F794FAF7F784FFF7F762FFF7F7ECF9C5
:10102000F3F7D6F92078F7F75BFAE078F7F7A4FB47
:101030002B7823B96079A1682269F7F7D7FC2B7860
:101040000BB1F8F7C5FAF8F747FDF3F7E7FCFAF745
:10105000E5FBF3F72DFDF3F743FDD0F101064FF06B
:10106000010038BF0026F3F77DFAF3F76FFBF6F7C0
:10107000CFFAF8F70FFBF9F76BF82A4B4FF4004261
:101080005A61F7F745FF0746F6F7C2FBF9F76CF828
:10109000F8F701FBF7F73CFFC01B0028B8BF404240
:1010A000B0F57A7F23DD2B7883B1F3F7A9FA68B91D
:1010B0001B4B1870F8F7A7FAF8F793FAF3F760F8F4
:1010C0006079A1682269F7F791FC0DE02B785BB994
:1010D000F3F796FA40B1F7F7C7FD114B01221A70EA
:1010E000F3F74EF8F8F774FAF7F712FF0746F3F73D
:1010F000DFFCF3F701FD0028C6D00EB1FAF78EFB36
:10110000F8F7EAFC0026F6F783FAF9F721F8F8F782
:10111000D9FAB9E7480F0020000801400800002074
:10112000580E00200010014000210A2200F0ACB847
:101130000F4B30B405461C6802E0D01A16D1ABB193
:1011400015F8013BE21850781A4600F00300012818
:1011500008BF03F1200211F8013BE018407800F0CD
:1011600003000128E9D12033D01AE9D030BC704700
:101170005C0500202DE9F00F424C82B0D4F800C08D
:1011800001900E4600E02646344614F8015B0CEB55
:101190000500407800F0080000F0FF0A0028F2D1B6
:1011A0002D2D5BD02B2D04BF7578B41C33F01000AF
:1011B0003CD09946BAF1000F0CBF6FF0004B4FF0D6
:1011C000004BBBFBF9F8002709FB18BB38460CE0C5
:1011D000303DAB4219DD7E1C05D0404523D820D0E0
:1011E00009FB0050012714F8015B0CEB050676782B
:1011F00016F0040FECD116F0030606D0012E14BF32
:1012000057263726AD1BAB42E5DC7B1C15D0BAF167
:10121000000F21D10AB1EFB9116002B0BDE8F00FA3
:1012200070475D45DCDD4FF0FF37DCE7302D1AD02D
:10123000002BBED10A239946BCE70199BAF1000FF1
:101240004FF022030CBF6FF000404FF000400B60E6
:10125000002AE2D0611EDFE74042DBE7B41C75786C
:101260004FF0010AA2E7207800F0DF00582803D0F1
:10127000002B9ED108239CE7102365789946023401
:1012800098E700BF5C05002030B4044C0D461346BF
:1012900001462A46206830BCFFF76CBF5805002085
:1012A0002DE9F0418AB004460D4600F06DF8DFF8F4
:1012B000D080064698F900300F4601330BD0204607
:1012C000294600F059FA30B1204629460022002371
:1012D000FEF7DCFF20B1304639460AB0BDE8F081A8
:1012E000234B98F800600890CDE90245CDE904450C
:1012F000019346BB1F4B4FF06042CDE906232046C9
:10130000294600220023FEF799FF70B102239E4276
:10131000009322D0684600F057FAF0B1089B0BBB4F
:10132000DDE906010AB0BDE8F0810123022E009339
:101330000ED0684600F048FA50B10F4800F046FA67
:10134000CDE90601EAE70D4B0022CDE90623D6E7F9
:1013500000F042FA21230360EFE700F03DFA222378
:101360000360DBE700F038FA089B0360D8E700BFB2
:10137000141B0108FFFFEFC7181B01080000F0FF56
:1013800060050020000000002DE9F04FB1F5801F3E
:1013900087B002460B460F465BDA21F00046064353
:1013A00000F0F5800029C0F2A4810022B24BFEF7C4
:1013B000DDFC0F460B46B14902468F426FF0350502
:1013C0004BDCC7F3130606F5152101F6647101F431
:1013D000801484F07F5181F4401141EA06031046E5
:1013E00019460022A64BFEF70DFB4FEA2758B31C07
:1013F000A8F2FF38C3F31303A844022B08EB1458D8
:1014000082468B464FF000022EDC0023FEF716FFCB
:10141000002800F0C580B8F1000F00F0718140464F
:10142000FEF73EFC80A3D3E9002306460F46FEF7F5
:101430009DFC7FA3D3E9002304460D463046394680
:10144000FEF794FC02460B4620462946FEF7DCFADE
:1014500007E08A4900258F42B3DD10461946FEF7A2
:10146000D3FA07B0BDE8F08F4FF08043FEF7CCFA17
:1014700002460B4650465946FEF7A2FDCDE9020151
:101480004046FEF70DFCCDE90401DDE9020102460C
:101490000B46FEF76BFC02460B46CDE90001FEF75A
:1014A00065FC65A3D3E9002304460D46FEF75EFC08
:1014B00063A3D3E90023FEF7A7FA22462B46FEF7E3
:1014C00055FC61A3D3E90023FEF79EFA22462B4682
:1014D000FEF74CFC5EA3D3E90023FEF795FADDE9A5
:1014E0000023FEF743FC5CA3D3E90023CDE9000110
:1014F00020462946FEF73AFC59A3D3E90023FEF71C
:1015000083FA22462B46FEF731FC57A3D3E900238A
:10151000FEF77AFA22462B46FEF728FC0B460246D7
:10152000DDE90001FEF770FAA6F5C223C6F5D7265D
:10153000A3F27A4351361E43002E04460D4657DD72
:101540000022504B50465946FEF710FC52465B466F
:10155000FEF70CFC06460F46B8F1000F40F09680EF
:1015600022462B46FEF750FADDE90223FEF7FEFB8A
:1015700002460B4630463946FEF744FA02460B4611
:1015800050465946FEF73EFA07B0BDE8F08F0022FC
:10159000002300203C49FEF713FD07B0BDE8F08FA3
:1015A00052465B4650465946FEF7E0FB30A3D3E96E
:1015B000002304460D4650465946FEF7D7FB024627
:1015C0000B4600202F49FEF71DFA02460B46204627
:1015D0002946FEF7CBFB04460D46B8F1000F40F05C
:1015E00092805046594622462B46FEF70BFA38E7C2
:1015F000B8F1000F00F0AB800BA3D3E90023DDE9C5
:101600000401FEF7B3FB22462B4606460F46504622
:101610005946FEF7F7F9DDE90223FEF7A7FB04467A
:101620000D46DDE904017CE00000E0FE422EE63FCD
:10163000763C7935EF39EA3D44523EDF12F1C23F44
:10164000DE03CB966446C73F599322942449D23F88
:10165000935555555555E53F9FC678D0099AC33FD8
:10166000AF788E1DC571CC3F04FA97999999D93FEF
:10167000555555555555D53F00005043FFFFEF7F59
:101680000000F03F0000E03F000050C336A3D3E964
:101690000023DDE90401FEF769FB22468046894606
:1016A0002B4630463946FEF7AFF9DDE90223FEF757
:1016B0005DFB2FA3D3E9002304460D46DDE90401B9
:1016C000FEF754FB02460B4620462946FEF79CF9DE
:1016D00002460B4630463946FEF794F952465B46C1
:1016E000FEF790F902460B4640464946FEF78AF956
:1016F000B7E6FEF787F900220023FEF761FCB0E6AB
:1017000000200021ADE64046FEF7CAFA16A3D3E951
:10171000002380468946FEF729FB06460F464046D1
:10172000494613A3D3E90023FEF720FB02460B46EC
:1017300020462946FEF766F952465B46FEF762F9F7
:1017400002460B4630463946FEF75CF989E602460A
:101750000B4650465946FEF755F9DDE90223FEF7E0
:1017600005FB0BE7AFF300800000E0FE422EE63FF2
:10177000763C7935EF39EA3D31F0004310B408D0BA
:101780000F4AA3F5801494420AD804205DF8044B54
:10179000704700280CBF022003205DF8044B7047FF
:1017A000B3F5801F01D20320F7E7064A934201D028
:1017B0000020F2E7D0F1010038BF0020EDE700BFC4
:1017C000FFFFDF7F0000F07F00207047002001490D
:1017D000704700BF0000F87F014B1868704700BFDA
:1017E00058050020F4010000640000000180080892
:1017F0000000000000640000000000000000000085
:10180000C80000000000000000000000010003E824
:101810000000000000000003E800000000000200DB
:10182000FA06000300000000003706000000000078
:101830000000000032035400720069006E00610075
:101840006D006900630020005300740065007000A3
:101850007000650072002000440065007600690099
:1018600063006500200026035400720069006E00CA
:1018700061006D00690063004D006F007400690035
:101880006F006E002000430074006C000403090424
:1018900009024300020100C03209040000010202F3
:1018A00001000524001001052401000104240202A6
:1018B0000524060001070582030800FF0904010052
:1018C000020A00000007050302400000070581022C
:1018D00040000012011001020000403C2A000101FA
:1018E0002A01020301524F5200000106524F4C00E0
:1018F0000002064D5354000003024D5650000004F0
:1019000007534150000005074741500000060353AC
:1019100054415000070352534150000803534750AD
:101920000000090747475000000A0353544750007E
:101930000B0352534750000C0352465300000D0353
:1019400053494F00000E0747494F00000F03534112
:101950004300001D0753434F00001E0747434F003D
:10196000001F0343434F0000200341434F00002763
:1019700003554630000040075546310000410755E9
:1019800046320000420755463300004307554634AF
:10199000000044075546350000450755463600000F
:1019A00046075546370000470752554E000081054F
:1019B00053544F5000800042494E00008B000000FD
:1019C0000000000000020000000000000100000014
:1019D00000010203040102030406070809020406C9
:1019E00008313134305631343200414253005245CF
:1019F0004C00434F4F5244005354415254005354EF
:101A00004F50005354415455530000004300000010
:101A100000202020202020202020282828282820BE
:101A200020202020202020202020202020202020B6
:101A3000208810101010101010101010101010101E
:101A4000100404040404040404040410101010100E
:101A500010104141414141410101010101010101D8
:101A6000010101010101010101010101101010102A
:101A700010104242424242420202020202020202AA
:101A800002020202020202020202020210101010FE
:101A90002000000000000000000000000000000026
:101AA0000000000000000000000000000000000036
:101AB0000000000000000000000000000000000026
:101AC0000000000000000000000000000000000016
:101AD0000000000000000000000000000000000006
:101AE00000000000000000000000000000000000F6
:101AF00000000000000000000000000000000000E6
:101B000000000000000000000000000000000000D5
:0C1B1000000000006C6F67000000000087
:081B1C00F8EEFF7F010000005C
:101B2400E1190108000100000001020000080000A2
:101B3400010000000200000000000000000000009E
:101B44000000000000000000000000000000000091
:101B54000000000000000000000000000000000081
:101B6400000000000000000000C2010000000800A6
:101B7400A9940008819200088191000895910008B9
:101B840097910008F1910008159200085D930008F0
:101B940069930008759300080000000040000000ED
:101BA400D318010812000000901801084300000037
:101BB4008C180108040000006618010826000000C3
:101BC4003418010832000000140100201A0000003B
:101BD4000100000031F000085D91000831F00008B8
:101BE40031F0000831F0000831F0000831F000084D
:101BF40031F00008759100080401000031F000087C
:101C040031F000085592000831F0000831F0000866
:101C140031F0000831F000085191000831F000085B
:101C240031F0000831F0000831F0000831F000080C
:101C340031F000081A0354004D00430053005400CF
:101C440045005000000000000000000000000000FB
:101C5400000000001C04002084040020EC04002088
:101C64000000000000000000000000000000000070
:101C74000000000000000000000000000000000060
:101C8400000000000C1A0108000000000000000021
:101C94000000000000000000000000000000000040
:101CA4000000000000000000000000000000000030
:101CB4000000000000000000000000000000000020
:101CC4000000000000000000000000000000000010
:101CD4000000000000000000000000000000000000
:101CE40000000000000000000000000000000000F0
:101CF40000000000000000000100000000000000DF
:101D04000E33CDAB34126DE6ECDE05000B000000A3
:101D140000000000000000000000000000000000BF
:101D240000000000000000000000000000000000AF
:101D3400000000000000000000000000000000009F
:101D4400000000000000000000000000000000008F
:10207400000000000000000030010020101A0108D8
:042084000100000057
:04000005080041109E
:00000001FF
